:10000000F01F00102D5D00002B5D00002B5D000037
:100010002B5D00002B5D00002B5D00000000000048
:100020000000000000000000000000002B5D000048
:100030002B5D0000000000002B5D0000F923000094
:100040000122000001220000012200000122000024
:100050000122000001220000012200000122000014
:100060000122000001220000012200000122000004
:1000700001220000295D0000295D0000C100000090
:10008000C1240000D9240000ED260000052700004F
:10009000295D000049280000295D0000295D00005D
:1000A000295D0000295D0000295D0000295D000038
:1000B000295D0000295D0000295D0000295D000028
:1000C000554B10B51A6801321A60544B1A68544BDC
:1000D000D2B2302A69D01ADC182A44D012DC082A9D
:1000E00032D0102A00D094E04E4A002111604E49CF
:1000F0000A68501C08604D49895C4D4AC9B21160BC
:10010000282287E0202A63D0282A32D081E0482A9A
:100110005ED004DC382A51D0402A53D079E0502AEE
:1001200060D0582A75D13F490A68501C0860404980
:1001300008684049C0B288543F4A0221FF3111602B
:1001400080221021D20563E0374A00211160116836
:10015000481C1060354A515C354AC9B211602822EA
:100160001A6001223CE030490A68501C08602F499F
:1001700009E02D4A314910680968884207D21168A0
:10018000481C1060294A515C294AC9B240E02C4AF7
:1001900011688022D205002901D0202138E02649AB
:1001A0000220FF300860102132E08022D2051021A9
:1001B000116008221A608122520011E08221490058
:1001C0001D4A25E01E4A1168042201291AD11DE0AA
:1001D0008022D2051021116008221A600422FF3209
:1001E000154B17E00F4A1168481C1060104804684E
:1001F0001048E4B244541068114A116804220139CD
:10020000884203D28021C9050A6002E01A6000E03A
:10021000116008221A6010BD640100100400004043
:100220001800004058010010600100108803001001
:1002300008000040780300105C01001098030010D3
:10024000740300101B4B02211A6810B50A431A6090
:10025000194B20211A68041C0A431A60174B1849CD
:100260001A680A401A601868012210431860154B7A
:1002700018680140196019680A431A60124B6C2211
:100280001A60124B1249186805F0D6FD114A106029
:10029000114A1060022C02D1104BA0221A60104BA0
:1002A000802212021A6080234022DB0501201A609E
:1002B00010BDC046048004408080044030400440AB
:1002C000F8FCFFFF34400440180000406C030010AD
:1002D000400D030014000040100000400C000040DE
:1002E00000E100E0034B1B689A06FBD5024B186047
:1002F0007047C0461480004000800040FFFFFFFFB1
:1003000008B502F0D7FE08BD70B5061C00200D1C14
:1003100001F06AFA002801D002F0BAFE00242C6035
:10032000301C3460291C01F08DFA201C01F05CFAAD
:10033000A04207D002F0ACFE2C60301C3460291CB7
:1003400001F080FA70BD08B502F086F808BD08B566
:1003500000230B60036001F075FA08BD10B502F0D0
:1003600055FE0D4B0020196802F036FA002002F00D
:1003700023FA002002F000FA084B01241C60084B0D
:10038000201C198802F0E4F8201C02F0D1F8201C8F
:1003900002F0AEF810BDC046680300105401001012
:1003A0007003001010B5062401200021013C02F06A
:1003B0001FF8002CF8D1FFF7D1FF10BD08B50020C1
:1003C00002F0EAF9012002F0A3F802F027FE08BDCE
:1003D00038B5051C0C1CFFF7C1FF054B0122281C7A
:1003E000211C5A6205F0B6F9FFF7E8FF38BDC04698
:1003F0001C1A001010B5041CFFF7B0FF201C05F0FC
:1004000077F9041CFFF7DAFF201C10BD08B50020A7
:10041000FFF7F0FF08BD000008B5021C02490348C1
:1004200002F038FC08BDC046185F0000105F0000F5
:1004300037B501F06FF80322164B1748002101F081
:1004400037F901F071F8FFF7E1FF1448FFF7E4FF17
:10045000134B144A00241A601D1C2B689C4211DAAD
:1004600002F0D4FA002803D001F0A6FD00240FE02A
:100470000A2001F0F1FF684601A9FFF745FF009B44
:10048000002B05D0FFF7C2FF074802F003FC37BD81
:100490000134E2E7E46A00001D5F00002C5F000009
:1004A0005802001070170000325F000070B58CB069
:1004B00000F0FBFF01F02EF8184D2B1C8C331C684C
:1004C000201C03F06BFC061C601C03F067FC221C64
:1004D00000901349331C02A802F0E8FB114C0121E3
:1004E0000A1C231C02A801F0E3F8231C0E4801217A
:1004F000092201F0DDF801F017F8FA24A4006420C5
:10050000013C01F0A9FF002CF9D12B1C8C332C6786
:1005100094351C602C600CB070BDC04624040010E3
:100520003D5F0000DC6A0000595F00001B4B73B5A3
:10053000041C1B49186805F07FFC1A4900901A4AF0
:100540001A4B201C02F0B2FB01F058FA002812D01E
:1005500001F070FAFA218900061C05F06DFC051CFB
:10056000201C02F0F4FB124B20186B431149F318C6
:100570002A1C02F09BFB201C02F0E9FB0E4B20180A
:100580001B68002B02D003DA0C4A02E00C4A00E0A0
:100590000C4A0D4902F08AFB73BDC0466C03001083
:1005A00040420F007C5F0000185F0000895F000080
:1005B00018FCFFFF8D5F000024000010795F000031
:1005C000765F000055600000985F000070B5051C64
:1005D0000E1C141C00F09EFF301C291C0022064B30
:1005E00001F066F8201C01210922044B01F060F89B
:1005F00000F09AFF70BDC046E46A0000DC6A0000AB
:10060000F0B58DB008AD002301242B700194FFF7E5
:10061000FDFE019A16012643362E06D0512E05D135
:1006200004A8364902F042FB05E0462604A83449F6
:10063000321C02F03BFB142004A92A1CFFF7C6FF62
:1006400096277F0002A803A9FFF75EFE0298002804
:100650003CD0C0B201F046F8021C512E06D0039BDC
:10066000002B03D1412E04D0412802D1FFF7CEFE4A
:1006700041E0B2421FD0281C224902F017FB039828
:1006800000280BD0C0B201F02DF80090281C02F019
:100690005EFB1D492818009A02F008FB04A92A1CD9
:1006A0001420FFF793FFFA204000C82103F006FB57
:1006B000FFF7ACFE0AE000261448642101342E70D6
:1006C00003F0FCFA0A2C0FD1341CA0E7029A002A8E
:1006D00002D0C82001F0C0FE04200321013F01F038
:1006E00087FE002FAED106E0631E5A425341019AA5
:1006F000D21801928BE70DB0F0BDC046A05F00009C
:10070000B65F0000B25F0000BF5F0000B80B0000E2
:1007100000B5084B89B01A78074B68461B78074923
:1007200002F0C4FA01206946054AFFF74FFF09B0FD
:1007300000BDC0461800001000000010C75F000098
:10074000D55F0000F0B52A4C2A4D237885B001937F
:100750002F78FFF7DDFFFFF759FE002602A803A957
:10076000FFF7D2FD029800282BD0C0B200F0BAFFEC
:1007700040280CD004D830280ED0392817D01BE0E0
:10078000462830D049280DD0412815D126E02B78B5
:100790003E2B11D8013303E02B78002B0CD0013B0A
:1007A0002B7009E02378062B06D8013303E0237869
:1007B000002B01D0013B237000F098FEFFF7A8FF4B
:1007C0000026029B002B02D0C82001F045FE042029
:1007D0000321013601F00CFE1D2EBFDD019B2F70A1
:1007E000237000F083FEFFF711FE05B0F0BDC04698
:1007F000000000101800001010B590B0041C6846EE
:10080000FFF794FE201C69466A46FFF7DFFE10B032
:1008100010BD000010B50E490E4A8AB0521A0B1CCA
:100820000D481C68844201D10433F9E7591A531A60
:10083000009102A8094902F039FA02AA01200849E8
:10084000FFF7C4FE3220002101F0D2FD0AB010BD36
:100850005C1A0010F01F00101DBAFE7AE95F00005C
:100860000160000000B52D228DB0002800D02B22A1
:1008700068460D4902F01AFA04A802F09BFC012018
:10088000694604AAFFF7A2FE0320002101F0B0FD93
:100890000220FFF7AFFD0028EED00A20002101F072
:1008A000A7FD0DB000BDC0460860000070B58CB05B
:1008B000FFF7ACFD02A8144902F052FA2E25FF35CD
:1008C00004AE301C02F076FC6846002409A9093009
:1008D000F47402F045FA02AA0420311CFFF776FEF8
:1008E000201C032101F084FD684601A901940094B5
:1008F000FFF70AFD009BA34202D1013DA542DFD1D3
:10090000FFF784FD0CB070BD56600000F0B5002408
:1009100093B00594FFF77AFD022296230194039287
:10092000251C5B00029300F0F5FD019B9A4F002B04
:100930006DD10AAE301C02F03DFC019AF2743274A3
:100940007273B272F2713271002C01D1012D05D196
:10095000301C042100223B1C00F0AAFE8F4E3B1CE1
:10096000301C1E21002200F0A3FE8B4F012C01D170
:10097000012D06D168462D30252100223B1C00F0B8
:1009800097FE301C332100223B1C00F091FE824E6A
:10099000022C09D1012D07D0684633304D210022A9
:1009A000331C00F085FE09E00CA83A210022331C1C
:1009B00000F07EFE032CEFD1012DEDD0784F331CDB
:1009C000381C5921002200F073FE734E042C01D113
:1009D000012D06D1684636305F210022331C00F01D
:1009E00067FE381C6C210022331C00F061FE052CD0
:1009F00001D1012D06D16846393072210022664BA3
:100A000000F056FE0FA804210922664B03E0664859
:100A1000042100223B1C00F04BFE00F085FD059BED
:100A2000002B0AD0143B012B05D8052C03D09620AF
:100A300001F012FD01E0FFF7E9FC0320011C01F0C9
:100A4000D7FC5A4B1E68002EF7D1301C00F0CCFEAC
:100A500006A9071C05A806960596FFF755FC059BF9
:100A6000002B72D007AE08AF301C391C09AA02F067
:100A7000D5FB019000286ED1301C03F04BF8051C0B
:100A800005981438032865D805F074F9230B02047F
:100A9000601C00E0601D062105F024FA00250C1CF6
:100AA00059E0052C56D8201C05F064F903060B0DFF
:100AB00010393388013316E0B0780C2105F0B2F913
:100AC00018E001355DE0387801301AE078780130BF
:100AD0001FE0052C3ED8201C05F04CF903070F1130
:100AE00019213388013B338044E0B0780C210A306F
:100AF00005F0F8F90131B1703CE0013D41E0387892
:100B00001730182105F0EEF9042239703FE07878AB
:100B10003B303C2105F0E6F9032379702FE00023F8
:100B2000BB70281C072105F0DDF9301C0A1C099157
:100B3000391C052C02D102F0CCFB02E0039B02F031
:100B400087FB01259623AB4007E0002F06D1012348
:100B50005D4003E0012596235B000293059B132B68
:100B600017D0182B15D0029B029A013B002A00D007
:100B7000D8E60EE0301C02F0CDFF0523051C0393E0
:100B8000CFE7281C311C02F0F5FF02240522039256
:100B9000C7E713B0F0BDC046E46A00001160000072
:100BA00006600000DC6A0000136000003C010010D9
:100BB000F7B502F099FA18200021FFF709FC00248C
:100BC0007B4EFFF7FBFB7B4D00236B62201C02F08A
:100BD0009FFE002C02D00020012101E0062003210D
:100BE00001F006FC201C02F027FE01A9071C684644
:100BF000002F03D0FFF7ABFB012728E0FFF7A7FB8F
:100C0000009B002B23D1002CE0D16B4F3B1C983371
:100C10001B68002B0DD1694BF618D7D51820002181
:100C20009437FFF7D5FB3C6863425C4100F026FC3B
:100C3000CCE7634B00941A6811321A60009B102BAA
:100C4000E9DC04F005FD009B01330093F6E7002C7E
:100C50000CD0009B182B01D0002FB2D000F06CFC00
:100C60005848FFF7D9FB544B0122DA6602F05AF9D3
:100C7000009B182B68D1019F0024F8B200F032FDD0
:100C8000012601946E6219283BD00ED8132835D066
:100C900004D8102842D0112821D052E0152835D090
:100CA00016284ED1FFF74EFD4EE0292846D00BD82E
:100CB00021281BD0262844D1434B05221C70434BCE
:100CC0001A7000F013FC3FE044282AD045282DD0AC
:100CD000352836D1F02300930723019334E03C4BB1
:100CE0001B68002B30D0FFF7E1FD05E0384B1B6897
:100CF000002B29D0FFF70AFE009425E0FFF798FBB0
:100D000022E0344B1868301A00F0CCFF0120FFF7C6
:100D100073FDFFF77BFBFFF745FB15E0FFF770FC6A
:100D200012E02D4802F0EEFA201C04E0E120000160
:100D300002F0E8FA301CFFF795FD05E0FFF76AFDC9
:100D400002E0002301976B621B4B1A1C463212789B
:100D50001C1C002A15D0009BD8B200F0C3FC32281E
:100D600007D0432809D031280BD1F02300931B4B27
:100D700006E0F02300931A4B02E0F0230093194B96
:100D80000193FFF7EBFA0098019904F0E3FC02F0FD
:100D900059FF6B6A002B01D0FFF738FB94342368AE
:100DA000002B00D00BE700F069FB012408E7C046E8
:100DB00020BF02001C1A0010240400100CFEFFFFCC
:100DC00068010010216000001800001000000010F1
:100DD0002400001008000010F0F1FFFF9BA60000A7
:100DE0008BA600009CA6000073B501F0F7FF444CF1
:100DF00000F0BCFC4348002101F076F90021424894
:100E000001F072F900F08AFD02F02EFF00F028FFD9
:100E100023680726B3432360236801252B43002062
:100E20002360021C0B2101F0E9F8201C374C102133
:100E300001F05AF923680022B34323602368281C79
:100E40002360042101F0DAF8201C002101F04CF9A4
:100E500001F0BEF89620000201F034FD2C4D012374
:100E60005B4200202B60FFF7C7FC00232B6050245F
:100E70000120FFF7E7F900F0F3FE02F0FBF82B6822
:100E8000002B05D16420043C01F0E6FA142CEFD1CC
:100E90000020FFF7B1FC1F4801F0FCFE192001F013
:100EA000DBFA01F0B3FD002802D0FFF7C1FA02E03F
:100EB000013C002CF2DC184A184B013AFF3A191D8C
:100EC000043B9A4203D3164818600B1CF7E702F064
:100ED0002FFF04F095FA1E230093292311490022C5
:100EE00001931148114B04F0C3FA114804F0FAFAC7
:100EF000104804F0FDFA104804F000FBFFF758FE1C
:100F000074400440984004409C4004409440044095
:100F1000240000102B600000F01F0010601A001069
:100F20001DBAFE7A09030000F55C0000680100109C
:100F30000D3C00000103000054010010F7B500282B
:100F40003BD00378303B5A425341C0180378782B8A
:100F500003D101301026012501E00A26002503787F
:100F6000002201922D2B02D1012301300193002395
:100F70000278002A1BD0171C303FFCB2092C02D883
:100F80007343DB1911E020273A43002D08D0171CCA
:100F9000613FFFB2052F03D81B01573A134304E00A
:100FA000064801F077FE002007E00130E0E7019AF3
:100FB000002A00D05B420B600120FEBD35600000BE
:100FC0000378202B01D10130FAE77047031C303B36
:100FD000DAB2092A01D8181C0AE020231843031C9E
:100FE000613BDBB2052B01D8573801E001204042BC
:100FF000704770B50E1CFFF7E3FF0025041C207836
:10100000002807D0FFF7E2FF002803DB2D0105438E
:101010000134F4E73560201C70BD000008B500F015
:1010200009FD011C014801F035FE08BD43600000C8
:1010300000B589B0684602F0BDF86946024801F083
:1010400029FE09B000BDC0467F600000F7B50F1C47
:1010500001A9161CFFF772FF002814D0019C0B4950
:10106000201C04F03FFF0D1C081C642104F03AFF13
:10107000281C3970642104F0DFFE04493070201C04
:1010800004F0DAFE01E001204042FEBD102700001E
:1010900037B50D1C48686A46694607310632FFF7C6
:1010A000D5FF01AC69466A4620800132A86802314A
:1010B000FFF7CCFF6B4618702288044B9A4203D985
:1010C000201C694602F005F937BDC0466B070000D9
:1010D00007B5486801A9FFF731FF019B3C20584341
:1010E00002F010F907BD000007235843054A101805
:1010F0009C30013B04D3C25C002AFAD0002000E0FF
:10110000012070472404001030B51A4885B001F062
:10111000C1FD0024651CA30719D1201CFFF7E4FFC3
:10112000002810D0281CFFF7DFFF00280BD0A01CE0
:10113000FFF7DAFF002806D0E01CFFF7D5FF0028F4
:1011400001D004340EE00C48211C01F0A3FD211C49
:10115000684602F069FE684601F05AFE074801F051
:1011600099FD2C1C064B9C42D4DD01F05FFE05B0BE
:1011700030BDC046185F00004F60000055600000A1
:10118000EF02000070B50E1CFFF71AFF0D25041CBE
:101190000134631E1878FFF719FF002806DB70552D
:1011A000013DF5D2201CFFF70BFF00E0002070BDD1
:1011B00070B5444C86B023680868251C002B06D106
:1011C000414801F067FD04F01BF9012309E0012B00
:1011D0000DD13E49042201F0CCFD002803D1236843
:1011E000013323606CE03A4801F054FD60E003787D
:1011F000412B17D1374C0230211CFFF7C3FF0028C9
:1012000056D00378422B53D1211C02300E31FFF708
:10121000B9FF00284CD00378432B49D1211C023060
:101220001C3103E0532B06D12B490230FFF7AAFFF4
:10123000002845D13CE04D2B1FD1284C0230211C09
:10124000FFF7A0FF002833D003784E2B30D1211CAC
:1012500002300E31FFF796FF002829D00378472B84
:1012600026D1023001A9FFF7C4FE019B002B1FDB32
:10127000184A1B4853651B491EE001A9FFF7B9FE38
:1012800004782023061C9C4312D1301C02A9FFF7CE
:1012900079FF019B061CE118134B994202DC02A85E
:1012A00002F0D8FD002E03D00134042CEDD107E06C
:1012B00004F0A6F80A480D4901F0ECFC00232B606D
:1012C00006B070BD2801001058600000185F0000D3
:1012D0006E600000240400106A0400104E04001028
:1012E0007A600000A55F0000EF020000846000004B
:1012F00037B54C682378002B25D0201CFFF760FE03
:1013000001A9FFF776FE019B041C002B1BD0D8B26D
:10131000FF2B09DD00F002FA019B051C1812C0B278
:1013200000F0FCF9019003E000F0F8F900250190CD
:101330000198002802D0291CFFF74AF823785A1E8A
:101340009341E418D6E737BD064A08B51378012162
:101350004B40137001D0044900E00449044801F0F7
:1013600099FC08BD5C020010286000008B60000042
:101370008F60000007B5486801A9FFF7DFFD019BFA
:10138000002B01DC01230193019B1E2B01DD1E2399
:1013900001930199034A044B4A4304481A6001F03F
:1013A00079FC07BD70170000580200109E60000015
:1013B00038B5051C002D09D0642402200021013C11
:1013C00000F042FE002CF8D1013DF3E738BD70B5C6
:1013D000061C01200821021C00F060FE07240120E9
:1013E0000821002200F05AFE321C012522412A4029
:1013F0000020022100F052FE281C08212A1C00F0C7
:101400004DFE013CEBD270BD10B50021041C0A1C3E
:10141000022000F043FE201CFFF7D9FF10BDF0B5FD
:10142000012385B002930023061C039372B60024A7
:1014300002AB1B59502040421843C0B2FFF7E4FFF3
:101440000020FFF7E1FF1020FFF7DEFFE020FFF7AD
:10145000DBFF212767430025F71902200021012225
:1014600000F01CFE785D0135FFF7B1FF842DF4D14B
:101470000434082CDCD162B605B0F0BD08B5AC2050
:10148000FFF7C2FFAE20FFF7BFFFA520FFF7BCFFAD
:1014900008BD38B50122051C0C1C00F0AFFD281C4E
:1014A000211C012200F0FAFD38BD08B5AF20FFF77E
:1014B000ABFFA420FFF7A8FF08BD08B5AE20FFF7DB
:1014C000A3FF08BD10B5041CF820FFF79DFF201CEA
:1014D000FFF79AFF10BD10B5041C8120FFF794FFA1
:1014E0003F202040FFF790FF10BD000008B5074BDC
:1014F00020201B781843FFF787FF0A20FFF758FFCB
:10150000034B1878FFF7E7FF08BDC0460000001046
:101510001800001008B5842202480021520001F092
:10152000F3FB08BD5D02001008B50248FFF777FF26
:1015300008BDC0465D02001008B501200821FFF774
:10154000A8FF00200221FFF7A4FF02200021FFF7DF
:10155000A0FF02200621FFF79CFF0320011CFFF7DC
:1015600098FF0320011C002200F098FD02200621B4
:10157000002200F093FD06210122022000F08EFDE2
:10158000FFF7C8FFFFF7D0FFA220FFF73DFFA02025
:10159000FFF73AFFC020FFF737FF0020FFF792FF69
:1015A0000A20FFF705FF4020FFF72EFF2C20FFF752
:1015B0002BFF3220FFF7FCFE2E20FFF725FF322005
:1015C000FFF7F6FE2F20FFF71FFF0A20FFF7F0FEC0
:1015D000FFF78CFFFFF769FF08BD000083280ED8D6
:1015E0000F290CD8CB08842253430722C01811407E
:1015F000034B80220A41111C1A5C11431954704795
:101600005D020010F0B51E1C87B00592F2780491BF
:101610005B68824201D2307845E0244AB478934234
:1016200005D10322041B54430192E4180CE0001B73
:101630000022824204DA1978013202315B18F8E79D
:101640001A789C1C5B780193A218002503922F1C2A
:10165000019B9F4226DA08220023029200937378AE
:10166000009A9A421CDA029A082A06D1039B9C42ED
:1016700018D00022257802920134EB0708D5049A8D
:10168000009BB818059AC0B29918C9B2FFF7A6FF17
:10169000009B029A013301326D1000930292DEE743
:1016A0000137D5E7019807B0F0BDC046C260000021
:1016B000F7B5041C0D1C161C1F1C01F048FB20185C
:1016C0000190019B9C420BD0832D09D82078291CC6
:1016D000321C3B1CFFF796FF01302D180134F0E758
:1016E000F7BD000010B50021012204230A4C0C5D57
:1016F000844203D118010243D0B20BE0013B002B1E
:1017000004D10132092A00DD1A1C042301312829E1
:10171000ECD1002010BDC046F46A00000F2302097E
:1017200018408000031F00D52833511E00200329D4
:1017300006D8242B04DC04218A1A0249CB18985CB1
:101740007047C046F46A000038B5051C0024054BFC
:10175000291CE05C044B0134C01800F0C5FC0A2CC5
:10176000F5D138BD386B000000400440F8B50D4F8E
:101770003C68002C15D11020FFF7E6FF0A4B002231
:10178000E65C1B195D78301C291C00F037FC023424
:10179000301C291C012200F081FC142CEED1012305
:1017A0003B60F8BD1C000010246B000070B50024E5
:1017B0000B4B0122E65C1B195D78301C291C00F0E4
:1017C0001DFC0234301C291C002200F067FC142C84
:1017D000EED10020FFF7B8FF024B00221A6070BD67
:1017E000246B00001C00001038B5051CFFF7BEFF7D
:1017F000002D09D007210122022000F0FFFB104B31
:1018000080211A688A431A6000200B2100F01CFC1A
:101810000124002805D000200B2100F015FC4442D3
:101820004441002D09D007210022022000F0E6FBF0
:10183000034B80211A680A431A60201C38BDC04639
:10184000FC3F0250F0B587B00026029001200391C2
:1018500004960596FFF7C8FFB04202D01823049300
:1018600001260021284C009120786178012200F0A7
:10187000C5FB20786178002200F010FC234B9D1DF1
:10188000012E24DC6A782F78111C381C019200F09C
:10189000DBFB002808D100991D4AB3008A5C103395
:1018A00069465A5001360BE02878697800F0CCFB85
:1018B0000028F0D0381C019900F0C6FB0028EAD0BF
:1018C000009A144B0132023D00929D42D8D12778F4
:1018D0006578381C291C002200F090FB291C381C5C
:1018E000012200F0DBFB0C4902348C42BCD1002009
:1018F000864206D0049A029B05991A60039A012039
:10190000116007B0F0BDC046246B00001C6B0000E6
:10191000F46A00001A6B0000386B000008B5012063
:10192000021C0B2100F06AFB01200B21002200F0B9
:10193000B5FB03200221012200F060FB03200221FD
:10194000002200F0ABFB08BD234B37B51A6810210D
:101950008A431A60214B8022196892010A431A6057
:10196000051C0B210120002200F048FB01200B2167
:10197000002200F093FB1A4B9F211A68194C8A43EE
:101980001A601A6818491A60184B186804F054FA5B
:101990008023000218432A1C20600221032000F04B
:1019A0007DFB142000F058FD2368FF229343236041
:1019B00023680F4A134323600E4B1B680193019B5E
:1019C000002BF9DA22680C4B13402360FFF7A6FFC7
:1019D00001980004800D3EBD3882044080800440A0
:1019E0009840044000C0014000093D006C03001015
:1019F000800000012CC00140FFFFFFF810B50C4C27
:101A00002068002813DA00202060FFF79DFF0A28D5
:101A10000ADC0120FFF798FF0138C023FF385B0084
:101A2000984201D801232360FFF778FF206810BD9A
:101A30000400001008B5FFF7E1FF002801D10020E5
:101A400007E00120FFF780FF011EF8D0014804F0F5
:101A5000F3F908BD50BB120008B5FFF7CFFF00280F
:101A60000AD0FFF7E7FFFA22031C0021C00FD200C3
:101A70009A424841014B186008BDC0462000001042
:101A800008B5074B02221A60064BA2221960064BCA
:101A90001A70A32258709A7000F0EEFD08BDC0467F
:101AA00098030010740300108803001008B5064B5B
:101AB00002311960054B00221A60054BA2221A70F0
:101AC000587000F0D9FD08BD980300107403001091
:101AD0008803001070B5051C0E1C0324281C311C43
:101AE000FFF7CEFF0223FF33984202D0013C002CC7
:101AF000F4D170BD70B5051C0E1C0324281C311CCC
:101B0000FFF7D4FF0223FF33984202D0013C002CA0
:101B1000F4D170BD0B4B10B51C6800239C420ED055
:101B2000094CA31CA270140A5C70140C120EDA701B
:101B30009C70FFF7DFFF831EFF3B5A425341181C86
:101B400010BDC046240000108803001070B50E4C74
:101B500025680024A54215D00C4C160AA270E67028
:101B6000160C120E6271A371A21D26711C0A54700C
:101B70001C0C1B0E9470D370FFF7BCFF841EFF3C3F
:101B800063425C41201C70BD2400001088030010DB
:101B900008B5064B1A6800239A4205D0FFF79AFF52
:101BA000831EFF3B5A425341181C08BD24000010FD
:101BB00008B5074B00201B68834207D0022007218D
:101BC000FFF788FF0238FF384342584108BDC0463E
:101BD0002400001038B50F4B051C1B680020834201
:101BE00017D00924641B631E062B10D8072C05D0C0
:101BF0000948A91E0918221C01F064F8E8B2211C4A
:101C0000FFF778FF0238FF384342584101E00120D6
:101C1000404238BD240000108A030010012010B596
:101C2000011CFFF757FF0223FF3398420ED1094BE7
:101C300001211960084B1C78230709D0074B0322A8
:101C400022409A70081CFFF755FF01E0012464420E
:101C5000201C10BD24000010780300108803001021
:101C600008B5FFF7DBFF02200121FFF733FF022356
:101C7000FF3398420FD1084B1B787F2B06D9842263
:101C8000022007215204054BFFF760FF09200421C1
:101C9000034AFFF73FFF08BD78030010020114005C
:101CA0008080808010B500280CD0254B80211A68D8
:101CB0008A431A60234B1B68D907FBD5224B0322AA
:101CC0001A6001E0204B1860204B012200211A60AD
:101CD00019601A60196801221142FBD01C4B802147
:101CE0001A601C4A49021468214311601A1C00281A
:101CF00004D1134B8024196821431960164B1968CD
:101D000088421CD01860002801D0144800E0144814
:101D1000116804F043F8134BFA2118608900041C81
:101D200004F08AF81E2358430F4BC821186049015C
:101D3000201C04F081F80D4B186001F039F810BD3B
:101D4000388204400C800440708004407480044059
:101D5000788004408080044008000010006CDC02A1
:101D6000001BB7006C030010680300107003001024
:101D700008B500F035F9134B00211A68120B120355
:101D80001A60114B1A68120B12031A600F4B1A6873
:101D9000120B12031A600E4B1A68120B12031A6010
:101DA0000C4B012219600C4B1A6019601A601A68FA
:101DB00001200242FBD0094B23221A60FFF772FF79
:101DC00008BDC046008000500080015000800250D5
:101DD0000080035040800440448004400880044058
:101DE00038B50F490F4800F055FF0F4D0024281C4F
:101DF00000F050FF0D4A0E48A1581219D2682B1C52
:101E0000143400F047FFC82CF4D10A4800F042FF18
:101E100000F042FB011C084800F03CFF38BDC04602
:101E2000185F0000426B0000926B0000886C00009D
:101E3000546B00005F6B0000816B0000F0B53B4B02
:101E40008BB01E68041C002E01D1351C08E0384BF5
:101E500002901B6801209B6854E033681E79019D45
:101E60002378002B31D0082D33D02378202B01D1BB
:101E70000134FAE7002B28D06A1CAD0008356B4608
:101E80000192EC50FF2E4CD02278002A07D0631C20
:101E9000202A01D01C1CF7E7002222701C1C019A8A
:101EA000012ADCD1224E234B0B253360371C013D28
:101EB000002D2ED03B680298196800F06BFF0028B7
:101EC000CBD03B6814333B60F1E7002D1CD0022DD2
:101ED00002D0B54206D911E00398174900F05AFF25
:101EE0000028F6D1124C15482368D96800F0D2FEBC
:101EF00023681348196900F0CDFE05E00C4BE8B2E9
:101F00001B689B6802A99847084A1368002B0BD1ED
:101F100003E0281C291CFFF763FF0A4800F0BAFE03
:101F200002E0019D0026D2E70BB0F0BD28010010B1
:101F300030010010886C00007A5F00008E6B00009A
:101F40007F600000956B000038B5041C164D0A2810
:101F500008D002D8082811D01CE00D2802D07F2814
:101F60000CD017E02A6800231370104800F092FE8E
:101F70000F4C201CFFF762FF2C6013E00C4B2A680B
:101F80009A420FD90B48211C00F084FE2B68013BBC
:101F90002B6007E00748211C00F07CFE2B685A1CD0
:101FA0002A601C7038BDC0462C010010926B0000E6
:101FB000280000109E6B000008B500F027FD0028E7
:101FC00004D000F0F9FCFFF7BFFFF6E708BD000002
:101FD000014A024B1A607047280000102C010010C3
:101FE000044B40211A680A431A60034B01221A70FD
:101FF0007047C04680800440340100100F4B70B51C
:102000001B78061C0C1C151C002B01D1FFF7E8FFE8
:10201000701E022803D80A4B8000C35800E0094B09
:102020001A68012D04D1A5402C1C14431C6003E048
:102030000121A1408A431A6070BDC04634010010DE
:10204000506D00000080005038B50F4B051C1B7808
:102050000C1C002B01D1FFF7C3FF0020032D12D869
:10206000281C012203F086FE02040608074B04E048
:10207000074B02E0074B00E0074B1B68A2401340F0
:10208000181C421E904138BD34010010FC3F005026
:10209000FC3F0150FC3F0250FC3F03500F4B70B51A
:1020A0001B78061C0C1C151C002B01D1FFF798FF98
:1020B000701E022803D80A4B8000C35800E0094B69
:1020C0001A68012D04D1A5402C1C14431C6003E0A8
:1020D0000121A1408A431A6070BDC046340100103E
:1020E0005C6D0000FC3F005038B5084B041C1B78A9
:1020F0000D1C002B01D1FFF773FF236818229343B7
:10210000236023681D43256038BDC046340100109C
:10211000054B3F221A60054B01221A60044B4021F7
:102120001A688A431A60704724800440D8800440AB
:102130003882044008B5044B40211A688A431A606B
:10214000FFF7E6FF08BDC0463882044008B500F03E
:1021500059FAFFF72BFB0A480021FFF7C5FF094892
:102160000021FFF7C1FF08480021FFF7BDFF074826
:102170000021FFF7B9FF06480021FFF7B5FF08BDB2
:102180000840044000400440AC4004401440044077
:102190001C40044008B50120FEF754F808BD0000BB
:1021A00008B5114B8022DA675200DA678022D2002C
:1021B000DA6780225201DA6780221201DA67802210
:1021C0009200DA67094A002313600121084A494254
:1021D0001160084A1360084A1360084B01221A6014
:1021E000FFF7D8FF08BDC04604E100E004820440C8
:1021F0000882044004C000403CC0004000C00040D1
:1022000008B5064B1A6801321A60054B1868FFF7CB
:1022100049FDFFF7C5FFC046C04608BD38010010A4
:1022200008000010F7B5071C0C1C72B6FFF78EFFF4
:10223000524B1A68524B1A60002F01D0514B00E0EC
:10224000514B524A04211360514B524D1A680A43B4
:102250001A6000232B60A1071ED04F4B4F4A19680C
:102260000A401A6029684E4BA2070ED5EC22520193
:102270000A432A6080221A6052001A608022D2002B
:102280001A60802252011A6003E0802212010A4380
:102290002A60802212011A60002F53D0414B002483
:1022A0001C60414B414E1C60414B301C1C60414B3B
:1022B000211C1C60FFF718FF201C0921221CFFF7BE
:1022C0009DFE201C0921221CFFF7E8FE3A4B8021CD
:1022D0001A683A480A431A60336807229343336006
:1022E00033680222134333600A21784303F056FD1A
:1022F000334B03221860334B1C60334B1A60334B53
:10230000334A19680A401A601A6880210A431A6021
:10231000234A8B001360204A1168194311602A6810
:10232000022113432B602B4B01221A602A4B1960A8
:102330002A4B1C491A601C601A601868012210425E
:10234000FBD00A60264B012252421A60254B002224
:102350001B680193244B1A6062B630BFC046214B04
:10236000019A1B689A4208D11F4B01221A601F4B29
:102370001868FFF797FCFFF713FFF7BD388204409A
:1023800034820440BF180000FF180000308204406F
:1023900010ED00E004820440008204407FE2FFFF71
:1023A00000E100E004C0004004000140644004403B
:1023B000044001400480014080800440841E0000ED
:1023C00018C0004008C0004014C000403CC000409D
:1023D0000FF0FFFF78800440708004407480044058
:1023E00008820440380100103C0100100800001071
:1023F00008B5FFF717FF08BD074B1A68013203D174
:10240000064A1168013111601A6801321A60044BE2
:102410001A6801321A6070474C0100104801001020
:1024200040010010074B98420AD8074A0023136066
:10243000064A01381060064A1360064B07221A60EC
:102440007047C046FFFFFF004C01001014E000E0A1
:1024500018E000E010E000E00B4A10B51368002817
:1024600000D10120C1438B4208D91168994209D398
:10247000591C146809188C42FAD3F6E71168C91A76
:102480008142FBD310BDC0464C010010014B1868BF
:102490007047C0464C010010064BFA211868064BE5
:1024A00010B589001C6803F079FC044B5C432018CC
:1024B00010BDC0464C010010480100103789410092
:1024C000034B01221A60034B1A6801321A607047ED
:1024D00000C0004050010010034B01221A60034B62
:1024E0001A6801321A607047000001405401001060
:1024F000002803D1044B01221A6003E0012801D116
:10250000024B18607047C04604C000400400014000
:10251000002802D1044B186004E0012802D1034BCB
:1025200000221A607047C04604C000400400014009
:10253000002801D1044B02E0012804D1034B1A68A2
:1025400002210A431A60704704C0004004000140A1
:1025500010B5002900D1134900280DD1124B802459
:102560001A6822431A60114B03221860104B19603D
:10257000104B1A60620211E0012811D10A4B80222F
:102580001868520002431A600B4B00221A600B4B72
:10259000032219600A4B1A6080229202094B1A60CA
:1025A00010BDC046FFFF00008080044050010010B5
:1025B00018C0004014C00040540100101800014031
:1025C0001400014000E100E080231022DB051A60C6
:1025D000094B08221A6000238022D2051268D10616
:1025E00004D5064A934201D00133F5E704489842E6
:1025F0009B4158427047C04618000040FF0F000042
:10260000FE0F000008B58022154B1202DA67154B49
:102610006C221A60144B154A196800201140196089
:1026200019681960124B19680A401A601A68042167
:102630001A600122FFF7E2FC002004210122FFF7CB
:102640002DFD002005210122FFF7D8FC01220020EA
:102650000521FFF723FD074B00221A6008BDC04685
:1026600004E100E01800004030400440F8FCFFFFA7
:102670003440044004800440F8B5174A174C002346
:1026800023601360164A202113608022D205116056
:102690002168144A012903D0934203D00133F7E79C
:1026A000934203D1FFF790FF002014E00E4F002566
:1026B0003E68013E2368FF2B0CD83B689E4204D045
:1026C0003E68FFF7E3FE051C0A35FFF7DFFE854293
:1026D000F0D1E7E72068F8BD580100105C01001058
:1026E00060010010FF0F000064010010034B012285
:1026F0001A60034B1A6801321A60704700400140AB
:1027000068010010174B70B501241C60164B1A6845
:1027100012191A60154B1A68002A22D01A68144D33
:10272000013A1A601E68002E0DD02A68201C211C58
:10273000FFF7B4FC2B68201CE31A2B602A680221E7
:10274000FFF7ACFC0DE01B68201C2B602A68211CE5
:10275000FFF7A4FC2A68201C0221FFF79FFC054B11
:102760001E6070BD00800140700100106C010010FF
:102770007401001004800140002803D1044B0122A1
:102780001A6003E0012801D1024B18607047C0466F
:102790000440014004800140002802D1044B18602D
:1027A00004E0012802D1034B00221A607047C046A2
:1027B0000440014004800140002801D1044B02E0A4
:1027C000012804D1034B1A6802210A431A6070479A
:1027D000044001400480014010B500280FD1124B85
:1027E00080221C68920022431A60104B032218605A
:1027F0000F4B19600F4B1A608022D20211E00128A2
:1028000011D1094B80221868D20002431A600A4B8A
:1028100000221A60094B03221960094B1A608022BA
:102820001203084B1A6010BD80800440680100103C
:102830001840014014400140700100101880014010
:102840001480014000E100E008B5184B1A680E231F
:102850001340062B0DD1164B9E221B68134205D048
:10286000144ADBB25360144B1B681EE0D9071CD519
:1028700001E0042B05D1104B1868C0B200F0B1F88C
:1028800013E00C2B06D10B4B8022596852000A43EF
:102890005A600AE0022B08D1054B1A68054B9106D5
:1028A00001D5002200E001229A6008BD08800040A6
:1028B00014800040780100100080004000487047FC
:1028C00078010010F7B52D4B2D4C8022002192038A
:1028D0000191061CDA67201C902200F015FA019B7A
:1028E0000725A360274B284F1A68AA431A60196866
:1028F000012211431960254B1968A9431960196811
:1029000011431960224B8021186849010143196065
:10291000204B1A6083223A601F4A126819681F4BC5
:102920001868504303F03AFA311C000903F036FAF4
:102930001B4B10221B491A60030A0B601A4BC0B2D2
:10294000032218603A60194A1560194A1D1C106864
:102950000190106860230340602BFAD110680123B6
:10296000184202D02B680193F8E723708022114BA4
:1029700092031A6005230B60F7BDC04604E100E036
:1029800078010010A44004400C800040A84004409E
:102990008080044098800440788004406C030010DC
:1029A00028800040048000400080004008800040F3
:1029B0001480004000E100E008B5FFF77FFFC26827
:1029C000031C1202120E8218D07BDA681202120E59
:1029D0000132D2B29A7352B2002A01DA00229A73FB
:1029E00008BD10B5041CFFF769FFC2681204120E7F
:1029F0008218D473C2681204120E0132D2B242732A
:102A000052B2002A01DA0022427310BD08B5FFF766
:102A100055FFC268C36812021B041B0E120ED01AA7
:102A2000431E9841C0B208BD70B500241D5D061953
:102A3000002D02D005550134F8E7121B301C131C81
:102A4000002B03DD0170013B0130F9E7D043C017D3
:102A50000240A01870BDF7B5051C01910093561EE9
:102A6000092B01D8041C0CE000980A2103F096F908
:102A70000199031C321C281CFFF7EDFF071C2C18C2
:102A800007E0671B002E04DD019B013E237001342B
:102A9000F7E700980A2103F0C5F93031781C21705E
:102AA000FEBDF8B50C1CD9175F18051C4F40561E0B
:102AB000092F12D9381C0A21002B03DA03F06EF912
:102AC000434202E003F06AF9031C281C211C321C5B
:102AD000FFF7E7FF041C2D1814E0002B00DA961E08
:102AE0002A1CA919891A002902DD14700132F8E79D
:102AF000F443E41734402D19002B03DA2D232B70F7
:102B000001340135381C0A2103F08CF93031297069
:102B1000601CF8BDF7B5089F1E1C051C013A3B0957
:102B200001D1041C05E00093331CFFF7F3FF2C18C0
:102B300006E0601B002A03DD2170013A0134F8E74A
:102B40000F231F40092F01D8303704E0002E01D099
:102B5000373700E0573727700130FEBDF0B585B03C
:102B6000041C029101D00021017000251178002978
:102B700006D1029F0023BD426CD22370281C6FE057
:102B8000029FBD42F5D2252902D00132217004E016
:102B90005178252904D12170023201350134E5E74D
:102BA000302902D0561C202100E0961C32782D3AA4
:102BB00050424241B6180022307830277F423F18F9
:102BC000FFB2092F07D80A277A438218D2B2303AC7
:102BD000D2B20136F0E7AF18BC46029FBC4501D91E
:102BE0007A1BD2B2692818D00BD863282AD064285F
:102BF00013D0582832D11F1D1B68201C00930123BD
:102C00001DE075280FD0782814D0732826D11F1DF9
:102C1000201C1B68FFF708FF0AE01F1D201C1B6813
:102C2000FFF73FFF04E01F1D201C1B68FFF713FF89
:102C30003B1C0BE01F1D1B68201C00930023FFF7AB
:102C400069FFF5E71868043320700120721C24180E
:102C50002D188BE7013C2370681E01E001204042E3
:102C600005B0F0BD10B50C1C131C6421221CFFF72D
:102C700075FF10BD00B5031C9BB00A1C01A8191CF0
:102C8000FFF7F0FF632800DDFEE701A800F0B6F8CB
:102C90001BB000BD0FB407B504A908C9181C0191E9
:102CA000FFF7E8FF03B008BC04B018470EB403B543
:102CB00003AA08CA191C0192FFF7D4FF02B008BC8E
:102CC00003B0184730B50C1C044303232340041CF5
:102CD000002B01D0002310E0032AFBD9CC58C450AC
:102CE0000433D41A032CF9D8131F9B0801339B001B
:102CF000C418C91803231A40ECE7934203D0CD5CF3
:102D0000E5540133F9E730BD30B5031C840701D128
:102D1000032A01D89A1814E00B060C041D1C254345
:102D20000D430C022543031C20C38418E41A032C12
:102D3000FAD8131F9B0801339B000324C3182240B9
:102D4000E8E7934202D019700133FAE730BD021C64
:102D5000031C981A0133591E09780029F9D17047CC
:102D6000031C0A781A70002A02D001310133F8E7F7
:102D7000704730B50023934208D0C45CCD5C651B1E
:102D800006D10133002CF6D1201C02E0002000E027
:102D9000281C30BD10B50022835C8C5CA34204D19A
:102DA0000132002BF8D1181C00E0181B10BD0000E8
:102DB00008B5094BFA211868890003F03DF8FFF7C0
:102DC00031FB96200002FFF77DFD0120FDF73AFA66
:102DD000FEF746FF08BDC0466C03001008B5FEF7BD
:102DE000C7FFFFF7FDF8FFF7A5F9FEF7A5FBFEF714
:102DF00091FBFFF7DDFFFFF7EBF808BD10B5041CF2
:102E00002078002803D00134FDF76CFAF8E710BDF4
:102E100038B5051C0E24013C04D3295D0248FFF798
:102E200039FFF8E738BDC046686D000038B519486D
:102E3000FFF730FF184C201CFFF7EAFF174D422127
:102E4000281CFFF727FF201C0E30FFF7E1FF43216E
:102E5000281CFFF71FFF201C1C30FFF7D9FF10486C
:102E6000FFF718FF201C4630FFF7D2FF0D48FFF791
:102E700011FF201C2A30FFF7CBFF281C4E21FFF743
:102E800009FF201C3830FFF7C3FF616D0648FFF7CC
:102E900001FF38BD6B6D000024040010716D00004F
:102EA000786D00007E6D0000846D000003110A2221
:102EB00053430F2210401818704738B50A21041CDC
:102EC00002F0BAFF0A210501201C03F00BF8281CB0
:102ED000084338BD08B5C12252000E200221FEF77A
:102EE00019FE024B01224E331A7008BD9C030010DC
:102EF00010B50B4C231C4E331B78002B01D1FFF770
:102F0000E9FF231C4D331B784F340C221A432378DE
:102F100001205B001A43011CFEF7FCFD10BDC046FA
:102F20009C03001010B5094C231C4D331B78002B5B
:102F30000BD1231C4E331B78002B01D1FFF7CAFFA6
:102F40004D3401232370FFF7D3FF10BD9C03001005
:102F500008B5084A111C4D310B78002B08D000230E
:102F60000B70111C51314C320B701370FFF7C0FF06
:102F700008BDC0469C03001038B5051C4079FFF71A
:102F80009CFF0B4CA0702879FFF797FFE070E87862
:102F9000FFF793FF80232071637104210920FEF75E
:102FA000A9FD044B01224F331A70FFF7A1FF38BD72
:102FB000880300109C03001010B501210220FEF7C9
:102FC000E7FD074B041C18787F231840FFF76EFFBE
:102FD000044B1A1C4A32503310701C70201C10BD58
:102FE000780300109C03001008B5064B064A1B68C6
:102FF00064201168584302F01FFF632800DD63203E
:1030000008BDC0464001001044010010024B0122DF
:103010004B331A707047C0469C030010034A0023CC
:10302000111C4B3151320B70137070479C03001010
:1030300008B5FFF7C1FF0C490C4A0B1C4B3318783D
:103040000B1C5133002808D01878012801D8013012
:1030500003E01068064B186000E0187000234C3144
:103060000B70136008BDC0469C03001040010010A7
:103070004401001008B5FEF7D1FD0C23184004D020
:10308000024B49331A781043187008BD9C03001096
:1030900010B5FFF7EFFF064B1A1C493212781C1CC3
:1030A000530701D5FFF7C4FF49340023237010BD37
:1030B0009C03001008B50020FEF796FB002801D005
:1030C000FFF7E6FF08BD000010B5064C00235034A2
:1030D0002370FFF7EFFF2378002B01D1FFF76CFF80
:1030E00010BDC0469C03001008B50A48542102F0E8
:1030F00005FF094BFA22D2001A80FFF7E5FF074BC4
:1031000000221A60064BFA2292001A60054A064B0A
:103110001A6008BD9C030010F0030010400100106D
:1031200044010010FD3900001002001070B51D4C64
:10313000061C637822781B021343A278A07912043C
:103140001343E2780D1C12061343174A13401A0A60
:10315000237062701A0C1B0EE3706379A2702279DF
:103160001B021343114A134023711B0A6371FFF7BB
:103170009DFE0F4B1B88C01830806079FFF796FECC
:10318000B070E078FFF792FEF070A078FFF78EFE47
:1031900028706078FFF78AFE68702078FFF786FE57
:1031A000A87070BD780300107F7F3F3F071F0000AD
:1031B000F0030010F0B58DB0051CFEF7F9FC0028F7
:1031C00004D1281C1249FFF771FD1EE00AAE0BACBA
:1031D000211C301CFFF7AAFF3388F7780793B378D8
:1031E000267808936378A47809930A4B187900F03D
:1031F00045FC099B04900293009701960394281CB8
:103200000549079A089BFFF751FD0DB0F0BDC04678
:10321000906D000078030010956D000070B5061CDD
:103220000D1C141CFEF7C4FC00280AD0301C291CFD
:10323000FFF77CFF002C07D0044B00201B79236094
:1032400003E00120404200E0201C70BD7803001024
:10325000F7B504880E1C051C6421201C0092019304
:1032600002F0E0FD114B8FB2B078E41B1C80FFF739
:1032700024FE0F4CA0707078FFF71FFEE0703078CE
:10328000FFF71BFE2071E878FFF717FE009B6071C7
:10329000A371A878FFF711FEE071381CFFF70DFE4F
:1032A00020720198FEF796FCFEBDC046F0030010A8
:1032B0008803001008B50223FFF7CAFF08BD08B550
:1032C000021C501E8241520100200121FEF722FC07
:1032D00008BD38B5041C01200D1CFFF7F0FF201CB1
:1032E00000F018FC072102F0FDFD201C0A1C291C1F
:1032F000FFF7E0FF96204000FFF7AEF80020FFF751
:10330000DEFF38BD73B5041CFFF756FE002801D15F
:1033100000203FE0204B1A1C4A3215781E1C331C3B
:103320004A331B78AB4207D10A20FFF795F8FFF725
:1033300043FE0028F3D1EBE7FEF73AFC0028E7D084
:1033400001A96846FFF7F2FE684600F0E3FB051CA2
:1033500001A800F09BFB114B04199C420DD9E31707
:1033600001221343ED18281C694600F003FC002CD1
:1033700001DA0B4B00E00B4BE418201C01A900F014
:1033800097FB281C072102F0ADFD68460A1C01A925
:10339000FFF790FF76BDC0469C0300107F510100EF
:1033A0008051010080AEFEFF10B5094A094B0A4862
:1033B000995C0A4A8C0707D4094C1C5D002C01D18A
:1033C000CC0701D5012100E000211954995410BD0A
:1033D000EB15000024040010941500009315000064
:1033E000EA150000031C012210B50020134204D08E
:1033F00010491148405C80081040022213420AD054
:103400000C490D4C615CCC0705D50C498C6A0C4904
:103410008C4200DC1043042213420AD0054B0649BB
:10342000CB5C990705D5054B196B054B994200DC20
:10343000104310BDEC150000240400109C03001084
:10344000E70300000368642B04DC034A534342682B
:10345000981800E00148704700D6830000987F3339
:1034600008B5044A044B0220D15C0143D154FFF754
:103470009BFF08BD24040010EB15000038B5051CA7
:103480000C1C081C0E2102F039FD2B68D821890084
:103490005943201D02F08EFB6968201C02F08AFB54
:1034A00038BD000070B50C1C0421051C02F0A3FB04
:1034B0000921061C281D02F09EFBD8218900051C4D
:1034C00002F010FD054B281C59437618D821666080
:1034D000890002F0B1FC206070BDC04610270000DA
:1034E00038B50268054B051C0C1CD01800F042FBD7
:1034F0006868211D00F0F2FA38BDC046ADD924003D
:10350000F0B53F4D85B02B1C4C331A78002A57D1AB
:103510006F682D69012403951C70FEF749FB002894
:103520004BD0384B1A787F2A03D9FFF799FF022432
:1035300044E05B795AB2002A09DA334A072011883D
:10354000643111801F221A40211CFEF7E3FA2F4D2F
:103550002C1D211C281CFFF7E9FDFFF745FDE87134
:10356000201C00F09CFA2E1C103E7060C41B291C0D
:1035700003A800F0C2FA071E0FD13268281C01927E
:1035800000F0C8FA224B019AC0183060801A431E1E
:10359000EE2B06D81F4B58432418E343DB171C407F
:1035A00000E03C1C1C491D4BCB5C5A0724D51C4B2E
:1035B0001348C918FFF762FF1EE0012464421BE0B4
:1035C0006C68FFF711FDE875061C281C143000F02C
:1035D00066FA124B6860104D041BEB5C5A070BD562
:1035E000301C0A2102F07EFC0D4B301CE9540A21EC
:1035F00002F022FC0B4BE854201C05B0F0BDC04685
:103600009C03001078030010F0030010AC030010BE
:103610005326DBFF00D6830024040010EB150000C6
:1036200096150000971500004368054A934206DD91
:10363000044A9B184360036801330360F4E7704752
:1036400000D68300002A7CFF4268002A08DA03685B
:10365000002B05DD0349013B521842600360F3E78C
:103660007047C04600D683000168054A08B58B182C
:103670004168044A03608B184360FFF7D5FF08BD1B
:103680003A9BB00000C40900436810B5041C002B2D
:1036900002DAFFF7D9FF01E0FFF7C6FF2368002B2E
:1036A00002DA201CFFF7E0FF10BD436810B5591A7D
:1036B000041C4160FFF7C8FF63680020834206DCFA
:1036C0002368834203DC201CFFF7CEFF012010BDDE
:1036D000F8B5FFF715FF254B254C061CE25C254D80
:1036E000254B51070BD5A96B4218E96BAA638A4297
:1036F00005D3E25C01210A43E2540022AA63E35CA1
:1037000008273B4219D01D4A311CA01802F052FA7A
:10371000002803D01A4BE25C1743E7541349635C5B
:103720009A070AD51748311CFFF7BFFF002804D0BD
:10373000134B0421E25C0A43E2540C490127635C09
:103740003B4209D01048311CFFF7AFFF002803D0DF
:103750000B4BE25C1743E7546A6C002A02D02B6CD7
:103760009E192E64FFF720FEF8BDC046EC15000040
:10377000240400109C030010EB150000A4150000A9
:10378000EA150000CC030010C403001008B50720A0
:10379000FFF728FE0023984204D0FFF799FF024B61
:1037A000024AD35C181C08BD9315000024040010C5
:1037B00038B5114C636C002B1CD0FFF789FF206CCF
:1037C000616C884216DD02F037FB231C0130483360
:1037D000C50F1B782D186D10002B00D06D42281CD2
:1037E000FFF790FD002805D0636C5D43236C6D00EE
:1037F0005D1B256438BDC0469C030010F8B50C4E17
:10380000041C351C4A352F78FFF75EFC002C02D1D2
:103810002B78BB4208D0074A00234C363370136024
:103820009C4201D0FFF7C4FF201CFFF7AFFFF8BD9B
:103830009C0300104001001008B5FFF7DFFF08BD32
:103840007FB5041C0720FFF7CDFD051C002C4ED0D2
:10385000FFF7AEFF002D0BD1FFF77AFB264B5B6C19
:10386000002B48D002A8012343710371C3703BE0D1
:10387000224EE80708D5204BDC6B9B6BE41AB44260
:1038800003DCFFF74FFB36E01D4CA90705D51D48AB
:10389000FFF7D8FD844200DD041C6B0705D51A48EC
:1038A000FFF7D0FD844200DD041CB442E9DDFFF7E0
:1038B0004FFB114E6B46321C03CA03C3201C134935
:1038C00002F010FB7368201C591801910F4902F097
:1038D000B3FA009B181800906846FFF7D5FE6846BB
:1038E00002A9FFF7FDFD02A8FFF746FB03E0002851
:1038F00001D1FFF72DFB7FBD9C0300104F46000058
:103900000085E201C4030010CC03001000D6830040
:1039100008B5FFF795FF08BD70B5061CC4000E2062
:1039200070430E4B0E4D18180E4B6419C018211C15
:10393000FFF7B8FD002E0FD12E1C1036201C311CB5
:10394000FFF7CEFD2068072102F0CCFA14350A1CDF
:10395000301C291CFFF7AEFC70BDC04624040010CB
:103960009C03001096150000011C0E20484308B56A
:10397000054B03311818054BC900C018044BC91872
:10398000FFF790FD08BDC04624040010B2150000EA
:103990009C03001038B5C11C094BC200C900D218E5
:1039A000C9180C6815680530C000C018631B496849
:1039B00003605368CB1A4360FFF766FE38BDC0460C
:1039C0009C03001010B50948094C0A4A0023825C88
:1039D0002364231C48331A70074B0321C01802F0DC
:1039E0000AF9C8231B025843606410BD2404001068
:1039F0009C030010F1150000EE150000013808B519
:103A0000062830D802F0B6F904070D12212A2D003D
:103A1000FFF75EFE27E0144B144AD05CFFF77CFFF3
:103A200021E0114B114AD05CFFF79EFF0F4B0E4A6D
:103A3000985C0F4A9B5C002802D09A0713D501E0DE
:103A4000DA0710D5FFF7A6FF0DE00A48052102F0BE
:103A5000D2F8094B0022D8639A6304E0FFF7A4FC74
:103A600001E0FFF7AFFF08BD95150000240400102A
:103A7000EC150000161A00109C03001007231840D4
:103A8000014B8000C0587047086E000002783C234C
:103A90005A4341785218534382789818704710B5AA
:103AA000041CFFF7F3FF64225043E378181810BD9D
:103AB00038B50C1C3C21051C02F014FA281CA1701E
:103AC0003C2102F0B9F93C2102F00CFA6170E121CD
:103AD000281C090102F0B0F9207038BD38B50C1C63
:103AE0006421051C02F0FEF9281CE170642102F03B
:103AF000A3F9211CFFF7DCFF38BD10B54A884488C4
:103B0000031C0020944204D118880B88C01A434239
:103B1000584110BD70B5837802210022994252416C
:103B2000048896214901051C64180C20A41A4243FC
:103B30009B18033B992058430521023002F07CF981
:103B40006E26FF3666436421A31086194942201C65
:103B5000F61802F071F9C82136184900201C02F04D
:103B60006BF9034B3018C018EB78C01870BDC04615
:103B7000D382FFFFF8B5204B0C1CC5181F4B8000EB
:103B8000C0181F4902F058F903235843C617B60F4F
:103B90003618B610AE19B600953E301C194902F021
:103BA000A1F9CD17AD0F6D180527AD107D43023576
:103BB000281C992102F096F9081C391C02F03CF9E6
:103BC0000130E0709921281C02F036F90C210230F6
:103BD00002F088F94D1CEDB2A570301C094902F0C5
:103BE0002BF9094B0C21C6180E20401B02F024F9BA
:103BF00036182680F8BDC04679050000652F040000
:103C0000B13A0200B505000094EDFFFF0B4B1A68B6
:103C1000002A01D101221A60094B022219680028EA
:103C200005D00A431A601A6804218A4304E09143CC
:103C300019601A6804210A431A60704708020010CC
:103C4000FC3F0150064B02211A688A431A601A6829
:103C500004218A431A60034B00221A607047C04651
:103C6000FC3F01500802001070B5124E124D301C7E
:103C70000021FEF739FA281C0021FEF735FA3268D8
:103C800007239A43326032680124224332602A6853
:103C9000201C9A432A602B68211C23432B60221C82
:103CA000FEF7ACF9201C0221221CFEF7A7F9FFF752
:103CB000C9FF70BD7C4004408040044038B5184BBB
:103CC000072219680124914319601968051C2143D2
:103CD0001960144B201C1968914319601A68211C43
:103CE00022431A60221CFEF789F9221C201C0221A3
:103CF000FEF784F90C4B291C186802F09DF8011C92
:103D0000201CFEF769FD201CFEF756FD074D6423BD
:103D1000201C2B60FEF730FD2B68002BFCD138BD3A
:103D20007C400440804004406C0300106C01001093
:103D30000D4A0E4B0021D1540D480E4B18600E4811
:103D400011540E4898600E4811540E490E481961DE
:103D5000012111540D4898610D4811540D4A9A6281
:103D60000D4ADA627047C046240400107615000040
:103D700044960000F40300107715000044AA0000E8
:103D80007815000044BE000079150000446E000064
:103D90007B15000044D200004482000010B5144995
:103DA0000313021CAB204001C918091889790020AF
:103DB000052B1CDC01291ADC5B0059180D4C89000D
:103DC0000B59834213D01105090D8810802418184F
:103DD0006401001904780320024052000820801A70
:103DE0008440201CC024A4005B5C2040184310BD0C
:103DF00024040010F4030010094A0313AB21D21865
:103E00004901521892790020052B06DC012A04DCB6
:103E10005B009A18034992005058431E984170471E
:103E200024040010F40300100723594310B5084B75
:103E300059189C310023CC5C0F2222400270CA5CCE
:103E40000133120942700230072BF4D110BDC04675
:103E5000240400100723594310B5074B59189C310F
:103E600000234278047812012243CA5401330230FD
:103E7000072BF6D110BDC0462404001070B5AD4C20
:103E800086B0E36E6E465A1E934117363370AA4BC6
:103E90009A6A191CD006400F0138062807D801F08D
:103EA00069FF040C2012181A1D00022509E0636E38
:103EB00016339B001B591D1C15E0636E16339B00C7
:103EC000E55800230FE0A36DE56DAB420BDD0D253A
:103ED00009E0022503E00C25032304E00D252B1C3B
:103EE00001E00D25EDE70D6150111F2800D91BE100
:103EF00001F04AFF2000220029002C002F0033008F
:103F00003B00440048004C00540061006E00760005
:103F100083008F009B00A800B800C500D500D30027
:103F2000E100E400E700EF00FE0002010B010D01DB
:103F30000F011501E01801E0E0180E30EB1A591CD2
:103F400001F0DCFFF0E0E0181C30F7E7211C0E3137
:103F500005E0E0180E30E1180BE0211C1C31201C9C
:103F60001A1C2B1C01F06BFDDEE0E018E1181C3080
:103F70000E31EB1A5A1CFEF7A5FED5E06F48011C66
:103F80000E31EDE7E018011C1C31F2E7226E102122
:103F9000002A00D00A21221C0E3206E0226E1021D7
:103FA000002A00D00A21221C1C32029100950196A1
:103FB000201C211C53E0216E0122327010220029A6
:103FC00000D00A22009501960292201C211C45E097
:103FD000226E1021002A00D00A21221C0E3213E08A
:103FE000216E012232701022002900D00A22009591
:103FF00001960292201C211C4DE0226E1021002A05
:1040000000D00A21221C1C32009501960291201C2E
:104010006AE0226E1021002A00D00A21484A02914B
:1040200000950196101C111C19E0216E102000292A
:1040300000D00A20424A0290111C1C3900950196BA
:10404000101C0CE0216E012232701022002900D0D9
:104050000A223B49009501960292081C002201F0B9
:10406000F8FC61E0226E1020002A00D00A20344AB9
:104070000290111C1C3900950196101C35E0216E30
:10408000012232701022002900D00A222C4900950A
:1040900001960292081C002227E001223270226E53
:1040A0001021002A00D00A21254A0291009501968C
:1040B000101C002119E0009620481BE000962048C3
:1040C00018E0226E1021002A00D00A21221C1C3286
:1040D00006E0226E1021002A00D00A21221C0E3296
:1040E0000095019602910020211C01F0DAFC1BE0F2
:1040F0000096201C002103E0211C1C310096201C8E
:104100001A1C2B1C01F02AFD0EE0201C02E00B48BB
:1041100000E00B48191C2A1C01F037FD04E0201CAC
:10412000191C2A1C01F03BFD33780120E36606B020
:1041300070BDC046240400101C1A00103204001088
:1041400040040010064910B50A1C883213681C1C74
:104150001E34A4006050013303210B40136010BDD6
:1041600024040010054B0322191C8831086801380B
:1041700002400A601E329200D0587047240400109A
:10418000F8B5194EFF24351C8C352868A400013081
:10419000FFF704FE154F0440BA6AA40193101C43B4
:1041A000B36E0122F86202409A420FD1830708D40D
:1041B000201CFFF721FE002808D028680230FFF7F6
:1041C000C1FF331C8C331C600123FB60201CFFF7F4
:1041D00013FE002806D18C3630680230FFF7B2FF9C
:1041E000FFF7C0FF0220F8BD240400101C1A0010C5
:1041F0000C490D488A6A031C8C3370B51D68D305C1
:104200009B0E0C1C910500D5403B866E921001213F
:104210000A40B24203D18C30EB180360E160012008
:1042200070BDC0461C1A0010240400100A4B591C13
:10423000C87F991CC97F000109020843D97F1A1C55
:1042400003330843D97F031C09030B438C321360EB
:10425000024B0120D8607047240400101C1A001083
:1042600008B5FDF7F9FB014BD86608BD2404001022
:1042700008B5084B5A1CD07F9A1CD27F000112024D
:10428000104303331A7FDB7F10431B031843FFF7F0
:1042900059FF08BD2404001008B5FFF763FF03238E
:1042A000044A0F219A180140013311770011072B9E
:1042B000F6D108BD2404001008B5FFF753FF034BE7
:1042C00001228C331860024BDA6008BD2404001010
:1042D0001C1A001010B5064CA36E002B06D0FFF779
:1042E00041FF044B8C3401222060DA6010BDC046CF
:1042F000240400101C1A001010B5064CA36E002BED
:1043000006D1FFF72FFF044B8C3401222060DA60C6
:1043100010BDC046240400101C1A001008B5104B34
:104320000022596A1A62914214D05969914216DDED
:10433000012906D1D969914203D0DA610A22996133
:104340005A615A69032A02DD06490120C866013A0A
:104350005A6104E0044B1B68002B00D0984708BD4D
:104360001C1A00102404001014020010074B5A6A93
:10437000002A02D05A69002A07DD9A690F21044BEE
:104380001140D97712110133DA7770471C1A0010E7
:10439000240400100949FF230A1C8C3210681B02F8
:1043A00003401360064A506A002802D05069002872
:1043B00003DD92698C3113430B60704724040010B5
:1043C0001C1A00100A4B10B51A1C8C3211681C1CE8
:1043D00001311160231C8C331868421C1A60FFF7EE
:1043E000DDFC01231842F5D0024AD36010BDC0465F
:1043F000240400101C1A0010114BF7B51A1C8C3243
:104400001268104912139A1852189279061C0192D8
:1044100000240B4A0C4915196B181B78019A93421A
:1044200009D10A4B2003ED182F782E70FFF7E4FC1A
:10443000002800D12F700134102CEAD1F7BDC046FE
:1044400024040010701500007615000066150000A9
:10445000034BD96D986D421A51424A41DA66704752
:1044600024040010034B597F1A7F09011143024AAB
:1044700099547047240400102C150000074B084A7B
:10448000197F9954597F074A9954997F064A99543C
:10449000064B022259680A435A60704724040010F0
:1044A00058150000591500005A1500001C1A00107C
:1044B000054B064A9A5C1A77054A9A5C5A77054A70
:1044C0009A5C9A777047C046240400105815000083
:1044D000591500005A150000F0B5002385B0029070
:1044E00003911D1C039FBD4223DA134A00210124BE
:1044F0000298204216D0161C0B3E0196101C461E38
:1045000037780770301C019EB042F8D10B485E1C12
:10451000C318187F022901D101231840331C161C2F
:104520000B3E3070013164000E320329E0D10135B9
:10453000D8E705B0F0BDC0465D1900102404001096
:10454000F0B5002385B0029003911C1C039FBC4270
:104550002DDA002201200E215143164D8C461649BA
:104560006E18029D664405421BD00121775C0197BD
:10457000019D7718013F01313D700C29F6D1591C7E
:10458000022A05D10B4EF3181D7F01231D4002E0C6
:10459000084FFB181D7F0B1C0649084E6144891902
:1045A0000D7001324000032AD5D10134CEE705B0A9
:1045B000F0BDC046240400102E150000391500007F
:1045C000F7B500220190151C8D421EDA0F4B012415
:1045D0000198204212D01E1C0C3E0096181C461E4C
:1045E00037780770301C009EB042F8D118781E1C36
:1045F0000C3E3070064EB61830770132054F0E3340
:104600006400BB42E4D10135DEE7F7BD5E1900105E
:104610002404001088190010F7B500240091261C0E
:10462000009B9E4219DA0D4B012528420ED01A78C4
:104630001A730122995C9F18013F013239700D2ACB
:10464000F8D1074ADF7A121917770134054A0E3379
:104650006D009342E9D10136E2E7F7BD521900102F
:10466000240400107C19001010B50E21041C2148F0
:1046700001F044FC01230F2C37D8201C01F07AFBF9
:10468000080A0D0F1215191B1E20222527292B3071
:10469000012000E002200C2124E00420FBE703209D
:1046A00006211FE0072004211CE0FFF701FF022381
:1046B0001BE0042015E00120011C0EE002200BE0AD
:1046C000042009E00120011C0CE0022009E0032085
:1046D00002E0032005E007200121FFF79DFF03E032
:1046E00007200121FFF76CFF0123034A51680B43A8
:1046F000536010BD400400101C1A001008B50F28AC
:1047000035D801F037FB080A0F1114171A1D2022A3
:104710002427292B2D30012000E002200C21FFF757
:104720000FFF24E00420F9E703200621F7E7072024
:104730000421F4E70320062117E00720042114E0F8
:104740000120011CEBE702200BE0042009E001201E
:10475000011C0AE0022007E0042005E0032003E03A
:1047600007200121DBE707200121FFF7B5FE034BFE
:10477000012259680A435A6008BDC0461C1A00103D
:1047800008B5034B1B68002B00D0984708BDC046F6
:104790001002001008B50120FFF7F2FF064B074A90
:1047A000995C074A985C002901D0072100E00B21A1
:1047B0000140995408BDC04624040010951500001E
:1047C000EB15000038B50F2800D9C1E001F0D2FA8E
:1047D000080815244551C0676F7B8995A6A9BABC06
:1047E0005C495D4B0E22C85C5C4B50430818C018F6
:1047F0001C31FEF767FA02200BE05649564B0E2299
:10480000C85C574B50430818C0181C31FEF75AFAC1
:104810000320FFF7B5FF9BE04E4C4F4BE35C002BB2
:104820000DD0504B211CE0181D310422FEF74AFA2E
:104830004D4B0122E15C07200A40E254E9E74B4B73
:10484000227FE15C06200A40E254637F0C221A4377
:10485000474BE15C0A40E254DBE73E493E4B0E2207
:10486000C85C444B50430818C0181C31FEF72AFAA4
:104870006EE0414C414B201CE1180522FEF722FA64
:104880003F4B0420E2183F4BD15C01430520D1543B
:10489000FFF776FF201C052101F030FB58E00120D6
:1048A000FFF76EFF2B4A374B0B21D05C23E0294BDF
:1048B000294A9A5C002A02D0334A985C1AE0314AAD
:1048C0000721985C17E0234B234A9A5C002A03D007
:1048D0002D4A0120995C02E02A4A0820995C014394
:1048E00035E01C4B1C4A995C264A985C002901D093
:1048F0000D2100E00E21014029E0174A154B995C7B
:10490000204A002902D0995C022001E0995C012034
:1049100001421DD10143995404207AE7FFF73AFF81
:1049200016E00C4C0C4B124DE35C002B05D0012023
:10493000FFF726FF635D082201E0635D0422134355
:10494000635505E0012100E00021034B014AD154E9
:1049500038BDC046240400109515000096150000CF
:10496000B2150000EE150000F1150000EA15000078
:10497000EB150000CE150000161A00102AEAFFFF02
:104980000EEAFFFFEC150000ED15000038B5052814
:1049900057D801F0EFF90603131D3B48FFF7FAFE65
:1049A00002E00120FFF7ECFE2648274A031C1C3BCF
:1049B000995C0E225143254C5B1830E02148224A75
:1049C000031C1C3B995C0E225143214C5B1826E0D2
:1049D000204C1D4B251CE35C1C35002B09D0281CEA
:1049E0000E2101F08BFA1C4B201C1D30E118042213
:1049F00016E00120FFF7C4FE184B281CE118042222
:104A0000FEF760F9201C20300A2118E00D480E4AFC
:104A1000031C1C3B995C0E225143114C5B18191965
:104A2000FEF750F90DE00120FFF7AAFE054C0D4BF3
:104A3000201CE1180522FEF745F9601D092101F04F
:104A40005DFA38BD40040010951500009615000071
:104A5000B215000024040010EE150000EA15000055
:104A6000CE150000D6150000064B597F9A7F09012C
:104A700012020A43197F0A435A67034A00219954D4
:104A80007047C046240400102C15000080239B00B2
:104A9000994205D100230022C25401330E2BFAD1D2
:104AA0007047000030B5184D85B06C6F002802D0FB
:104AB0000F239C430443154B6C67EB5CFD2B02D129
:104AC000FFF7D2FD1DE0FB2B02D1FFF75FFF18E0DF
:104AD0000F4B9C4205DD281C1C300E2101F00EFA04
:104AE0000FE06846211CFFF79FF96846211CFFF77D
:104AF000CDFF00236846C15CEA18013311770E2B05
:104B0000F8D105B030BDC046240400102C150000BB
:104B1000EF020000164B30B55C6F0F229443154A2C
:104B200004439A5C85B05C671D1CFD2A02D1FFF727
:104B3000E5FD1BE0FB2A02D1FFF744FE16E00E4B19
:104B40009C4213DC6846211CFFF76EF90023EA182B
:104B5000127F6946CA5401330E2BF8D16846211CD6
:104B6000FFF794FF6846211CFFF774F905B030BDCC
:104B7000240400102C150000EF0200001FB5134C98
:104B8000134BE35CFD2B02D1FFF778FC1CE0FB2B01
:104B900003D10020FFF716FE16E0616F0D4B99421E
:104BA00012DC6846FFF740F90023E218127F6946DD
:104BB000CA5401330E2BF8D16846616FFFF766FFC8
:104BC000616F6846FFF746F91FBDC0462404001018
:104BD0002C150000EF02000010B50D4C631CD87FAF
:104BE000A31CDB7F00011B021843E37F1843E31C77
:104BF000DB7F1B031843FFF7D1F80F23021C1A4079
:104C000022770211134000126377A07710BDC046CF
:104C100024040010044B5A6E16329200D258121A15
:104C200051424A41DA66704724040010044B5A6E20
:104C300016329200D158013900D50D21D15070475C
:104C400024040010054B5A6E16329200D1580131DF
:104C50000E2900D10021D1507047C0462404001015
:104C6000094B5A6E16329200D2580D2A03D11A1CE3
:104C70002932127805E09A18507F117F0001021C3A
:104C80000A435A657047C04624040010084B10B50B
:104C90005A6E0F2416329200D1585A6D581814408B
:104CA000013104770D2902DC5B1812111A7710BD4F
:104CB000240400100E4B30B55A6E596D1632920016
:104CC000D2580D2A07D11C1C2934F0202478084022
:104CD0002043586507E09818447F057F24012C4342
:104CE0005C650C1144779B180F221140197730BD79
:104CF0002404001008B503480E22011C1C39FDF7DE
:104D0000E1FF08BD5C04001008B503480E22011C39
:104D10001C31FDF7D7FF08BD4004001008B504485A
:104D20000022011C1C310D2300F089FE08BDC04685
:104D30004004001008B503480E22011C0E39FDF78F
:104D4000C1FF08BD4E04001008B503480E22011C27
:104D50000E31FDF7B7FF08BD4004001008B5044848
:104D60000022011C0E310D2300F069FE08BDC04673
:104D7000400400100023044A00219A1846320133EF
:104D80001170082BF7D1704724040010C31C421E79
:104D90000020934207D00449400059184631097851
:104DA000013B0843F5E770472404001010B50B1DC4
:104DB000994208D0044A01248A18044046321470EB
:104DC00040100131F4E710BD2404001038B5002074
:104DD000FFF7DCFF084C051C0021207FFFF7E6FFF2
:104DE00004202577FFF7D2FF0421051C607FFFF721
:104DF000DDFF657738BDC0462404001010B50020E3
:104E0000FFF7C4FF034C20770420FFF7BFFF607754
:104E100010BDC0462404001010B5054C0021207FB1
:104E2000FFF7C4FF607F0421FFF7C0FF10BDC0463D
:104E30002404001010B50020FFF7A8FF041C042074
:104E4000FFF7A4FF054B0001054A0443D454054B6A
:104E50001B68002B00D0984710BDC0462D150000E0
:104E6000240400100C02001038B5074D074C0F2326
:104E7000285D00211840FFF799FF285D04210009F3
:104E8000FFF794FF38BDC046240400102D15000024
:104E9000F8B50020FFF77AFF061C0420FFF776FF25
:104EA0000B4C0C4D071C285D0F2318400021FFF709
:104EB0007DFF285D04210009FFF778FF064B3F01C5
:104EC0001B683E432E55002B00D09847F8BDC046C6
:104ED0002D150000240400100C02001010B5094C20
:104EE000231C8C3318680130FEF758FF064B021C58
:104EF000D8620F231A402277021113400012637701
:104F0000A07710BD240400101C1A001010B5084C26
:104F10000E21201C00F0F2FF201C0E300E2100F0AC
:104F2000EDFF201C1C300E2100F0E8FF10BDC04634
:104F30002404001010B50C4B191C0E311A1C187FDC
:104F40001C7801332043D8768B42F8D1936E002B26
:104F500008D0064B1B690D2B04D1137F111C29317E
:104F60000B70537310BDC046240400101C1A0010AF
:104F700010B50C4B191C0E311A1C1C7F187801330C
:104F80002040D8768B42F8D1936E002B08D0064B88
:104F90001B690D2B04D1137F111C29310B70537326
:104FA00010BDC046240400101C1A001030B50021AA
:104FB00085B00E4B421C1818007F6C4608550D2515
:104FC000D40F181C002395425C41644201312240F9
:104FD0000E2901D0101CECE76C46E15CC2180133CD
:104FE00011770E2BF8D105B030BDC0462404001057
:104FF000074B10B55A6E16329200D458611E1C1918
:10500000D1502077002901DA0D21D15010BDC046C2
:1050100024040010034A0023111C943198320B60C1
:105020001360704724040010034B01229433196865
:105030004A401A607047C04624040010044A002306
:1050400013678C321360034B0122DA607047C0464D
:10505000240400101C1A001010B5A04C0F20A16AE7
:105060009F4A8B1018408911013852560E284DD88E
:1050700000F080FE080F171E224C284C3034384CAC
:105080004C424600002A41DB964B9A1840320023DE
:1050900005E0002A3ADB934B9A18403201239371C2
:1050A0006CE1002A32DB8F4B9A184032927921E072
:1050B000081CFFF79DFF61E1002A27DB101CFFF7AA
:1050C000A9FD5BE1002A21DB864B596E1631890070
:1050D000CA5053E1081CFFF775F94FE1081CFFF7B0
:1050E00019FD4BE1002A11DB7E4BAC219A184901D6
:1050F0005218D279DA6641E1081CFFF7D3FC3DE192
:10510000002A03DB101CFFF751FF37E1782B02D197
:10511000FFF78CF832E1782B00DD8FE0402B09D1CE
:10512000002004E05C2B6BDC502B52D10220FFF7F7
:1051300063F923E1402B47DC1C2B02D1FFF7DAFD9A
:105140001CE11C2B1EDC0C2B04D1664B0120983378
:10515000186014E10C2B0BDC0120002B00D10EE1B8
:10516000082B02D1FEF7FEFF08E10120404206E1D4
:10517000162B02D1FFF774FD00E1182BF5D1FFF7D4
:105180005DFFFBE02C2B02D1FFF7BEFDF6E02C2BE0
:105190000ADC262B02D1FFF779FDEFE0282BE4D1C2
:1051A000504B00225A66E9E0382B03D14D4B0120C9
:1051B0005866E4E03C2B02D1FFF7B0FDDEE0362B71
:1051C000D3D1FFF777FDD9E05C2BABD1FFF750F8D7
:1051D000D4E0502B0ADC482B02D1FFF739F9CDE09F
:1051E0004C2BC2D1FFF77AFE0220C8E0562B02D129
:1051F000FFF7A0FDC2E0582BB7D1FFF731F8BDE0B3
:10520000682B02D1FFF782FEB8E0682B08DC602B28
:1052100001D101208BE7662BA7D1FFF795FDADE00B
:10522000702B01D1032082E7762B02D1FFF796FD88
:10523000A4E06C2B99D1FFF72FF89FE0D62B02D179
:10524000FFF7EAFD9AE0D62B4EDCA62B02D1FFF742
:105250000BFE93E0A62B1DDC962B02D1FFF7EAFD97
:105260008CE0962B0ADC882B02D1FFF77FF885E0D3
:105270008C2B00D079E7FFF78DF87FE0982B03D1D6
:10528000184B00221A6679E09C2B00D06DE7FFF7DF
:10529000EBFB73E0B82B02D1FFF7BCFE6EE0B82B3E
:1052A0000BDCA82B03D10F4B0120186667E0B62B4F
:1052B00000D05AE7FFF7ECFD60E0C82B02D1FFF702
:1052C000B3FE5BE0CC2B02D1FFF786FC56E0BC2B93
:1052D00000D04AE7FFF752FC50E0C0461C1A00100D
:1052E00044E6000024040010F22B02D101202062C9
:1052F00045E0F22B21DCE62B02D1FFF77FFD3DE0FC
:10530000E62B0ADCD82B02D1FEF7E4FF36E0DC2BDB
:1053100000D02AE7FFF70EFE30E0EC2B02D1FFF7BA
:1053200027FE2BE0F12B02D1FFF724FD26E0E82B2E
:1053300000D01AE7FEF7E0FF20E0F62B02D1FFF7DE
:1053400045FD1BE0F62B0ADCF32B02D1FEF7E6FF4E
:1053500014E0F52B00D008E7FFF768FC0EE0F82B0F
:1053600002D1FEF7A9FF09E0F82B02DAFFF76AFC89
:1053700004E0FC2B00D0F8E6FFF774F8012010BD24
:1053800038B5184C231C8C331868FEF707FD164BF4
:105390000022E16EDA60E26603229862A1661040A4
:1053A0001D1C022809D090420AD0012802D0FFF724
:1053B00053FE07E0FEF7E4FE04E0FEF75FFD01E0C8
:1053C000FEF716FF00280BDDEB68002B04D1231C31
:1053D0008C3319680A181A609034226813182360F5
:1053E00038BDC046240400101C1A0010034B0122D3
:1053F000DA660F229A775A771A77704724040010DA
:10540000F0B5144D85B0291C10226846FDF75AFCF2
:10541000114B1249EC18201C00F070FD6946281C45
:105420001022FDF74FFC0E4B0427E25C01263A43A5
:10543000E2540C4B281CE25C09213243E2544D300B
:105440000A22FDF761FC084BE754FFF7CFFF6666C1
:1054500005B0F0BD9A1900108AEAFFFFF8150000A8
:10546000EB150000EC150000DD1500007047000092
:1054700030B50E4D049C28600D4801600D490A604E
:105480000D4A13600D4B039A1A600D4B0D4A1C60B8
:105490000D4B1C600D4B1A600D4A0E4B1A600E4BE3
:1054A0000E4A13600E4A136030BDC0463C02001025
:1054B0004802001050020010240200101C020010CC
:1054C00010000010655500001C1A00101402001096
:1054D0003D5500000C0200106D5400004C020010FD
:1054E00034020010014B18607047C04618020010CB
:1054F000014B18607047C04634020010014B186021
:105500007047C04620020010094B10B51A68191CDC
:10551000084B002A03D1084C2468226003E01A6873
:10552000904200DA101C186001230B6010BDC046C9
:1055300028020010440200102002001010B5064C92
:105540002368002B07D06420FFF7DEFF034B044ADB
:10555000D05C2368984710BD180200102D1500007C
:105560002404001013B5002300930193114B124C37
:105570001A68124B11681868814202D122680092A1
:1055800008E012681A600E4B1B68002B02D06846B8
:1055900001A99847009B2360002B04D0094A64208E
:1055A0009361FFF7B1FF009A531E9A41064BDA66EA
:1055B00013BDC04624020010380200100C00001079
:1055C000480200101C1A001024040010034B1B6832
:1055D000002B01D1024A13607047C0463002001010
:1055E0002802001038B5164B1A1C98321268002A8F
:1055F00004D0144B1C6801231C4001E094331C6848
:10560000114DAB689C4202D16A68002A16D0002C6A
:1056100002D1002B0AD111E00C4B1B68002B02D0E9
:10562000201C6968984700236B6006E0074B1B68E5
:10563000002B02D0201C211C9847AC6038BDC0460E
:10564000240400102C0200101C1A00103C02001050
:1056500008B5084A084B126819688A1A05D5FA2253
:1056600052001A60054B1A6801321A60FFF7BAFF40
:1056700008BDC0461C020010140000102C020010CF
:10568000F8B50E1C0E21041C171C00F037FC174B3C
:1056900003259E4211DD092363730123237323E055
:1056A000301C0A2100F01EFC301C61550A2100F05C
:1056B000C3FB0135061C0D2D01D0002EF0D1EF1BD0
:1056C000033F27706B1E022B05D0E15C621BD218D2
:1056D0005173013BF7E70F235D1B013D6B1C032B4F
:1056E00002DD00236355F8E7F8BDC046FFC99A3BC9
:1056F00037B5041C0025002300930193124B1B684F
:10570000002B02D0684601A998470098013500286F
:1057100000D000250220FAF716FE0C4B1A680C4B3D
:105720001168186881420AD012681A60FFF790FF6A
:10573000002C04D0013C002C01D1201C02E0032DE0
:10574000D9DD01203EBDC0464802001024020010F1
:1057500040020010F7B5061C0F1C6A4CF0282DD033
:10576000231C9433684D1B68A861E961002B17D195
:1057700018280BD1C32909D1644B1B680F2B05D105
:10578000201C38300E21162200F044F9A869182890
:1057900004D1EA69332A01D100F0E2F8FFF726FECE
:1057A000002E02D00A236B6100E06E61AA69584B9B
:1057B0001A60584B1B681A68574B19E0072912D01A
:1057C000251C1C35281C0E2100F098FB0422381CD7
:1057D000291C00F01DFA514A00232A67504AE3664B
:1057E0006367A35405E00023E3664E4A231C8C3311
:1057F0001A60FFF7EBFE00250123236701954A4B52
:105800001B68002B1AD0494E3368371C002B15D06B
:105810001B68002B04D1464B1B6898473B68F7E791
:1058200033681A68013A1A60424A1368002B05DD92
:10583000013B1360002B01D1FFF7C8FEFFF7A0FD6D
:10584000002801DAFAF732FE3B4B01982E4F9842BE
:1058500005D04023021C9A43384B9A420BD1BB6AB5
:10586000374A934204D008229343364A934202D1E6
:105870000A20FFF749FE344B9D4206D1334BBA6AEA
:105880009A4202D11420FFF73FFE261C8C36BF6AD5
:1058900035682F4B01979D4203D02E4B9D420FD070
:1058A00018E0281CFEF77AFAB8239B00984211D121
:1058B0003368FA200133C0003360FFF725FE09E0AA
:1058C000281CFEF76BFAC8239B00984202D133686C
:1058D00001333360204B1B6898470E4B1A681F4BEF
:1058E00011681868814206D012681A60FFF7B0FE8E
:1058F0000F4B1B689847226F002A80D1FFF772FE7A
:10590000F7BDC046240400101C1A0010100000103F
:1059100038020010240200100C00001001070000E3
:105920002C15000032020000280200102002001096
:105930004C020010440200106E020000260200001B
:10594000FB030000E3030000F42700002202000034
:10595000990800009E080000340200104002001068
:10596000F7B5274E002033681C68FFF7C1FE336887
:105970001A689442FCD01B6801272D33FF33019332
:10598000FFF734FD1F4C0A231F4D63611823A361E9
:105990001523E3612B1C9033002267621A60FFF726
:1059A00025FD2F673368019A1B689A420CD0FFF7D8
:1059B000E7FC3268154B116818688142F2D0126812
:1059C0001A60FFF745FEEDE72B1C012790331820E6
:1059D00000211E686762FFF7BDFE0D4B301C196881
:1059E00000F02AFA3835011C0422281CFFF748FE73
:1059F0001823A3610023301C6762E361FEBDC0462B
:105A0000240200101C1A0010240400104002001090
:105A10001C02001070B5002A10DD047801231C4020
:105A20004B1E002B08DBC55CE4006E083443C454F5
:105A30000124013B2C40F4E7013AECE770BD30B59E
:105A40009A4205DC845C8D5C85548C540132F7E706
:105A500030BDF0B5069E051C07A804783078002AF2
:105A600017D0059EB34217DCCE5CD75CF7193F1800
:105A70000020A74201DB3F1B0120EF540133F0E778
:105A8000CA5C12180020A24201DB121B0120EA545A
:105A90000133059A9342F3DD01231840069B1870E9
:105AA000F0BDF7B50AAC2478099D0094089E2C78C7
:105AB00000282DD0002928D0002A18D0B34248DC75
:105AC000CF5CD55C7F1B3F1B0024A74202DA009C01
:105AD0003F190124C7540133F0E7CA5C121B0024AC
:105AE000551C02D1009A0124013AC2540133B34239
:105AF000F3DD2EE0D15C4942091B0024A14202D013
:105B0000009F0124C919C1540133B342F2DD20E0E2
:105B1000002914D0002A08D0B3421ADCCD5CD05C36
:105B20000133281A041BE40FF6E7B34211DCCA5C08
:105B30000133141B013462425441E4B2F5E7B3422D
:105B400007DCD15C013349420C1B611E8C41E4B27D
:105B5000F5E701231C40099B1C70F7BD70B5049C40
:105B60000125257000290BD09A420BDC865C8D5CE8
:105B7000AE4209D10132F7E7815C002904D101323C
:105B80009A42F9DD0023237070BD914204DA431874
:105B90005B7843540131F8E70023435470478A424D
:105BA00005DD8318013B1B788354013AF7E7002396
:105BB00083547047F8B50024071C0E1C251C002ECA
:105BC00015D0301C0A2100F02DF93B5D6918C91869
:105BD0000025092901DD0A3901253955301C0A2122
:105BE00000F0DCF80134061C0E2CE8D101E0002D99
:105BF000E7D1281CF8BD10B542180B1C0020013954
:105C000005D30A246043D41A645C0019F7E710BD79
:105C10008A18914205D00F2303400B70000901310F
:105C2000F7E77047F0B5061C85B0FBF773FC00245E
:105C30006A46351C54730B35AB7B0C221A4001921B
:105C4000032213401A012B7FFF219B010B401343BA
:105C50002A7803A8134301336A461373211C214B8E
:105C60000022FBF725FD019B002B13D0271C0837D2
:105C7000FFB2381C0821FBF7B1FC019A082A02D1B7
:105C8000381C032104E0019B0C2B03D1381C092193
:105C9000FBF7A4FC0B34013D842CCDD1331C2B33FA
:105CA0001D7801331B782D011B021D43331C2A3341
:105CB0001B780C241D43EA070CD50B4AA300D3180C
:105CC000043B1868094B09221B19013B1978084B42
:105CD000FBF7EEFC013C6D10002CECD1FBF724FC33
:105CE00005B0F0BDEC6A000084E60000B4E60000F8
:105CF000DC6A000008B5002805D0FBF7D6FB074892
:105D0000FFF790FF08E0FBF7D8FB054B1B78002B53
:105D100002D00448FCF7BEFF08BDC046521900106F
:105D20005C02001054E60000FEE7FEE708B5002321
:105D30000B4A0C499A188A4204D20B49C95C0133B8
:105D40001170F5E7094B0A4A591C013B934203D2F3
:105D500000221A700B1CF6E7FBF746F8FEE7C04678
:105D60000000001018000010C0E60000190000102C
:105D70004C1A001002B4714649084900095C4900F8
:105D80008E4402BC7047C04603B4714649084000C7
:105D90004900095A49008E4403BC7047002934D099
:105DA0000123002210B488422CD301242407A142ED
:105DB00004D2814202D209011B01F8E7E400A142AA
:105DC00004D2814202D249005B00F8E7884201D345
:105DD000401A1A434C08A04202D3001B5C0822431D
:105DE0008C08A04202D3001B9C082243CC08A0428E
:105DF00002D3001BDC082243002803D01B0901D07A
:105E00000909E3E7101C10BC7047002801D00020EE
:105E1000C04307B4024802A14018029003BDC04627
:105E2000D90000000029F0D003B5FFF7B9FF0EBC80
:105E30004243891A1847C046002941D010B4041CB7
:105E40004C40A44601230022002900D549420028E5
:105E500000D5404288422CD301242407A14204D219
:105E6000814202D209011B01F8E7E400A14204D2F9
:105E7000814202D249005B00F8E7884201D3401A10
:105E80001A434C08A04202D3001B5C0822438C0832
:105E9000A04202D3001B9C082243CC08A04202D39C
:105EA000001BDC082243002803D01B0901D009098C
:105EB000E3E7101C6446002C00D5404210BC70473C
:105EC000002806D003DB0020C043400801E080200A
:105ED000000607B4024802A14018029003BDC04664
:105EE000190000000029EBD003B5FFF7A7FF0EBC97
:105EF0004243891A1847C0467047C04642180023DB
:105F0000002903D0037001309042FBD17047C04696
:105F100025732025730D0A00444D3431005345523A
:105F200049414C20434F4E534F4C450072656164CC
:105F300079000D0A4279652E2E2E0D0A00554E4924
:105F40004D504C20494E53545220253034583A2558
:105F5000303358202530335800504C532052455090
:105F60004F525420495420414E44205245534554E9
:105F70002043414C43004E4F00203F002573202515
:105F800073202025694D485A0056323500202025BF
:105F9000692E253033695600202573525443200062
:105FA000444D3431204F4B0020204552523A202599
:105FB0006900424144204B45592025303278002069
:105FC0002D2025303278004C43443A253032692068
:105FD0002D20256900505245535320454E544552BB
:105FE00020544F20534156450053495A453A25699C
:105FF00020555345443A256920465245453A25697E
:1060000000535441434B3A0025633120484F5552C9
:10601000002D005254432052454144204641494CF2
:10602000007475726E6564206F6E003C5245534576
:10603000543E0D0A00426164206E756D6265722ED9
:106040000D0A004241543A2025696D560D0A000D93
:106050000A2530327820200057616974696E672004
:10606000666F7220646174612E2E2E0D0A004261EB
:1060700064206D6F64656C0D0A00526561642025B3
:10608000730D0A004641494C4544006F6666004C5A
:1060900043442064656275672025730D0A00436FD1
:1060A0006E736F6C652074696D656F7574207365B0
:1060B0007420746F202569206D696E757465730D89
:1060C0000A00000000005C000C000C7C287C7C4472
:1060D0007C241048285408000C0038440044380040
:1060E00020100810381080400010101000400020D0
:1060F0001008384438007C006454484454281C106C
:106100007C4C542438542004740C285428085438E7
:1061100000500080500010284428282844281004EB
:106120005408384C5C7814787C54283844447C44B7
:10613000387C54447C14043844347C107C007C004B
:1061400020403C7C106C7C40407C087C7C047C7C47
:10615000447C7C14083844787C1468485424047CBB
:10616000047C407C3C403C7C207C6C106C1C601CA3
:1061700064544C7C4400081020447C0008040880CF
:1061800080800408007844780D0778008601320189
:106190004902390242027C0E07800170004C004324
:1061A000004C00700080010B060000FF011101117E
:1061B000011101EE0B06FE000101010101010101C7
:1061C000820B06FF0101010101010182007C0C0626
:1061D0000000FF0111011101110101010B06000076
:1061E000FF01110011001100010C06FE0001010168
:1061F0000111019100F2010C06FF011000100010C6
:10620000001000FF010804000000000000FF01076B
:1062100004C00000010001FF0E070000FF0118008C
:1062200024004200810000010C060000FF01000173
:106230000001000100010E07FF010C003000C0004A
:1062400030000C00FF010C06FF01060018002000C2
:10625000C000FF010B06FE00010101010101010167
:10626000FE0B06FF0111001100110011000E0C06BB
:10627000FE000101010141018101FE020C06FF0146
:106280001100110011002900C6010B0600008E004C
:10629000110111011101E20B06000001000100FFD4
:1062A000010100010B06FF000001000100010001D7
:1062B000FF0D0703001C006000800160001C00034C
:1062C0000D071F00600080017C00800160001F0E30
:1062D0000783014400280010002800440083010DBA
:1062E00007030004000800F00108000400030E0783
:1062F0008101410121011101090105010301080486
:1063000000000000FF0301020A050000060018005B
:10631000600080010804000000000102FF030D0777
:10632000080004000200FF0102000400080C06003F
:106330000200020002000200020002000404020047
:10634000007F0109050000070000000000070B06A0
:106350004400FF0144004400FF01440B0600008C90
:10636000001201FF032201C40D0782004500250031
:10637000920048014401820C060000E60019012643
:1063800001C0002001070400000000010002080411
:1063900000000000FE0101020804000000000102EC
:1063A000FE010B0600008800500020005000880B02
:1063B00006000020002000F8002000200E0710003A
:1063C0001000100038005400920011010B0600006C
:1063D0002000200020002000200D07110192005411
:1063E0000038001000100010090500008001600056
:1063F0001800060B060000FE00010101010101FE6C
:106400000804000002000200FF010C0600008201E7
:106410004101210111010E010B0600008200010162
:1064200011011101EE0B060000600058004600FF4C
:1064300001400B0600009F00090109010901F10B51
:10644000060000FE00110111011101E20B0600001F
:106450000100C10131000D00030B060000EE001128
:106460000111011101EE0B0600008E001101110156
:106470001101FE0E07FF01930155013901550193EA
:1064800001FF01080400000000000208010A0500E5
:106490000020005000880004010B0600005000504E
:1064A0000050005000500905000004018800500011
:1064B000200B06000002000100610111000E0D0713
:1064C000FE0010001000100010001000100A05C09F
:1064D00000280128012801F0010905FF0108010831
:1064E000010801F00905F000080108010801900AFF
:1064F00005F000080108010801FF010905F0002866
:106500000128012801B00B06000002000200020071
:106510000200020B060000020002001E0002000240
:106520000B060000820042003E000200020B060043
:1065300000820042003E004200820B0600009200F2
:1065400052003E004200820B060000920052003EC4
:10655000005200920B060000FC03800080007C00CB
:10656000800B060000A800680038002C002A0C06EA
:106570008301450129011101010101010D07C0003D
:10658000A0009000A800C4008200800D070800044D
:1065900001FC0004000400FC01040E07F0000801E7
:1065A00008011001E000180100010B060000FE01C7
:1065B000010011011E01E00B0608000400B80140B3
:1065C00002A0011C0E071E001000F0013000500058
:1065D000900010010D0760009000080108011801EB
:1065E000E800040B060000020002000200020002A4
:1065F0000B060000FE01020002000200060B06006E
:1066000000820042003E000200020B0600008200F1
:1066100042003E004200820B060000920052003E03
:10662000004200820B060000920052003E00520021
:10663000920B060000FC03800080007C00800B06AB
:106640000000A800680038002C002A0E0700000493
:106650000182007C008000000100010D07C000A045
:10666000009000A800C4008200800B060000020019
:1066700002001E000200020A05C0002801280128AD
:1066800001F0010905FF01080108010801F00905F1
:10669000F000080108010801900A05F0000801084F
:1066A000010801FF010905F000280128012801B0B7
:1066B000070400000000FE01090C060000780284B7
:1066C0000284028402FC010C060000FF0110000895
:1066D000000800F0010804000000000000F90108B3
:1066E00004000000000002F9030C060000FF012076
:1066F000005000880000010804000000000000FFB6
:10670000010E07F80108000800F00108000800F079
:10671000010C060000F801100008000800F0010B51
:10672000060000F000080108010801F00B06000057
:10673000FC03840084008400780C06000078008448
:106740000084008400FC03090500000000F8010833
:106750000008090500009000280148019008040085
:10676000000000FE0008010C060000F80000010017
:10677000018000F8010B0600001800600080016035
:1067800000180D077800800160001800600080018B
:10679000780A05000098016000600098010B06006F
:1067A0000000023802C0014000380A0500008801DC
:1067B000480128011801080400001000EE01010240
:1067C0000E078001600118010601180160018001B7
:1067D0000905000000000102EE01100C06830145CE
:1067E0000129011101010101010D07FE0010001036
:1067F00000100010001000100004040200007F01CF
:1068000009050000070000000000070B064400FF18
:106810000144004400FF01440B0600008C001201FB
:10682000FF032201C40D07820045002500920048A5
:10683000014401820C060000E60019012601C00097
:10684000200107040000000001000208040000000D
:1068500000FE0101020804000000000102FE010B1D
:106860000600008800500020005000880B06000041
:1068700020002000F8002000200603000000040093
:10688000020B06000020002000200020002006034C
:1068900000000000000109050000800160001800F0
:1068A000060B060000FE00010101010101FE0804C3
:1068B000000002000200FF010C06000082014101FD
:1068C000210111010E010B060000820001011101DE
:1068D0001101EE0B060000600058004600FF014069
:1068E0000B0600009F00090109010901F10B0600D8
:1068F00000FE00110111011101E20B060000010070
:10690000C10131000D00030B060000EE0011011162
:10691000011101EE0B0600008E00110111011101A1
:10692000FE0804000000008C018C01080400000037
:1069300000000208010A0500002000500088000441
:10694000010B060000500050005000500050090597
:106950000000040188005000200B06000002000126
:1069600000610111000E0D07780086013201490215
:10697000390242027C0E07800170004C0043004C3B
:1069800000700080010B060000FF011101110111D0
:1069900001EE0B06FE000101010101010101820B64
:1069A00006FF0101010101010182007C0C060000CB
:1069B000FF0111011101110101010B060000FF018E
:1069C000110011001100010C06FE0001010101116E
:1069D000019100F2010C06FF0110001000100010E0
:1069E00000FF010804000000000000FF010704C0D0
:1069F0000000010001FF0E070000FF011800240045
:106A00004200810000010C060000FF0100010001AE
:106A1000000100010E07FF010C003000C000300033
:106A20000C00FF010C06FF01060018002000C0004A
:106A3000FF010B06FE000101010101010101FE0B36
:106A400006FF0111001100110011000E0C06FE00DE
:106A50000101010141018101FE020C06FF0111004B
:106A6000110011002900C6010B0600008E00110163
:106A700011011101E20B06000001000100FF0101FC
:106A800000010B06FF000001000100010001FF0DE5
:106A90000703001C006000800160001C00030D075C
:106AA0001F00600080017C00800160001F0E0783D2
:106AB000014400280010002800440083010D070352
:106AC0000004000800F00108000400030E07810123
:106AD00041012101110109010501030103072061A1
:106AE000C26000000D0C205AF8670000070A018000
:106AF0008861000018C6111012C53130C43271709F
:106B000072C2818082C3C1C0131383731716151418
:106B100037363534777675748786858400070008A4
:106B2000000A010002070208020100030109030430
:106B300002040205030500062024282C383C4044AA
:106B4000484C4669726D776172652025735F5632D5
:106B5000350D0A00252D3130732025732573000D66
:106B60000A5479706520273C636F6D6D616E643ED9
:106B7000203F2720666F7220706172616D730D0A6D
:106B800000557074696D65202575730D0A002573B5
:106B90000D0A0D0A00444D3431203E3E200025638D
:106BA0000048656C70004E6F20706172616D7300FB
:106BB0004B6579207072657373003C6B6579313E6B
:106BC000203C6B6579323E202E2E2E0044756D7070
:106BD000206D656D6F7279004C6F6164206D656D1D
:106BE0006F727900637400436F6E736F6C6520740D
:106BF000696D656F7574003C6D696E757465733E83
:106C0000004765742074696D650074730053657482
:106C10002074696D65003C595959594D4D44443EA5
:106C2000203C48484D4D53533E00746400557064F9
:106C30006174652074696D65003C6F666673657488
:106C40005F696E5F6D696E757465733E00546F6742
:106C5000676C6520646973706C6179206F757470FE
:106C6000757420746F20636F6E736F6C65006200C3
:106C700052656164206261747465727920766F6C0C
:106C800074616765000000007A5F0000000000008A
:106C9000E11D0000A16B0000A66B0000A46B0000CA
:106CA000FF000000F1120000B06B0000BA6B0000A2
:106CB000056E00000000000009110000CC6B000010
:106CC000A66B0000936D000000000000B1110000F1
:106CD000D86B0000A66B0000E46B00000100000010
:106CE00075130000E76B0000F76B0000E56B000018
:106CF0000000000031100000016C0000A66B0000D5
:106D00000A6C000002000000911000000D6C0000F1
:106D1000166C00002A6C000001000000D110000079
:106D20002D6C0000396C00002B6C0000000000008E
:106D3000491300004D6C0000A66B00006E6C000053
:106D4000000000001D100000706C0000A66B000029
:106D5000008001500080025000800350FC3F015031
:106D6000FC3F0250FC3F03502578000D0A413A20B9
:106D700000202025633A20000D0A533A20000D0A16
:106D80004D3A20002020473A20253032780D0A0065
:106D90006661696C00253034692D253032692D25F6
:106DA00030326920253032693A253032693A25304F
:106DB000326920257300253032783A253032783A0E
:106DC000253032692E253032690025303278203A5C
:106DD000202569202569203A2025303278004E4F41
:106DE0002052544300253032783A253032783A2503
:106DF00030327800253034782D253032782D25300A
:106E00003278202025730000286E00002C6E0000D0
:106E1000306E0000346E0000386E00003C6E0000E2
:106E2000406E0000946B00004D4F4E0054554500DD
:106E300057454400544855004652490053415400B8
:106E400053554E00193F0097013B01C60A430AD231
:106E5000057C01D201520A19008809B409AC0D5B06
:106E60000D630C16016907F7037206B20E62057313
:106E70000E3606AC080B0A7B0A85010303AF02B588
:106E8000068600B10DE403490F530F5B0EC30EBA23
:106E9000062D085F0E690E2F08050F2C0F350173A4
:106EA000035703C00C0400AC009D03B809A300E322
:106EB00006A20B2F0AFC00F7012001290132023C37
:106EC00002CE066C00009319050B0C030B80456283
:106ED0008432200E0306201418052D8D0F0F121377
:106EE000010B80556A8E0306201418052018032D07
:106EF000851A09131001C870F868385C581C0E38E0
:106F0000AA28B0445D5C385CD8284C9B5D1CCC271B
:106F10004C09820DFC0E0F20120F0F0DF1FE80BDEB
:106F20006A981209040D0581408001620DFC041568
:106F30001020060CF1FEBF0705124E78BC067CC679
:106F4000007DC68E130110A9D09868F8F67B0DFC61
:106F50000B0519030F0405D9FE009D0E809D66BF29
:106F60000E0E3D180B802D4ABF0E0E4D180B805D86
:106F70004ABF0E0E3C180B808D4A870E050C01F996
:106F8000C41379C40C1B06434E3005EA6DCC66A6CB
:106F900006E0980F140179C40C1B2E53468D8C9C6F
:106FA000985606F5C4B94A851A09130C068889E86B
:106FB000B08BBF051A0913C15C4E70783CC62B0E0E
:106FC0001B841E30107046F0A1144E708C60DE9C45
:106FD0007E7E2726D4E30A061E5C422FFAA6E30E25
:106FE0008EE0E1C40459A4EDA456E63F3005426AA0
:106FF000AF089C581C38FCAA0A7C28E04E70383038
:10700000081C901C0A838D150E0179C40C600B803E
:107010001162940F12010B80696660B0307CDADA7D
:10702000FC3A307C0B00E00B00E0D05C3066603A4C
:10703000C60E3006A075227E477E59F37E19637E08
:107040000D4EEDDA3CFE4E66A63A5C105C223730FF
:10705000C6E3692ED05C30C6D7CC2B71CC66D35535
:107060000E7C1C30060E7A30EA592FA6D3CCDD0EEA
:107070005D1C4CDF71CC66BFE92EBF0E0E3D3C1887
:107080000B80714AF80E30E82BF80E3000E6AE6146
:1070900050600E5637300306E3AE8D080626D3E067
:1070A0007E7E895360065E46FAA056607CA647FC49
:1070B000A62FFCA6B5A2E10A814081C866BFE6857D
:1070C0006813A3663168C66687E61568D34BD05C43
:1070D00030E613E07CE046E098E0D91C788C2B8405
:1070E000D8842388D888D8F0492660A0D91C783C59
:1070F000D888D8FC9B81130F100B80096A0B80F98C
:107100006A0B80256A0B00CD9E0286C6E0BF0E0E7C
:107110003E180B80C54AD91C30126A5F78D88C1F84
:10712000881384D8F06330706A63411C30186A9DFC
:107130007E4EF0057E78E2D3411C4CC76100D144FD
:107140001BC17E197EC676C3A5D00C60C6762330DF
:10715000EE134696864686AE0E7C0A85D026E61C41
:107160004E8223A6A2A2A21F26E386EA02AA0AEA68
:10717000EAEAAACA2AE0856813E0A6062658D94496
:10718000E0EB5D1C214687010C060C0312B830FFB2
:107190003CEEB94A87010C060F14130B80FD660004
:1071A000203C56069CE23BA0005D1C21463087E057
:1071B00099050B1405070B801D6681408488ED64DA
:1071C000BE58300289408808AD402570BE981D60C9
:1071D0008CA7FE1F0E5B0E300555703BA00EAE0057
:1071E000D164EE894C690208A140257088A39310F0
:1071F0000C03100B80696E9807120C030B80C162A0
:10720000863E3C1815C845CCB87CAA3CA845CCF5B0
:10721000C4CEE8711E5CE6A616E61376A6E6E6E6A0
:10722000C6A6D414A3E09828C488C4FD7E3E4E3080
:107230002C5808304070387CE0304070387C063C78
:10724000A6BCF0E059A413A63040562B3001B61668
:107250006660A5D00CA01C4A2A704E5CAA0A7C9CD1
:107260004AA606F07C70383CA606BCF0FBAE0E7C4D
:107270001CAAFC0E3040562B3001B6167030EF06BB
:10728000383C66237666471C4A2A703866F308AE97
:107290000E7C16300156BF0670F038665BA63606C7
:1072A00070F038661B062B1C90D0061CE076173653
:1072B00070383C668B3001763F2BEDA45626E6668F
:1072C00030075A133AC6F306E6BCE2667CE62B4E5C
:1072D0002E1CEA85D04666064B66861C82A0A2A2BA
:1072E0007BC666A5D046A063044E70F8EECE71C88A
:1072F000700439D006B0BCA6700C1F08B30C6078BF
:107300003C06B03C063C068C3BB958BC70B95A3CB4
:1073100070E06EA05627FAA6F330030C1B660846F1
:107320008EAE608D0A304056A03001B616E00413D0
:1073300008081B04044E7038DC9010101028844498
:107340004E5870381CFCEADCD0BEEB59A4EDA48A80
:107350001CEAAB0A302C6A1F48B3885E5BBE980CEF
:1073600023AA3C1B7CAA581C6A3005426AF78A98FB
:107370005E630C2B3C58BEC37C1C9010CB2E5F1C54
:1073800038FCCA7C288C6F0C0B0CA0CC23D5886AE7
:1073900041A47B0CA0986815980EEE734C670C778F
:1073A0001C9DA47C0E7C0AFD1A0DFC0E010D05D956
:1073B000FE830512140507884B8305120C03120186
:1073C000840B80A152E54C0CA0983C063C4C3B0C35
:1073D00017060C13463CA63C9C4A0EA04E2F8C7BF5
:1073E0005C628E66665C1BFAA642EB8C13BE600D77
:1073F000544924F828AEE8B5BCFD5A064C2B48B0D9
:107400003C06CE7CA6FCEEB0FC061C0201D0840833
:10741000CEFCAA0A7CEEEDA456E6C6762697CE7C74
:107420004C1F26136603047CAA0ABCC6BCEE8CC3A0
:10743000B07CA6265F0C4FA646BC26BC703A4BA675
:1074400026E6EDD063FCEEE626E6EDD00C60438840
:10745000983CAA7C58E0CE7C0698E6B07C463C700E
:10746000B0FC70BCA63C66063CF0E093010516013A
:10747000130B8099568891D04E70F80E30025570DB
:107480001BB5A2AEBCEE514C4E70783C06F8C4FE63
:107490001388CEF61348A67C9C4AFE1348A63C5897
:1074A0003154BCEE8940A808B156BF0E0E3D3E18BF
:1074B0000B80A14A4E75F0EE600DFC0E0F200412F9
:1074C000091605F1FE8C06130F1049F0F9C40B8064
:1074D000E6E956BD56585D1CCC604C6060B03AE0A1
:1074E0008D0F0F120D050B809D5A82151314050781
:1074F000443390140507480B80594200BCA8E04E65
:1075000000704468780605BCEE59DE785E3E683C43
:1075100006660401AC0EC1B01C0C0742271D145BAB
:10752000AE0120630C77AEBC4D14DDAC4924E304FE
:10753000B1BCC36E6EC9A46E085346F059A4E5A44D
:1075400059A404668E060404D91078065830301CFD
:10755000622B30B062275613B6D91CB8B81C101C69
:107560008C3342B8302DE876B63CA23C3E1E7E7E7F
:10757000851849245DBC99C844785CE291DF308469
:10758000CC2766EBB371CC663F785C62683DDE3039
:107590009366FBC8CC2FC8CC0D541C101C02784C31
:1075A000BB426F765B6267A21C10101C021776A2AA
:1075B00068C34E5C6244D302FDDA3668F6F65BE2DD
:1075C000E21FF63378562268E201DAFE435CE223DA
:1075D0004830F02BC1B0BD1C03011420050D101460
:1075E00019DDAC080170650E4E9C90CC67601B7A6B
:1075F0001F7ACB8859C8550E1CA020E2F9CFD91CA0
:1076000078584924300501ECC27012C38700233B2F
:10761000B313BB0D549B8CE378068605BC95BC6602
:1076200086660801AC4359C85B785C42688859C8D3
:1076300051DE8CEB48C393011405070B80ED52001B
:10764000000000009805160113883398140507847C
:107650003DF0B0063C2606F9FBE6C622BC70067C6F
:10766000F03DD04E70F8AE708C2F38EEB94AAEF0C7
:10767000E048F9C446C10238467CA65849F0DDD43A
:10768000B0E622FC06023DD08A983C0A05CC98421E
:107690000C172E0AF9FB4EB07C5CD070FCE0900514
:1076A0001601130B803D6A4CE57A040D7CF57A0BCC
:1076B000806946067038F61366663C1EE0D09C3042
:1076C000583A1C3A30E63A30C64FE63F5C50D0D0CC
:1076D000F19AE60EBC427CA67CCA70BCA6F6F6F611
:1076E000E33A3A0E303C1E78AE7E3A3A306A677E14
:1076F0008E8EFE2F4A2F440B4A97BC430E98AE7ACB
:1077000030EA8304D88C1B8408D86A3F8E8E0C37ED
:107710004A77BCFDE24AE748B19AE6C532308306B3
:10772000CE3C566637B85CE2E2E2313238FC9CA2CD
:1077300062CF1CA23C28352EE0DCA0DCF2C156A0B2
:107740000EAE1C72CD564EEB514CD1C8E653D1440F
:10775000E0C4F57E7D6813BB664670385C5228A68F
:1077600058BDE0BEEF983CA6BCBE580948EEEB867B
:10777000983C70380EC67066E6386E33EE773A6E17
:107780005F300406983A7EB75826371568A30DFC7B
:107790000E0F201315030820010C0DF1FE266F2992
:1077A000E60948EEDB33D1C8E62B4670F828B8EE80
:1077B0004670CEF0F1688E1C527C706944E86E759C
:1077C0004CA8987038F6274E70AB98267038463C17
:1077D00005688D70CE0EDC52BC7026266944684563
:1077E0004098803D6A84050B800172840C06120368
:1077F000844393010C0612038801C8E6B5A2DC900D
:107800008C133E68BDD00881F08CA1C34E70780601
:1078100066263DC25AEEAE3C700698F00DD0A60624
:107820005870CEF070088C6366700201D030FF8D06
:107830008CA658980E0DD0A65870B0662F704EF0DA
:107840009B0C234E6EF0C102847E1788B0FC580654
:1078500070BC9C4A1CBCF004738C060C033EA5E86B
:10786000B07E7E2B89F63E8C1B78EE55F2BDD07D26
:10787000F20DFC12050320140F0F200C0F0E07F160
:10788000FE9208031010018408B5E00CAFCEBC06D0
:10789000B07C8C2FA63C707C26E6CEFC0AEDD0AEE8
:1078A0007C0E9806CEBC4630FF063B3CAA8D8CB0C1
:1078B0003C0698E671D8849803920803130E098851
:1078C0004349EA830512130E0904B5E00CA7B03C46
:1078D00051D8CE3C0E889826587C9C0A7C1C0AAE57
:1078E0007098E6EDD0B0AA7C0EEDA4AEFCAE8D8C07
:1078F000AE7C0E7C6A93846262901C622751EC021B
:10790000AE8C2FFC0E888B987C0AFC66588C9BB33F
:107910008305121010014404B9E049D8987C0EFC8C
:107920002BEDA459A4AE7CAE8D8C01D0986637584F
:10793000AEFCAE734C6030FF8D8E8C061A130512B0
:107940000B807D4A5ABC1A203C06B0303AE62366CA
:10795000DF461AE0411CF53E30EFB616666F300187
:10796000B670387C06562306B66666E09819050B95
:107970001405070B8005427924B5BCC10208D8283C
:107980004E2E687088C4651C0488ED060000000057
:1079900000000000000000000000000000000000E7
:1079A00000000000000000000000000000000000D7
:1079B00000000000000000000000000000000000C7
:1079C00000000000000000000000000000000000B7
:1079D00000000000000000000000000000000000A7
:1079E0000000000000000000000000000000000097
:1079F0000000000000000000000000000000000087
:107A00000000000000000000000000000000000076
:107A10000000000000000000000000000000000066
:107A20000000000000000000000000000000000056
:107A30000000000000000000000000000000000046
:107A400000000000810F1418F8EECE7EFE595A1582
:107A5000C89C5839B69209040D052E009170A56C8A
:107A6000BDCC0646BCA63CF0BDCC26BCF0883E4E44
:107A70005859F08C53C1B01C4E901A987C5875B070
:107A8000BAD33020E8B03000E6E6C67EE3E8B0DCEA
:107A9000D00EA1144924385E285DBC8001529CC2DE
:107AA0002B387C663B0D54663002C61306F5C44E77
:107AB000708CB551EEE8D5CCA6A62FB5BCFD5AC149
:107AC000B0BD1C04091220050D101419DDAC08010D
:107AD00070B902DC901BDCD0FE84480453DC501BE0
:107AE000DCD0FE0444848404040E30407030BF06B1
:107AF00038661B08634C537C66B5F7EE7CE6FCEEFB
:107B0000AE0E3CA63C263C0E0C7F7038AED86E17ED
:107B100088D8AE2E6F8C1B6E582DD00CE7A6067041
:107B200038FCA6067C7026E63DD00C6F4C278C5F97
:107B300083CE7C6637FCEE4B84AE0E3C06704E6EF8
:107B4000F00C278C6B8485D0C6A686A6A5D046935C
:107B500030EEA62686065C424F9B880C2FB0BC16E2
:107B6000DEBCDEF376E30DFC060C2014191005D9FB
:107B7000FE0DFC060C200E0F1420060F150E04F14E
:107B8000FE1C3040704C57AE0EBC06387CA6BCF0D4
:107B90000CA04E2EBC30BFF0E09208030C05048808
:107BA000438305120C05048449F08808E9D48CF954
:107BB000FB8C7B4E7001C898A658CEBC06B07CC624
:107BC000E698A60627C6DB0686A6467098C606581F
:107BD000CEBCA6C63CAA8D8C98E63C0AEDD0987C1B
:107BE00083B07C46707C707CF0CEFC0AD9D0CE7C11
:107BF000AA0E84EDA4F0664BB0561C2A13886A1CAA
:107C0000F0AE7CAE8D8C8C60A293A63040562B30AB
:107C100001B616662F70383C06A2A2A28CAFAEFC4D
:107C2000AE88338C06121510A068A5E88EB05A589D
:107C30000881F0986E46262642EA4E7078063DC3CB
:107C4000BDCC46BCF0AE0E3C0A3DD0BA3CE6A670B8
:107C5000A638EE70EEF0DA3C66A084A63040562BD3
:107C60003001B616661FA5D0668C27887B98120552
:107C7000160113883B9812140507843DF0B058880C
:107C800091D0B0063CC61306BCA606BCD870E63C34
:107C900046268326E698A658B0FCA61C223DD0981E
:107CA000EEDB92140507843B920516011388DC90E5
:107CB000FE95E8C15C4E70783CC6A660E6B00697BB
:107CC0008C730DFC050E04200F0620060CF1FE66D9
:107CD000A6C686BCA6BCFAB0FC060DD07AB0FC7075
:107CE000BCC626BCF0AE7084448C57A67CA63CA6CD
:107CF000700488B308849B90011713070512484B42
:107D000085160F0D070512448491D0E613667006A0
:107D10003C063C06B958BCB958063C0627883C705E
:107D2000B00E3CA6BCA670840404B07C7038EEB0E3
:107D30007038EEF04C33B07C70CEF0B03C66603CF6
:107D4000048C7F8C1B661326700C600CEF3C080CB7
:107D50009B700E2DD0B0A68BAE7C0EB0E622FC063A
:107D6000023DD08AAE0E3C0A05CE94100B050513D9
:107D7000844B8114100B0505138889E84E7001C8E7
:107D8000FCFA1E7E7EB0FC70BCA6063C463C7080B1
:107D9000C15A94100C031284438114100C031288EE
:107DA00089E8B03CA6F5C4CEF07C06F5C46EA05AB6
:107DB000233003C6B01D60EEB94ABD1C2005121267
:107DC000DDAC080170ED8AA188C1B0BD1E49240454
:107DD000CDB4734E5C90D0D010309C6262BDC06B4D
:107DE00049A43DA48A3DA4E5A4581C22071CAA5816
:107DF0008CDF6AED1898EA6DCC3010701EA114D992
:107E00001C7E9EBEB8BEF37EBAFC8518F90E46F005
:107E100070B85CE2E2E24660E21BAE4BAEBC067CB0
:107E2000A63CA63C5EE00000000000000000000050
:107E3000000000000000000000000000000000043E
:107E4000320605E80000000000000000000000000D
:107E50000000000000000000000000000000000022
:107E6000000000000000540000000090010000002D
:107E7000042AD08822282280008051018045028077
:107E800001C05504C0242200602411005400500198
:107E9000400500240204100D2002C05000000C0C0C
:107EA00000E0344FC8834F8A4F3C372C8E20C13BB3
:107EB00008E168100D204E064065F3B8144DBFF47C
:107EC000830892220159C91D744FCC78E4452FC212
:107ED000F1020054D450C1D8C430FD3A06FE876187
:107EE00030164E418660434BC43D898BBBD1D3BB1A
:107EF00003101151D100034035312DE212133131FD
:107F0000D5C1725031E04C0005D10444151E5045D6
:107F10005D4C762F03005C000000194207C9C400C5
:107F200040660216F6460522501012B4CD460A00ED
:107F300019007400318F4F40384454F37F2B414770
:107F4000888714E04331410F3C4A34900994114032
:107F500031416630CD2823514ECA60CAC01F8FC23E
:107F6000E72F0801B60501C2C8105D07FC221030DA
:107F70001100FB042244448C738748E0C4073D038E
:107F8000A3064AA480C1084B31C1142013044B033B
:107F9000D60F1B02023D0CC1E724E200510860002D
:107FA00080000052D147842000923374CDFD6405D7
:107FB000C11111040004F04020800661761402C44F
:107FC000046400120012EE450D0511A08039001066
:107FD000214841005238B18C40225015F705005419
:107FE0009C0B00600020409A25CE660040050002F0
:107FF000205D3EA92686E8B534D00C004033C1414F
:1080000049C223A37463C71333CDEFD271885210D2
:1080100027BAD2E3C4B84EF9F3B5A78448F623C211
:10802000BAA24521A28D6CF63300004E32C884B846
:108030003260301D0100104CE98608B7203B2AE170
:108040000E0019000008804278001A0A8202800798
:108050008F442200215410E1417004001D65155D1C
:108060002275F3B8E322C140244354689FA88F2FA0
:10807000638F854B8B3D1F4FBCA244C05C357A9FFC
:108080002B0896D4C515724F45A1214505910921AC
:10809000A130E24429BD290000603C981F8E04886D
:1080A00046688191089282470BA9C55401110002CC
:1080B000008620A2833C683D4096408924020450FB
:1080C000018980073A8A500A640200E8C0A48C083B
:1080D0000000600080C1612444020555582C001442
:1080E0006001800E00040F809961104400090010A7
:1080F00073CD003C7D840900500011C8000049C0C8
:108100001D00007494D4CA63114113480DD40000BB
:1081100051DC7098191300000000000000000000FE
:10812000000000000000000000000000000000004F
:10813000000000000000000000000000000000003F
:108140000000000000804A0C004046139123020901
:108150000D54171D53B58F34215E94A016110436AB
:1081600030C5D10C0080938C20000802F01246CC60
:108170008002001448273487818990402022708231
:108180008153890231057041D43D51242300600898
:10819000000060100215828F8403800080427218F4
:1081A000468451C44820514800511110204241B426
:1081B00020B02C00F0514CD008550B3C0009404831
:1081C000A4803E0352098180487F314103FC038033
:1081D00000A010420451019D4400480420002800E2
:1081E000E0D4302200008640040480620208117C42
:1081F0001F0000000088488851C41004C14B02824F
:108200004022380C8838C693C0144008540000033C
:10821000000C184081124404C000C0000454E04423
:1082200000308093CCCC4406F5BF5A318CBC414021
:108230000484CC403708C25EF501D4080C0000006D
:108240000000004000F8615044FE1348260E767688
:10825000B5A3D91C78D88484D88C1326F046F009AD
:10826000C886E64B309EA62BA058F142CC2766EB81
:10827000A3D91C7858203C56069CE21B4EAB30120A
:10828000664761C86686A568E330C4064FC64ED00F
:10829000A646263CA3E6761C4E906AC6FB303162A9
:1082A000276A13A662AA3C26048C2B08A07E60587D
:1082B0005D1C98BC9CE22B0602A2E6C602A230031B
:1082C000622F1C42136230088C270C237B0C134650
:1082D00030555EFC06BC30E61BF61B2E03068C2FC9
:1082E000C16813C3A60EA05A7C1AFAFAFAFA5623EA
:1082F0003C3AFCEE1A46BC26260E55C4604C610082
:108300008859C87828B86898A859C4EA005ABC1A8D
:10831000B0303AE62366DF461AE0BDD065F04C2F58
:10832000A18002DBCC3F4E70B8584C7BCC6795A443
:108330003C0A59A4E5A4D88C1744A180FD188A856D
:1083400014064E70CA685878A6C6026A6DCCB05E34
:108350003C062B5DC4C830DA7004B07C0E01D0ED51
:10836000A4AE3C667F7098AE59A48D8CAE7C660638
:10837000FC584304987C1666C3084E70980E780625
:108380001BA668780E59A430C08D8C4DA4468D8CE8
:108390004E5870780E4C23C4BD8C783C667BEDA49F
:1083A000D884D88D8C29A429A4AE0E584E70780E8E
:1083B000B8BC5884E0DCA0DC1050121C8AE5A43C58
:1083C0005CF2CB7E0F02FF1C8A4DA4EDA47C6A22D6
:1083D000D398AA698C0A588C574DA459A4468D8C01
:1083E000980A29A41B1C6AF5A89B623C5888821B2A
:1083F00059A4468D8C42D762101C021F023BA66610
:10840000700A4EF098AA698C7038989C50F09806C3
:10841000467078A6682E063B6670EEF0EECB4924D7
:10842000F85A5EE830BF2684A80E78AE66CB703866
:108430000E4670AE3E8B1C8C137CEA330EFDBC9551
:10844000BCB88C1F884B781C0A29A429A4B8AAA8F8
:10845000A1801C3988E68F0C2F59C4F0000DFC0355
:10846000080B13150DD9FED5883E434670AA680A3D
:108470004DA4E5A4AA704670785816468386FDBCC4
:10848000EE4B66B8FCEE0825AC1B95BC780EE3D12C
:10849000486E2B59C42E1659C41916D1486ECFA355
:1084A000D1489D48FE738BD1486E4BBBD1486E437B
:1084B0009D48FE23FBD148CB4E3E304C0EB87E5B30
:1084C00081C806783C06B9586E63AE6E7F3A3A3A78
:1084D0003A3C70380E8E844E70F8E030546E9B300B
:1084E0005A6E73666E53666E33B5A20EA04E3E7E14
:1084F000C37E7EA07ECE7E574E43EEA0663346F608
:10850000A0BEE04E5EE76EE0CE7E1B5EE0E0DCA04B
:10851000DC5EEE1F237CF2F3AE5EEE1F237CF2F3F3
:108520000E03E0A5CCBC0E4670AE6881F04E7078AC
:108530009A66AE68304070AEF03E55F04E7084B032
:108540007E7E7E2F7E89F68801C8E6B5A286B0665B
:108550008DC61C06A54FC678A6063DC358B0FC06BE
:10856000707C26E6F002223DD0AED8E63C700602D2
:108570003DD0B0E60CC38604304006A5D00C49D1EE
:10858000C676431C0A6AA5D049D066B0E6C67038E4
:10859000A670A6F0986666776651ECA606704EF057
:1085A0009866BF8DC68451EC8C276688D326E6700A
:1085B00022FC06023DD0A658B026E6FC063DD09827
:1085C000BCA6588CA3BA44DDD47AFA9A983C069893
:1085D000767FA606BF0DFC060C2013091A05D9FEEE
:1085E000A5D00C9798762BA5D00C5F98E63CA6B04A
:1085F000FC707CF05DC40A3EE6B006A63CA60667A9
:10860000BC704E70F8FE2F66A6067038EE472DD06F
:10861000983C66AFBB0000000000000000000000B6
:10862000000000000000000000000000000000004A
:10863000000000000000000000000000000000003A
:10864000000000009CC2FFCC574626FBCC2F5DC427
:10865000243C71CC6653309066FBC8CC6100839C8F
:108660004262E2A5684E9C90CC5F601B7A1F7ACB79
:108670005DC4E01071CC664FA5689C228859C87B08
:10868000A568D91C78583012662761C8CB30C266FD
:10869000AF46F08C5B59C8BDCC66E627652073BC3D
:1086A000F05DC4293C26662F8865C82B49F08804F4
:1086B000E9D48C2B5DC47E3E4E70088C2B45400661
:1086C0001BF9C43018A6C6B07CEEBCA686A6061F51
:1086D00004A666983CC658B03C0671D84E70B87C6B
:1086E000D8040C1308D8BCA898668DC77C0EEDA4DE
:1086F000E601D0AE3C58C69C584E7051B41C53BDD8
:10870000D0C1D85E3E2DE0DDFCB1C0BDD04C1BE930
:10871000D071F0B0FC700602385AF051FCAAAE3CA1
:1087200058C9C099C0980A01D098AA0A5841C48073
:10873000E68741C44C5780E6AB708D8C987C0EB0B8
:1087400004D88C1308D826CABFAE3C580AB0665766
:108750007001D041C4808D8CAB0C2341C4804B0888
:108760001304980A30FF8D8CA156C1D8BDD04CD9C6
:10877000C85E7E7EFE39E098EEB5F604DCD01EB011
:108780007E7E2F087E29E331F40C533E85E0B05EF7
:108790003E7095F059C0B0CE46CE6E6E68BDD071B9
:1087A000F04E707858B0FC060201D0EDA48A045651
:1087B000705C0A0676265766D88C1B086AD86A6AE7
:1087C00098AACAE7AA581C4699C4B0A1C46AB06660
:1087D0004F7001D0EDA4A1C4B30C7B46A1C45B08CB
:1087E00030FF99C4640530FFA1C469D095DC0C55F5
:1087F0004AF9FA38BCA6BC288804E9D48C434E3028
:10880000913CEEE95ACEBC06B07CC698BC1ABCEED0
:108810004E70385CAA581C06BC065F3C0EEDA4598D
:10882000A4E6AEBC0EEDA4AE5884C61C6A17881C24
:10883000987C66E61F8CAF8CFBFC580A01D098AA86
:10884000BCDBE1563BB03C263C463C7098E63C0A1B
:10885000EDD02E8449D463BC6658CEFC0A01D0B05A
:108860007C263C70983CAA7C5806D3B0FC707CF007
:108870005DC45E3F7E2F06ABF0837E7E89F788481D
:108880000DD4CE584E70F80E8C2BEEC3F9FA3DD0B5
:108890000698BC067F0DFC050E04200F062012056D
:1088A00003F1FE66B03C065DD8554AA5CC06BCA6D1
:1088B0003CF081F0D5CC663002C61306F5C459C42D
:1088C0002E12000000000000000000000000000068
:1088D0000000000000000000000000000000000098
:1088E0000000000000000000000000000000000088
:1088F0000000000000000000000000000000000078
:108900000000000000000000000000000000000067
:108910000000000000000000000000000000000057
:108920000000000000000000000000000000000047
:108930000000000000000000000000000000000037
:108940000000000000000000000000000000000027
:108950000000000000000000000000000000000017
:108960000000000000000000000000000000000007
:1089700000000000000000000000000000000000F7
:1089800000000000000000000000000000000000E7
:1089900000000000000000000000000000000000D7
:1089A00000000000000000000000000000000000C7
:1089B00000000000000000000000000000000000B7
:1089C00000000000000000000000000000000000A7
:1089D0000000000000000000000000000000000097
:1089E0000000000000000000000000000000000087
:1089F0000000000000000000000000000000000077
:108A00000000000000000000000000000000000066
:108A10000000000000000000000000000000000056
:108A20000000000000000000000000000000000046
:108A30000000000000000000000000000000000036
:108A40000000000081C8E6B5A2064540B9CCA6BC2E
:108A5000A63CF04885F08C5BB0FC2670381CEE77A5
:108A6000709BD5CCA04E70EE59C4EA003CEAF30EE0
:108A70004E70AE68B01E4E3E1CBEBE3350105090BD
:108A80003B10BE2B10105003BE2B5050D0D3B0461D
:108A9000FC06F5C4A3F85E5AE8A878E630C00626BE
:108AA00063A60670383E334E7EF066A3A1803CD5A7
:108AB000883E7B70AE0E584DA459A4468D8C980EFE
:108AC000B0E66F705DC414218A4E6E56DC90688DDE
:108AD000B8BC08983C28441C6A8AEDA45606303A73
:108AE000067B303006AF3020469C58DD201C6A4E95
:108AF00030056A5B59A46A4C8FEB48783A87783A1C
:108B00008DC7B83CD808D87CA88CB5515DC4333B20
:108B10003045663F783A27301B83302B66832666C4
:108B2000378C7F301A23266627301CD32666678C45
:108B30009F4C4353F8EECE71C8700439D006B0BCD8
:108B4000A6700839D0E6172606B0BCA670783C0699
:108B5000B03C063C06B958BCB95826703C063CE609
:108B60004EA670A6F0B02606C78DC60E66176629FB
:108B7000C6BC069CE2D330901C02AB30316A8B300D
:108B8000460217669C024B501C62276A136AA6A60F
:108B900006C6E6A2065E233008465DC46A27F9C40D
:108BA0000C2F7015C8E68DC606F8FEB0C6FB46DE73
:108BB0001BA6C6A67079C4AA58B0665F701C980A36
:108BC000EDA49C58461C8D8C51B47B4E1C10CC2FB0
:108BD0006EEB4E4B203C56069CE21B4E5330C406B7
:108BE0004FC64ED0A646263CA3E6761C4E906AC6DB
:108BF000FB303162276A13A662AA3C26EE61005D53
:108C0000C42E1230FF06F8BC66470EB8A6AEA88D7B
:108C1000C6B8BC66B5A3840895D0302B06B006272D
:108C20003C061B810A06B8BC13EEA6F30EB03CE668
:108C300030A8AEEE176668A69C583508B0063C26EC
:108C40000677BC70783BF87EFE5F5C10EEAB1C7C58
:108C5000EAF33C3315C83C9C4A7079C40C2F8AB0A7
:108C600058EDA4AED87C1C846A1788D8AE987CEAEC
:108C70001F8CBF4E30051C6A538C2F6A59A40359B0
:108C8000A4034E7030913CEE3B79C46DCCF5C459D1
:108C9000C4EA00BDE0DC101E46FCBE77E6A6700606
:108CA0006638EE7066EEF0BEAB5DC4EE00307A66FC
:108CB000FB610278E8380E38D81CAA28E09CA01C7A
:108CC000380EF8AA7CE8AE7C280EE0D4948DC7A0BC
:108CD000EA73E2679846AE283B48084EDDE04E3026
:108CE0000BAAA0FA60E6133AA6CB3C30030E51C49F
:108CF0005DC42E12B87CD83C30300693302E6637D7
:108D00000C60A6A6E0300D664F302D06E0303A0626
:108D10006061DAB1D0AE0E3CEECEFCEA6DCC666698
:108D200086664E3007A63AC6F346703CEEBCC6686F
:108D300004044CE1C4E9D00881F08C4BB07EFEA164
:108D4000C3A1F4834E70780666263DC2EE4E9CCADF
:108D50001C3E70AE3C06027098F00DD0A60670B0B6
:108D6000F07A4670CEAA7C0EE5A4E6AEBC0E01D029
:108D7000C68D8CB0A626A67A2770AE5B7001D0B0E7
:108D80008D8C0DD0A6704E6EF05DC4F00049243875
:108D9000FC700638FCA67C70E04670387CAA0A3C61
:108DA00028E0040484E9D4983C1C0A0451FC4A2AB3
:108DB0002AE030600698467004261C7C4A300AFC83
:108DC00058B8A6A8E0D91C78D8E0EDA40616D91C9E
:108DD000303A6643302C6623302E6661DAE0B1D03B
:108DE0008E0441A444CE0637662FA20217484ECA0D
:108DF000686A054600000000000000000000000056
:108E00000000000000000000000000000000000062
:108E10000000000000000000000000000000000052
:108E20000000000000000000000000000000000042
:108E30000000000000000000000000000000000032
:108E40000000000088DCD0FE95E84E705C380AB067
:108E5000AA2845D81388D91C78468C1326F0256C8F
:108E600088080404E9D40C5B44DDD4CE7C06463B80
:108E7000A6265DD8705B7C0A556CB03C46BC70C5BC
:108E80007E256C044670387C1C0AEDA4563CAA7CF6
:108E9000EE3BCEFC1C0A556CDABC06B07C063B8669
:108EA000BC065DD870DA7CE6917AAE4670CE68C1B9
:108EB000B0E0B07C06300B0697300D46DA7C063306
:108EC0003017C63E9306301806BBB03C061EA114F0
:108ED000F87E7E9E066646F098A6581CB07C26E674
:108EE000CE7C0A04EDD098E67CAAFC58CE7C0AED34
:108EF000D098AA58CE7C0AD9D0DC101E9E9E1C9811
:108F0000AA58040893EDA48A06D91C79B01CCCE7B2
:108F100046F06A01D0987C6A6F98DE586A8744D917
:108F20001C987E2F581EA9763020E805768A4819AD
:108F30006C4479B098DE1EFCDC901E1F5E1BBE5E8A
:108F40003C5883EDA48A06D91CCC33D9B0083576B9
:108F500079B01C6A46F001D0986A63DE3FFCFE9B44
:108F60000C8BFEDE04F3D91C0CE37E9EBEC7F8BE5C
:108F7000F3A3D91CB8F8568A063040C64B46F06AAF
:108F8000196C1B79B0980C37FC1E9E3C1E3C9CE271
:108F9000042030F0E6E09CA0443020CC697766E302
:108FA000C6667977E699C8D91C9C6282B8A2F34C50
:108FB0001B98F306E094339C98A60658A0D88444E6
:108FC000D84C77C6A69C58301F6617260698069C74
:108FD000E8D09C0282B8A2F34C5177485576203CE9
:108FE000F64BA568711C5DC4E01078581A7A7A4E69
:108FF000203C5A1C5D001AE000105B504B903BF384
:10900000D0230000103C56063044668F788C1B84B9
:10901000138884D8F0A5680C6973517626669FB0D2
:109020007C06668C23300B4686BC0646F05DD8C9AC
:109030007A266677B07C0646268C1B300CC6530613
:1090400043492478FC5CEAEE9C300842A17CF6DDC2
:109050007B30088C1F4200957C068C47C1681BC181
:109060007A7C5898A6588CBB796C4A57C1B0BD1C05
:109070000E0F20120F0F0DDDAC78D884D8F04924E4
:109080006D58610030FF66675ACCE3203C0630C360
:1090900066DD7A697288489806C96C25E8E3CEBC1B
:1090A00006B07C662326E6CEFC1C0A04EDD0988D23
:1090B0008C066686B03C0671D8C97A3008957CE685
:1090C000EFDABC061C3001667FE6CEFC0AEDD0303C
:1090D000608D8CB03C9D7EB07C667766C6E6A658F7
:1090E000BC065DD87C26E633C626E6A658CEFC0A2A
:1090F00004EDD0983CAA7C58066611F4D3F6278C70
:10910000557B1C06300825400E7E9B9A0507088774
:1091100000D36B3BE3FBEBD323DBB17E75F44670EE
:10912000387C0AEDA4567626A3617E056C8C1B84E0
:1091300013883D766520056C8498F0A568F57279F2
:109140006C0AA17BB96CB0684829E84670787083D6
:10915000BB843BFB796C0A5788CEFC0AD9D0B03C63
:1091600026BC70EDA456768CEBE6556CC6263FAA5D
:109170007C5CCAEE83B96CB0FC5CEAC41C59E8059F
:109180006C8498F046F01B056C8C1B84138898F057
:10919000C97AB03CE6C17A6606265DD8056C84982B
:1091A000F0A5686972267F556CB03C06265DD80B29
:1091B0004666E68859C804C1B0BD1C07140F201EBE
:1091C0007E7EC63C30033E1B30017EFCE8BEB3DD34
:1091D000AC0C3B46F0C6E10803A5684E5C10901A43
:1091E000CC4F26EB99C8BACB7976300B01ECC3840F
:1091F00074348575358676363700233636363636FE
:10920000363636365B65209300000000E080E006CD
:10921000C61C22471C8622279C860882CD7EC61C3F
:10922000222B1C22DD7B02A29F8C174230555EFC54
:1092300006BC30E0000005CAF3EBE3DBD3CBC3038D
:10924000180D1467308AA630BD8B72201165E34F6C
:109250000B1D102350C604A89C60C74C81496A525C
:109260001BF515F314124485B60825C6205B15EBD3
:10927000A2262A0A400C50AD3C362203820F00354C
:1092800032388184D80400CCC040819010038074AF
:10929000D184F5B04DC000A409302333CC5068BB55
:1092A000881F88FB0D8C8C84D4CC0035C0A80303A8
:1092B0003C31818621F25B38338A1CC3A1362321DD
:1092C000B22485E82ECD8843480C08000638622376
:1092D00080C71082B02066CDC040FD657EFDF5E6FA
:1092E000D61831D118C0A82221727CBCEF43E2F01D
:1092F00030E363BBEF0C2320EC20ECFF10A2A08036
:109300002122282A8221C0C3953C412282101102C9
:10931000821108CC04002088310089FD0CCF0B108D
:10932000420849919D3055C3080018E00D78008827
:109330000350F08134242AF10200000000000000F4
:1093400000000000C9E0331053FE72482113E2030D
:1093500031158A351D23C6B0CB28320EF88A423229
:1093600003980C40102131411204B81BCE3925005E
:10937000C520F00452D9C408182044D91544914698
:10938000A603153D6D50210009076954011693A1EC
:1093900050421A4A1B050452C7AC8EA041801040AF
:1093A0009A4F5D11040481004227644114441785DB
:1093B000A224434861542468441EC98009CD33A1C6
:1093C000DC50106A821041C1B3060119452588039B
:1093D00033D64043482331E50800000610D0142955
:1093E0004304310000000000000000000000000005
:1093F000000000000000000000000000000000006D
:10940000000000000000000000000000000000005C
:10941000000000000000000000000000000000004C
:10942000000000000000000000000000000000003C
:10943000000000000000000000000000000000002C
:10944000000000002134432432A02C3222037A4849
:1094500084141117C54108160E3BD19008DA230871
:10946000D40C50B80320AAC428201417170E0031BA
:1094700083AAAE737F3703F17A18EB40E8C42EE37A
:1094800040E044E088114C2046211420D24F22D4E1
:109490001E7F7C8C3FCF143D4D34004238019D101F
:1094A00008E150320030344E4207C404A89C60C723
:1094B0004C81C84045D3F0D0801231CC44D4014116
:1094C0002433841B8E32F62E61200609FD73B40C02
:1094D000C10CF38C2108C44098186081620F848B02
:1094E0009EC0082708C70FEEC5174060865D24039D
:1094F000B731315CC744C7CB5000504464238493D8
:109500000C32E88C683D00088509240A60020400DA
:1095100084C00000880E841800A3512E4891801E3C
:10952000850804894F2F313131B13C1432C30852C0
:10953000000000000000000000000000000000002B
:10954000000000000B801A2838215A847209340167
:109550005C0504956824000054180D059034E24819
:10956000C5443411140F3113C411249811405844C8
:10957000587841C4084D700CC447E3244571A119C3
:1095800091368087D0CC54010C8D2B033B03713373
:109590000F45304634D6061D20F4E668C80037442F
:1095A000C8516C4B4C8C214BDD14E55131D0141E4D
:1095B0006300C0004931CDEC56540E954414C339B4
:1095C000144A3487064767C5C435C67D44753300E1
:1095D000E0B41B232DBC141F595580D10A901110E3
:1095E000105C9C61C4004500148D41050909414689
:1095F0005124C9447155591055508296A0968978C6
:10960000626E514D85094A4DF5430186E0510808C7
:1096100016C68CB19C01B0079E01E6167941C08840
:10962000F20C200521A1F70C331654E3D2160000EA
:109630000090AAAA884077282F3FC5A2474B85F6FD
:1096400030FF3F880106B5064E70F858985684D80A
:109650004C5B8C4B4C3B1C427070384BAE783C06DC
:1096600070B958CE8CA08D08849B76761908AE58B8
:10967000FC58F3999E990AB5960D9E1596BD966273
:1096800062C6CA501C231908AE58FC58E21BE237C8
:109690001100EE5C981C45028CA08411008D0858C6
:1096A0000CA0B5A27B9BCBC313E3DB4B43CB3B436B
:1096B0004B535BBDB25100E30E1C5016B523110C89
:1096C000AE0E93C48370FA70A033F0B80E6150F8F8
:1096D0006550C4F07C30147C3050BCE0C8CCF7300E
:1096E00008C8CC66EBE0D5884FA550F0D44FA55004
:1096F000D43FA8F0EECBA550AEB87C58AE8CA74CAA
:109700003344983CA883B5BC84634C610043130088
:10971000A550EED4D3B87C588C33A3B070E0A550DC
:10972000EED433B87C588CC378A84E703868F828CB
:10973000EEE8B5BC8860A04E70B85860434C37481E
:10974000ED04711CEC1F0C1B919CCC9BCCA3203C0A
:10975000560630186621463087662F110C1D02C848
:10976000CC5C5AD07038CC9704624728707C301497
:10977000FCE09066281C70381B2E28BC30EB33B8F8
:1097800098A8E000A383634323387C8338FC6B38BC
:109790003C53387C3B387C2338083C8C1BADBC30B8
:1097A0000670FCE048711C8C7F0C238914538C2BB1
:1097B0000441B023F8992C4C3F305166FB610044C2
:1097C000ED040CC70100D50CCC0F3008999C0CCFD0
:1097D000B83C580CD91C6000711CEB592430500661
:1097E000CC4F300CB19CA6CB091E201CE2153221B7
:1097F000460100E0D50CCC3F300A999C0CBBB8F177
:109800000C7CD804884484D83C467CA8C46100CC35
:109810004B30C306203C1C6ADB78EE30BF0E662658
:109820007BA6067038EE4B3EB75EF0FC56468B309A
:109830000770999C51844E7020B8BC588CC5028426
:10984000983CA8E06D5820091EC8CC6046F07030E6
:109850006906787C660FBC6670380EBAF038BA6E4E
:10986000B7F04670B858CCA03846BC30E660C47833
:109870003C1C420ABD8E60A05870585858707070D9
:1098800070E0DCA0C44484C44404B1702DD91C61D0
:109890000030FF0E4EF0E020F0AE70AEF0A6DB30F0
:1098A0009C3C30A73C309B685A2E28704E9C103050
:1098B00020E84E709C90105C1010A8883006999C8F
:1098C000306906787CA63C68D5060ECC1F4CA038C3
:1098D000CC432E28BC30B606E00C6B90662870385E
:1098E0007C1C0A1C4E70E06228E01908AE581C5817
:1098F000F6BDBE44F64348F62BF6603D02568C3367
:10990000841100B10EAE8E301EC63F4CC3301AC655
:10991000A36E3008EE4E702E3C86F313EE66F3EE27
:10992000B8AE3D02D588387E7E8953065E04467007
:1099300056607CA64708FCA627FCA64B3CED08E633
:1099400006E6E64646FC06E01C8ECECC474C377851
:109950004C1758E0CC8338BC3AEEE2DFCE308E1A9A
:109960003C7E1E4E1CAE3A30AEAA3CBECB133CEA47
:10997000F358AE6E1C53CE3A303C46FC6E1A3A3C5D
:10998000EA38CA28E044E23349A459A41B49A4E5B3
:10999000A43C1E4EBE4F58E5A4D898D83CBB2550D9
:1099A000581CDD8C6EB858E065BC8C1BCCA00448FC
:1099B00041B0336DBCCE992CF90C8C2F3C580C6700
:1099C00065204670B85888D3C4B83C5804987C5871
:1099D000042B4924B8587CD804D8FCD88404D87CFB
:1099E0008498A8E085BC390C048CBBB85804ED04FD
:1099F000C4E0B01A30E61B1C50BCAEC1B0AE4D1472
:109A0000DDAC492465205DBC651C4C752EB85888BA
:109A1000987C5808983CA81D02B85884987C580433
:109A2000A341B0F90C3330A7C8CCF91E66DB2DAAD0
:109A30008D08F6810B1C98B10A30FD70F0B8150A3C
:109A400046A809BA8BA3ABDBB3ABA39B93FBA3F3F1
:109A5000032B23C91230CFA663B51230903B1D14DF
:109A6000091230910286061D146684E37330D043D8
:109A700030CE066365169C021D1411B41DB4D88443
:109A8000D81B30A80629BF30AE06AF19B4D8D91CF0
:109A90008C2330E01B30D02D149388309C06138427
:109AA0001D1411B406D91CA6D88C7384D884E6BDC5
:109AB0001C090E04DD14661BD806163066066B1EE4
:109AC0007E8C177EA1140CDDAC5D1E307006C7665F
:109AD0008B307466D3069B3071463C301A7E3766F5
:109AE000EB305C46E80B3065DB307A4636BB3068DD
:109AF0009B301D06CB3B301A06CF6667B8D8485C52
:109B0000A2E21788D8E88B266637DD1430053B3093
:109B10002D23A61CD0E51411B46E5606D91C301D99
:109B20001C621F06970C2B301FE5140912E6161D48
:109B30001411B46E060404CC13081C02A65A56BCB9
:109B40001AD91CB83007E8BAEF6E49241C0C2DB5A1
:109B50000CE5A46E06D91CA675B0E9145B6E3DA495
:109B60001DB48E06D91C1C627330CF2D1449246E8F
:109B70003DA46EAEC512AA625830C02D14CCEF8C35
:109B8000DBE0B8B83044E86914061ED91CA11430D3
:109B900020E8F89CE213A83060A820045330C8489D
:109BA000C8CCA066E34404048449242DA806864C4E
:109BB0002BAD704393C1B01EA114C66FCC4F691476
:109BC000061ED91CA11409123020E84924B80E4100
:109BD000A41DB41CEAE38E56063C3040FCE0BD1CDC
:109BE00020120507204924785A0E43660E7038EE7D
:109BF000477A30C0661BAEA3AE3CE03020E80C577D
:109C0000302006F8A85666A00879B2D91CA6063CF2
:109C100030147C301C50BC087A3056D84C1B36446B
:109C20008C1B0484D8E80C8F3020E8E09E4EA0A660
:109C30000E3C2666EEEEEEEEE6A63C266606BEEE90
:109C4000EEEEEE06AEFC2E6E0E60DE77DC101E7CB5
:109C5000FE7FFCBEFE5FFCBE437E9EBE1F3CEB7ED5
:109C60003C1A9EFC9CBE603003FCE8D34670CEEDEF
:109C70002804141308AE58FECD7DE05CE0D460D01B
:109C8000DC6202D7629362E97CE0C2E223302C1BE3
:109C9000302ED4A0D57C33E97CE0D414030CA01C76
:109CA00098E217D4A03045D57C98F6CD7D7B1C3842
:109CB000BC44137A3076EF76DF7617483C0AE0CC66
:109CC0001BAA733988E60952D5883ED74DA6251CB4
:109CD000D91C3020E81538004C73B0E22F302DE845
:109CE00013B8957CD91C7B30C30E203C0A23652019
:109CF0002B4E203CD026E806303404661708B0C648
:109D000006C61CD00C1BE21722E866F13A0E304161
:109D10000660304B06F3302506FCE61C0A301E6A4E
:109D200023666A37FC0E66813A30CD6A2F3C3E3E90
:109D3000A366E030610660306606A0301ADBB03CF6
:109D40000E660401AC0C0F1CE22F0E16913E700142
:109D50002053AED80C27B0B13E088BC1B0B1BC497E
:109D60002444B0A11CF93E589DBC981C1D88FC1EC3
:109D7000BEBEDDA44E70E5A4D8B0D83CBEC325500D
:109D8000704670B068301E7CA11C0441EEB83CD80F
:109D900044D8FCA8D91C78D884D8F04926410CA80E
:109DA0003080A6E64EF070B858CC1F0C1B66664C8F
:109DB00017168C136E3C588C233080464C2F8C2306
:109DC000767676BC588C2B76767676BC56EE3C56FC
:109DD000EEEE4E30107030FDF0AEF046F070B85838
:109DE000E07CD80CDD2F580C2B30844D320CDF89F1
:109DF0000C4C3304B170434BF8E61F26E865144C55
:109E000019387DBC651CC8F84666E8B858F6F62BCC
:109E10009DBC410C04B898A859248C47C1B0302E81
:109E2000A84924C1024E28E8A89868E0FC5C0AB85A
:109E3000AAA8E0B030E83AF6E3E030107030FDF068
:109E4000E00000005AEEEEFCC6E6E6C63C06BC5C4E
:109E5000EA5A505C30662B22E399C63AC60E3006A9
:109E6000C3A6E67A5ABC1A30F6F63C58FC0E3C3AC9
:109E7000301C0A3C5AB03AE07AF30438BC585C987B
:109E8000FE9526FC10D0900EEE7E93EE0C31237ED4
:109E9000DBEE7EA3FE13081C78221BDCEB1465238B
:109EA0008C27787E6881228CAF88DB780EDC901E50
:109EB0006F080CC74E6E56DC5050087B0C5F0C1FB1
:109EC0000CE30C1F08330423780E561C561750DB86
:109ED0007E63EE7E4B9C78221BDCEB9443E030D01B
:109EE00066FB20E0D400980278A26838BC983C2831
:109EF000E01CAE580813044E6E56DC90688DB8B85E
:109F0000580C2BC98C89B68CB551884EE80CDDB63F
:109F100041A48A4924DD20792419B46A1C0A301D21
:109F2000623F0A2BAE9C58636E1DA4DD8CC1026E8D
:109F3000601CCB38BC58780ED91CE9501C622B62CF
:109F4000BEDCDBA20C471437D4A250DCDC8C5BBE39
:109F50001FDCEB8C1BD013D0DC4C9BD47F1EBE2FA0
:109F60005467DCDB8C1BD013D0DC9BBE131EBE5EA3
:109F7000DC0C1350BEE0DCA0760C831C6247A29C74
:109F8000622FA222230AA2501CE0169CE0D2D268C3
:109F9000AED2D2284EA846F070E0D91C78D808D8A6
:109FA000F0AB781C221BDCEB6206569C622BC6DCF5
:109FB00014DBA05613860EDC50BEDE774277FABE65
:109FC000E3A6426F7E07A6FAD31EBBBE2766EBE36D
:109FD0001E0C13BEAE0C83A550E854670CAD235580
:109FE000BC410C1D024EE860E078E05CA01E0C1B3A
:109FF0009C131C222B62BEDCDB0C83144742F21F35
:10A000000404D00B7676130456DBD45F8C2F543FB8
:10A010003E63BE538483B8580C2B410CFD8A4EE836
:10A02000203077E0689D2244781CEA31B60EB8AA49
:10A03000AE3C68F8AAAE3CA838AAAE3CE8387C4AE8
:10A04000FC2878FE3B09B8B8D84C578C47D8DE3E80
:10A05000FE31B8F34484D8063020665746F0703895
:10A06000566637D91CA6E853D91C230841B0CE6DDB
:10A07000B81902B83C5806F804A0965C1427D4B668
:10A08000E30EF62B8C63DC541F66E333D4144FA627
:10A09000E32E8A3A5B0E0A061C2A4F0E7E8E9C0A1D
:10A0A000BA60E0AE56E346A38C431B66239A3A3768
:10A0B0000C1F4E7384762B0C4B069CA206BF1BEE26
:10A0C000608DB8CE08D528EEE9502E0EA0B8BCEEB3
:10A0D0007EE6C6FE1BDC508C752A5CF65B752C5543
:10A0E0002CD4DABE26E37B661FD4EB46BE3F752C2C
:10A0F000552CD41447BEE3D4141FA2E39CE04C4378
:10A100007E9EBE47DCD4E3DCA07E83A28C1BD013F2
:10A11000D0DCA26B552C4C752DF3BEB6AE60EE5D57
:10A120001E5C4C93063003562FC6FB462746FBC6E3
:10A130008606A637D4BEE31ED3752CD4143FBEE3E7
:10A14000A2D414EBD61B1C501CA63033A6E00D2A5B
:10A15000C6A6C6A6F306F6C70BE0DC201FD4EBA00C
:10A16000E0A28C1BD013D0DCA2E0A01E7E7E43EDCB
:10A1700028D91CEE2526DC10FEE0DCD0D07C70D97E
:10A180001CB07C70061C4AD36A2775B0AB3020DE49
:10A190007E23204926E8D309CA008CB3F12E461A43
:10A1A000AEBCFA1A3A30E63A303CC61C3CA2BC02BD
:10A1B000F6F6DE6BF6277CD90E7CAE0819BCF90EDC
:10A1C000F6CF75CAAE5851000E389C0A983CBEAE08
:10A1D0002838FC2684E6C67C287E7E677E01CBCDAF
:10A1E000C63000EECC4371CC66250E22C8EE66A3C5
:10A1F0000B00000000000000E55CBB6100A3E55C13
:10A200008838FC66E6876B1CC4E666664B0950100E
:10A21000841CEE013041A478901C8C476A550E4D89
:10A22000A43DA49DA48C1F7CAAB18CC1B0041D14B4
:10A2300025FEA550EED44B4670B87C588CED02B08C
:10A2400070EEF0E04EE8286AB3B83C58A020BC306D
:10A25000C1FC1CE000105B504B903BF3D023BD8E43
:10A26000103C064C23308006708C83AE1CE2EEEE70
:10A27000EEFC5C50303CE6E60E9CF83C5842A6589A
:10A2800044D91C302006861CB86AF3AA6A37C6E88F
:10A29000A8B8D3F87E60BEB03AE006B8588C233038
:10A2A00055737C584C3305BCEEE91BB8580CDFB035
:10A2B0005A3C0630667E679CD0FE431CD03EFE535F
:10A2C000FE4706580ECD90EE87B00EB85830505E5F
:10A2D0007C067C3076B1B5BCEEB85CCA46A80C2BC7
:10A2E000E21B1C229C5858CEBC30147C301C50BC45
:10A2F00058703059E2B858E0D8A686251CC1B03055
:10A30000E02D14041D1030E09C58BC0E66483D3A08
:10A3100044251C1D3C984D14987A30F6453AF6F6C3
:10A32000167A30163C5804D89CA298A2580C932157
:10A33000382B4C51370C33BD386520A30CB5374C46
:10A34000C9370CB78CCD378C8F5E7B3091AEFC9CBF
:10A35000425D1CAE4D32C1B0711C9DBC110C1D0282
:10A360008C1B0CB31538838C6B4CF53B0CF53B4CBC
:10A37000C9376520838C653BD32D38DB4C41370CC6
:10A380003381346520A3203C0A30836A7F3031E872
:10A390002D383B0C81356520C3B8FB0C3B8C678C9A
:10A3A0001B492406A6A6B8A6A803B8F8E806A6F195
:10A3B0003B4924B83C0E8CA730CD8C2FD91CD5320C
:10A3C000AAAEBCA89858889858653A4C5330AEAAA3
:10A3D000AEBCA80C571B301E0C0B668CF39C98D897
:10A3E00044D8581C3001AAAEBCA8C1B030D02D143E
:10A3F000A83060E8D53649249C98D848D858D91C4C
:10A40000BD1C090E042021386B4C778C5F0C1BBDE2
:10A410003865209B3030E81B30305E172EE83CBE9C
:10A42000FCE8953ABEFCD056E82138430C1BBD38F9
:10A430006520BBB8E04936BD1C1314201538BB306D
:10A4400020A8A8A86D7CDC100E304C66CF21B0DDB2
:10A45000AC49249C9858B81CD04C1B1CD0AE7CA294
:10A46000813A65209B3057BE5E2B2666DF03305451
:10A4700066E3834EBEFC1CD0E81538630C276520CC
:10A48000CB4EBEFCD0E81BB8E0301F43301F23305A
:10A490001FE8E8E8DDAC4924F81C98E8B83C588887
:10A4A0000898FC6D1C61001106DCD01C0EB87E58AB
:10A4B0004CE706F8425646BE47A6E606E6E646A341
:10A4C0009C98584C2330804686DDAC4924B80E8CCD
:10A4D000A76686E683DDAC4924B80E30C8E0C8CC58
:10A4E0003B66E3201938436D00C1B020492495BC78
:10A4F000110C9C98D84C3B4C1FAEBCD1A6D84E5CDE
:10A50000D070AEBCFE6D076645023040E6C8CC6D2B
:10A510000266DB04B1703C30E866FB59364924A57D
:10A52000BCB8D888D8A84E68D91C1538734CD13E11
:10A53000957CB35D1C8498A84936492478EEAB7CA1
:10A540004A68251CD91CB81B0CCB6520E36D7C0622
:10A55000251CB6BB1C307F6A93303A6A73302E6A72
:10A5600053302C6A3378EA1FAA0A3C68EED91C21C2
:10A57000B0B300000000000049248C931C78EE4B1F
:10A58000255068B85884986D1CB83C06300F6A296D
:10A590001A86D91CDDAC492478E0DCA01CF2251811
:10A5A00066301E1C6ACF78581598EE8FB858F83C64
:10A5B0009C580C5FB80E95BC110C810A4C37587C26
:10A5C0007048840C2B88B0A11C44B8D80C23584880
:10A5D00098589C584C4B1D3C4924980E1DBCB80EF5
:10A5E00086813A8C537C560EB858AE444D32587C16
:10A5F000A11CB8581C98BC580C5B30E61BD03B3AE9
:10A6000030E617E09010589C583532F8E6C1B04C4F
:10A61000A066664C13061EA1143020E8E060B0303E
:10A620003360B0303A70EEEEDADADAEEEE7CE0412A
:10A63000A4584DA4EDA4D8E05CF84A0EBEBE175055
:10A6400031020E8C2248E30130028C043EAEC2423D
:10A65000880480BE202C51C0202ECC0DA241A9AA76
:10A6600084F902C450020D3384537FBC3F000000C4
:10A6700004DC787777A50400DC4E0DC0AD80407017
:10A68000097E4410226323144F8CCCC30DC912944D
:10A690002379D33F0030004100E45C4806402001AC
:10A6A00080840B303417E33B03614413D323C19000
:10A6B0003331FAF4E4D2CA44F24DD490882374388A
:10A6C00080DFCFB3F3BC6C759792E288CFD3CE40D6
:10A6D00060C156211E168C74E8237655D4B8708854
:10A6E000323931D5D193F0E04D472E1FB82F2C8948
:10A6F000617420C240844410A0363513834E847F99
:10A7000064D84E55E88080D274124C1BE360A307D6
:10A71000800F28CC1B31841C91DC3E01FC279EC09D
:10A7200001316D820FEEFF13DFCFFBFC27D90F9EA7
:10A730001BC4301372813CF7F73CF743182F2EE30C
:10A7400088A4033C000010D544483012D070C57175
:10A750003003B017470C3C12C470CC030D8BCF8074
:10A7600002470C4DF348CCC44C7888871F871EC71E
:10A7700015335F848F2341C0084013CF4688CC0037
:10A78000253840CD7512080A0D21334073C40443A7
:10A7900083C700F8B1C44CFC72FC85BFDB87C404DE
:10A7A0000C23203123715CC00E193400C684891437
:10A7B000C3703CD1F3CF90E150CE6192DFF120A97C
:10A7C00055A34A15A82A166262403C8777F84804C8
:10A7D00091C33833C3400431F3B0F7C9C4E4C88D22
:10A7E000BBCB347038E013130741C43C73242323DC
:10A7F00078D1C43D215E141F13CAC53884C4AC731C
:10A800007C7CC8B51012024080D844C8441761252A
:10A8100020B33D20C623FCECD36EC8C1EC0B542002
:10A82000F94400154F1534551823FBF73284FC4CBE
:10A83000018B8773E1F81727FF0113C760D1927866
:10A84000AF17C60394D754508F8FF450E4E5A41F7C
:10A85000659A3D8A6BDFCB3C02CA23A3CA8DC94DE2
:10A8600088421320668633F3ACFC18FE43A28D0B9E
:10A8700011A2CA834813144140001733CC0C0CB208
:10A880006D33847D03C74F3CC48314F3303D14CA39
:10A8900020CED19110CC3F3CC03EFD2EF2C6F1EE51
:10A8A00098127337D673F4480C30CDC980CB3483FB
:10A8B000D88F2072CA2033DEF32003C48A6D145867
:10A8C000608219A8C5878C047931ACCCF07340CC78
:10A8D0001EC97667F2355B43440B1D38CF7ED0C16D
:10A8E00062733F0A01630E80B8B3007C8E3C05B0F2
:10A8F000F4D20310BB0030CD0058885CC574351A03
:10A9000037C3D2EDE2D03010A2633C03F10C4D0C02
:10A91000E1E8CF30FD1107723C7012948ECB902588
:10A92000A18C23091C480F8A036AC214130FE30386
:10A9300000A3388B2AA04C03C431CF0C0CC02C02CE
:10A9400000DE0AE238FC494000C0001D841057199F
:10A950005F3DC44EC47FC3FF5DD64BD524CE0358A4
:10A96000C8CA196281D117FB420808B2338443F583
:10A97000FC414CCC125328C634B952B9CE0350C452
:10A9800000C846F2CE7FE00932713233F100402236
:10A9900033870C8C2CC5C40123EF0B0725F6538499
:10A9A00034013390CC4C04E415AFCECC013931C71F
:10A9B00010733303188101C831313E1E080700F2BD
:10A9C000C38071FC63C5C8C4AC85332246E31F3B1A
:10A9D00038072083DC0741FC13C33F6F88F8DDCCC8
:10A9E0005050D573444C18C04C58F8F883CC713291
:10A9F000C3C10C070692BD78413BC4BD8F1304B39D
:10AA0000F810FA18F3274ED1C7C7C7C7EBA48C08B4
:10AA10000081ABE37B48B13013223AC467233F4344
:10AA200076321688C0F0303F32516308408F12F3FF
:10AA300057B0804BF0CC0CD3C0C4DBD8567F5D340C
:10AA4000F2430503414600000201030442470000AF
:10AA500027242120434800002825220044490000E3
:10AA6000292623004540000F800000981E19B0459C
:10AA70006C63AB130D08B0C964F0B8C9640EB01DA7
:10AA80006088C964CBAD130D08B0BEF053ABB063A2
:10AA9000840F0DB071643BADB0BE001D606902AAA9
:10AAA000B03560D3A5A6A6B035603102B21E18B08D
:10AAB0000EBBAFB061603B930201B05EE0930F0349
:10AAC0000151848808080176008435928C031201B4
:10AAD000595A86081301215E8E0913015184338E61
:10AAE0001301A99E8F141301715E8E01140151840C
:10AAF000AB9705091601910E008883900505023079
:10AB000007455A94130200418A940103012E8603DB
:10AB1000355A810C034E68A8E828E08F141398F08A
:10AB2000E0840C03410C511E900C03318A87120CF7
:10AB30000308CD5ECE0C03C15294130C034E28685B
:10AB4000A82B980C034EE8090299100F03958692E2
:10AB50002D04B00566870504715E84011207995EB5
:10AB6000840112895E8C0504A18A0000BD8A8513C8
:10AB7000047D56840E05870E0548015A9E12051461
:10AB80000E05B550B8E81102981E05B0296A960462
:10AB90000175BCE094030106B0B162BF0306AEAE1E
:10ABA000AE2BB12D181E0548B0296A833F03063528
:10ABB000586B98090688015A940E09882383120657
:10ABC000B0ED66BF1306155A833F13063558C30010
:10ABD00065A68F14079208B0C966930D0888CB87C5
:10ABE00013098481568C020C8E0CB0156E870F0CE5
:10ABF00088CB9605041341743B8E01050DF97095C1
:10AC000002902D1251842574BB86060FE0300999FD
:10AC10009C150861004106982F31B02D62922D10CD
:10AC200051840808D578CB8B030110018288032555
:10AC3000BEBEBEB01D606666B86960310285131085
:10AC4000CC2308ED04B10E94100D0F1210810E8468
:10AC50002D12B03166900F1413A50E0000751E98CA
:10AC60002B310E0CB0CD6E981413010C38EE238CE2
:10AC700003128CB5514E70EEE8B902930803B0FA96
:10AC80001BBEE8B38910A06964EE3A460BBE3C18BF
:10AC900098F01B8E0412F552840E12BD2A8E1412E7
:10ACA0000D9E9E129552890313015A8613295AABA1
:10ACB0004E2172AD4E88DB8705124E655A930F0305
:10ACC00051846B8E01145184438E0913518488087A
:10ACD000E17A851A0913555E94121113B0F9629442
:10ACE000131300818A8E0F4552AA14134950356000
:10ACF00043AB141349501D60B92EAD141398A0BE78
:10AD0000589BAF1413495061607B981E3031E16E3F
:10AD1000850E0F14795A97050916BD0EBF304D18D0
:10AD2000455ABF194D18A55ABF303C18E956BF30D7
:10AD30003D3C18255ABF193D3C18055A993E3C1810
:10AD4000F8AEB8E8AEA8B902BF193C18BD56BF307E
:10AD50003D18195ABF193D18515ABF303E18C556F3
:10AD6000BF193E18E156001D92910518830504484D
:10AD70002394030FB0E57E8E070913D13E8E0F0199
:10AD800088ED04711E86060F0184BB00009D7CAB1C
:10AD90000000201CE2E2E283B87CD84C1F48134438
:10ADA000D83C98A84451064DBCE27F410C8C3B84B2
:10ADB00098A8448506880CCB53410C04840C1F08CA
:10ADC000830498A809B8634EE6BCAEB90C004A5497
:10ADD0005C6FD6CA767D4D453C8C92989EA4AAB2F3
:10ADE000BBC2C8CC3AD1E0E7EDF3F901097C0E2BE8
:10ADF00014242D32353E4763545A6B717C82881A75
:10AE00009199324593779E28A4A620ACB94F30C8BB
:10AE1000A3DCE761EC4209FC600EC01F2E52575CB8
:10AE2000B265696D7177883792989EB0B9A8C1DA1A
:10AE30001582D0D60EDCE8EF1A14E208F6204CFC9E
:10AE4000286B2A00C88C2409E71892C29EA3E72722
:10AE50004DE0489EECB83C5808987CA8E04E70F84D
:10AE6000E085B5E0FFA0B0BE001D6070E0FA174EAF
:10AE7000A05CF6A06636761B26E0F61B4E2B4A6ACF
:10AE800056D4D4E04A545C6F0820F66D7132454FB9
:10AE900061ECDCC0A66B982A3A47ACCA63887C8216
:10AEA000987DAA2BD67654DC1A20E80E777C0E0EFD
:10AEB00099935730F3FC42F96052280114E237EFBE
:10AEC000B9B2B2E0141F1A3E155CBBD192FCED453D
:10AED0003CC8094D2EDAB0B9A8C19E2DD677A48CF6
:10AEE000716535D0E7FDBCEEC10295BE69CC886BBB
:10AEF000825A23F09D585C0EAEF0AE6E70D494CBA7
:10AF0000E0A5504332EC4E70783C0602E01CEA604B
:10AF10003CEB4CA491EE6E98AE6150AEA0FEA03E0C
:10AF2000337EE0002800D58818B550B902B550B579
:10AF3000504E7038AE7828B868F8A8AEE8E0A04E59
:10AF40006E60EEE047710E834140424348700E0050
:10AF5000784645676075E00017141110534C0F00D8
:10AF6000A8869C725259911C1815121A515CCF96E2
:10AF7000A94E9D76565A901B19161305575DD0851C
:10AF8000AC4F9E98505B08000C0C0C00555E077788
:10AF90000C0C0C0041460E204C515559617E0E5E42
:10AFA0002D2B2A2F42473D004D52565A62257F00D5
:10AFB0003734313043483F4B4E53572C631D9A0D65
:10AFC0003835322E44493A504F545805643C9B243E
:10AFD0003936337E454A08000C0C0C00653E078765
:10AFE0000C0C0C88EE61501BDA26F6EF1D64989469
:10AFF00017D44AFAEE58AE0EF09C4A5CEA271C5071
:10B000005C0E0A4AEEEEEE5C262666421FFA06E267
:10B0100047FC4626E21FFC468C13BE70981D605804
:10B020000E38A606DA661FFAE7461AB160F088986D
:10B03000AE8C538550A0B0EED33E1BBB85508C9791
:10B04000A0B03E7BCB8550EEAB630EB07BF8615079
:10B0500070B0EE53630EB0CBB8AEF86EB7CC6F4E97
:10B0600070B8D84C3FD88C27AD7062C102B8AEF82A
:10B070006E6760CC4341A4E5A8BD8C834E70B8D800
:10B080004CA7D88C3FAD70641BCEB0EE8F2BEE700A
:10B090002BCEAE00B0A8AE58711C98AEE0B0A5584B
:10B0A000B0AE4E7078BC46063C68E078BCAE300569
:10B0B00060061972EE38A02E6EFE433E2F385E3EBB
:10B0C000537EF61B56765CE2174E60EE0EF0386E3D
:10B0D000334C810BC90ACEF0AEE0CE7EFEBBA11888
:10B0E000CC60B8584C608CA00841B0B83C580848B7
:10B0F00098FCA8E046705CA0D4D4542FCE58E09CB5
:10B10000D251B5A3983C98FC58B83CD88C132E0C5F
:10B110001B2E2EBCF3755830057558300875583005
:10B120000758B8BCD80CA0C4D8584E30FFD8BC0EB5
:10B130007CA0BE60F1585B657387A1C90B3F8F157A
:10B14000B01A30A67E677E777E8F1ED8BEFBA6DB48
:10B15000E0D8A6F3E0D800A6EBE0D80000A6E3E034
:10B16000A95C98BC6D1EA95C88CBA95C08ABB83CF7
:10B17000588404E0044E70783C5A70AE38EEAE0E3F
:10B18000F0386E60EE0C134EF06EAE7BD55C542B37
:10B190001C52F0E04EF0D460AE7038DCDCDCDC93A6
:10B1A000D55C544B3CDC5010F070F03BD4C7AE7013
:10B1B00038DCAADCDC7C94E36B300870AEE0DCA009
:10B1C0005C38521CAEEE6FAE0E7038D494BB5CF29D
:10B1D00060DCE09CD4D4F2EBE048A670851458C142
:10B1E0005C4E708E783CC6B0C67F08CEAE584E3CE2
:10B1F000E6BCEE785A7AAEC39806374C098348E02D
:10B200007806BCEE5A3AAE5878E62BBC1AEEF0EE51
:10B21000AE0C330633AE2E6366E3AE70FABC1A3C56
:10B22000E638EE3C70662FEEF098EE41A4CC17267F
:10B230006E78063C063C063C686E4435BEB85848FD
:10B2400098A8E0004E1B4EBE5C501B2E7AD8984644
:10B250003E5ED81CD4763654E3EEEE6BD86EEE4BE1
:10B260002687D86E26DFAED80E23D8AE2BD8AED820
:10B270006E9E5E5B8E1E263BD8FCD86EA66E264B5D
:10B2800066CEBE1ED4D4C34EAE98EE2E7676760031
:10B29000CB2E7AD898463E5ED8065E139E0ED8DC3A
:10B2A000DC8E132E62F354CB98AED898FE1B66CE7C
:10B2B000AE5C4ABFEEAE5C0EE66B3A5BC62622DEA3
:10B2C0006EFA604E1EE0C6C36E63424F66EAE32E1E
:10B2D000FAAE4ED84E5C50EEAED8AE332E7AD89839
:10B2E000463EFA23D8465E139ED85EAE6E2E2BD80D
:10B2F000EE66D85C4E13228EF32EEED4D4D3AE98E5
:10B30000C1622EFAAE5E1BB5A23ECE6EEEEE0EEE22
:10B310005A0EEEE613BA4E9C4217AE8E4E6EDC50BD
:10B32000CE5322CEF34EEE94C963D4CABBA63BC320
:10B33000FEB7F6A70E8E1CEE8A5C4A9766061B3691
:10B34000E04E22CE3EEEC21BAA260EC223EE2EFBFC
:10B35000DE338A6E262EFB6A626B7E5BEE865A5E59
:10B360002A4EBAE04E709ECE68B8A606A8E07E7857
:10B37000EE68B8A67EBB4E7078FED8B8DED8E01D69
:10B38000648CB56298941FD44AC9622EFAAEDCCEA2
:10B39000D86ECEF66026E63B66EE1ED44ECF66E053
:10B3A00076FA3B367E13484623B6AE932EF0BEF0B7
:10B3B0001E06FA8EFB2EEE66DB8EB0B5604CA0FA50
:10B3C000A00EF81D620E6964EEB03D6055646962BE
:10B3D0000E55643560696475624E5C2650E04ED847
:10B3E0008564EECEE05C4ED01050D050105090D01E
:10B3F000D050D0505CE0FAA00E8E2626065C464760
:10B40000D4941BCEE066D34EDA8C93DCD4239D64B7
:10B410002BDC9D64D4D49D640ECE95620E9564DCC5
:10B42000D417DC9564EE4EEE93CA0A0ACAEAEA4AD9
:10B430008C330E060E46E04ACAEAEFE0BE6E8ED8A6
:10B44000988E4E27980EE026CB5C626EA5622EFA8F
:10B45000AE045E13081E1A6ECEE673CE5E7FDCD499
:10B4600094856B26DBF568A3B9685C336E66AE33F2
:10B470003A8EF32EEE66539CE22B62E24F225C235F
:10B48000AEFAAEE26B4E5C6A0E1C500C13A66E0E4A
:10B490004C1B09608C1BBE1E1162228EF32E543F82
:10B4A000EE66D4EE0BEE4C2B2968AE6EDC909CFA67
:10B4B0009BDCE233628ED89883268E7E9BCECECEE6
:10B4C000626E0E0C396153AE7EF32E7E982BD898A7
:10B4D0008EEEEEEE0E6ECEEE2798AEE066CB8ED8F8
:10B4E0002695626E5A5E0E0C1BE1644C1F01604192
:10B4F0006AEE5C90D0109050105010509050501048
:10B500000B4E54977A103AD4E7543F148F94CF548B
:10B51000FF9CD05C6B9050D05010D05010105090C9
:10B520005CEEE000D0501050D050101010D0D09CE5
:10B530008B1CD0D0101050D0509010DC2B5CD0D091
:10B54000D01010D0505CDB5CD0D0D0D0501C9B1CF5
:10B55000D0D0D09C6B2EFAAE8964B861500EF85EE4
:10B56000BB06BAF6330D62E6EB66EE5ADFE64FBE77
:10B570001EFEFE1EFE1388B85E2EFAAE08DA77D1E4
:10B5800064FA1B98FE072E11622EFAAE3E5EBFDAF9
:10B59000ABA606E683461BA6080E5E5A5C8A6222AC
:10B5A0008ED8988B5CCE62AE4E4D6E422766EEE32F
:10B5B000D8A5608B0160B32EFA0EAE0E26E6B35E00
:10B5C00057AEE5645C4EA60E6E3B08CB54F7D43EF6
:10B5D00026DB738E7EF3982EBE333E6EEED4940B34
:10B5E000AE8EEAEAEAAE9CD086C6E35C8EEEF568E3
:10B5F000A56CFAE3D4BB2E9C822E8EB5680C376EF8
:10B600008E6E2E6E1CA56CFA3B8EDBEEDB8E235EFF
:10B61000EF665E0C1BBE00B5600CCBD16449609830
:10B62000FE356AA6EEDB8E29686E5C1B2E62F34245
:10B6300026DCE08CA04ED8B968EE75620EB968B011
:10B640003D60EB00000000B0094648167616810BFD
:10B6500070C15A010C1008012004011401040114E6
:10B6600001200512120F120D050D0F1219200C0FDB
:10B6700013140E0F0E0518091314050E140E150CD5
:10B680000C101209160114050F1514200F062012B4
:10B69000010E07051001030B090E071412192001F2
:10B6A0000701090E1905130E0F12010D120F0D08D7
:10B6B000B060303A70BC5C50100EC1B0AE307A064B
:10B6C00056A856D349240CA08DBCF10E2170B8F0B9
:10B6D000B00E4C23BD701BB57069708D70B00E3507
:10B6E0006069704C23B9701BB17081704670F84C62
:10B6F0001F48EB0EB835606970AD7081700E6269DD
:10B7000070A9708D70F04E70F8280D729D585CEE27
:10B71000615060EE6670EE38D494B34E70138CA016
:10B72000BEBEBEE025601B1D60A550F05CE0D4D419
:10B73000D4D4D4604E7078BC26DCD4EB667038A0CC
:10B740005CE02170B5701D74F0BD700EA970EE4EF6
:10B7500070EE6162842170B1700EA97035608164F1
:10B760008C27B5701BBD700E3560BEBEC9643160DC
:10B77000A97069608164A9702EFA0E0960C9644DD0
:10B7800060FE890305608C60F088B9706BB0FA3395
:10B79000FE2388885EF00E35608964B80E3560D16E
:10B7A0006431600560F00EB8AE6160FADF0ECB8CDC
:10B7B0001F88E084E0AE88FE13485EF0B0FAA00E69
:10B7C000EBAD74E32E0E7AFE4B480C338C23848849
:10B7D000445CA606E6B177468FCECE235C62EE5778
:10B7E0000C0785640EA6AE3D7A0C0D633960AD740E
:10B7F0006ECE5C5A5E26E6433ED454D3EE3D7AD8F4
:10B800004E3ECE6BAED8221ED8AEAEBEEB1E2EAED6
:10B810008ECE93D83ED86EEED454B3EEBD606ED8C3
:10B82000469CEEE178EE132E62F38E42FA1BDC9B0F
:10B830000CE389640160A9640960D16449601E0554
:10B8400060B05ED898464D60A606E6A176B176DC7B
:10B850006654EB5EB5608C3BBEBE696431608C2B78
:10B86000696431604C87696466660075608C3F4E20
:10B870005C66503D604C13BE0C60F0E04E6E5E5452
:10B880006F94EFD427544F14679CD09CE0DC9090C9
:10B890001090509010505050905CE09094F3631CC6
:10B8A0005D789C505C109CE05C5D789C50DCE05CBA
:10B8B0005D785CE01C5D781CE00808AE0E2EBAFED8
:10B8C00043880C1B8C13485EEE4C457B8C2BAE0ED4
:10B8D000CECE4E5C1050EE66F62F661B268EEED84E
:10B8E00098EEEEEECEEEF69F8EFB2EEE66DB4EEE83
:10B8F00098EE4C1B8ECEEE8E5B2EEE98EE4C0BE649
:10B90000F7EEEB8C47884C1F48734463840CC38C60
:10B910001B842B881B8564436E8E00AD743B26F61A
:10B92000278EB32E6600B5604C5F98EE66006960A6
:10B9300069644960D8AE0E263B6EEE3BD454B72600
:10B94000E36E4EEEE178EE133E8EF32ED4CEEE543F
:10B950009BD88E8E4E5C50D89C90905B8A8ABEEBB2
:10B960001ED8AE4E2ED88E1E62ABAEFAAEFA0B7E4D
:10B97000661E8E9B980C4F8C3B396023B0D898463E
:10B980004D60F0D16449608C13F08C13BEF00B5EF7
:10B99000D8AE98AE0C1F8C1F866EDAC3D8A5600C8B
:10B9A0007B8964D1644960016005600C8739604C13
:10B9B000A0BEE04E5C6A560E8E0CA02300ED64FA29
:10B9C0000D63B04C9F0E1E4E5C66D01D604E501035
:10B9D000D0D0D010501090109C506960F60D62E0ED
:10B9E0001CA09C6E138E26F34EAEEEEEEEEEFCA087
:10B9F000A2E0CED454AB139C42E60D63B0221FDA12
:10BA0000EBAEA24E2E5C105CEE22270D622EA2F34E
:10BA1000A637EEEEEEFA9BAEB04A1C5090B562B07F
:10BA2000064E30557C067C30E04924B83CD88C1F4B
:10BA3000881384D87CA8E0302D9C58A051B698DC9F
:10BA4000D0CB06C010000000008000000000000401
:10BA5000808004200020030001080CC41431000D74
:10BA6000320003CC2B2890021000331490013002D6
:10BA70001028400C4070A201503998033290000405
:10BA800080000000C0000580000000005002420A53
:10BA9000C0350030300000DC000C8A04000068CCA7
:10BAA000390000001AA031C1030230B9C040000CB7
:10BAB00000008C001303C680088000B3210000083A
:10BAC00050C800320800088000080800040001D9AE
:10BAD000200C80C8A024933920000000C38D0608E4
:10BAE000306800033000F3012500084000901390F7
:10BAF0000343A64D8E0C30700319000000000300B4
:10BB0000000000003000030000003000C3D000003F
:10BB100004C0004200380C20153700F7CA89886F2E
:10BB2000C8CB02F333840090D00300000240D95503
:10BB30005555550595657116695AAAA9EAAA2AAA02
:10BB4000ABEFAE0354285A3FEFFCE3C38B000BEE80
:10BB50002A1E80FC00AF02542196A9C091EB95E506
:10BB6000286ABB05550AC467A25A0A99872352F569
:10BB70001188FE4F8D13EF6E4D0CBA3833CCCC20AC
:10BB800000002CDA5555555515001555150055551D
:10BB900015405555151555151000100000000000F2
:10BBA0000000100000401040101560D50CEBD10CC7
:10BBB000448A1212FFDA8C88221341418B63680C8D
:10BBC00088592062800C302003C0083E2CC100AF91
:10BBD000C4C0F8BC07B3CE204F11138087FC110AF4
:10BBE000A08A8028B820C938808C02FEECC17FFB77
:10BBF00038FF40C2BBCFE3684E4C4CBCFF4E5CA844
:10BC0000030095392292DDDB4B2FF470010F3FFFCB
:10BC1000E12040F204C631E2C8C8FF310AC88CCC2A
:10BC2000DF87200109C9BFF3EF0B1220131124C4D1
:10BC30000889E01B484322C4008F24003E46402C64
:10BC400026233C3F800314D0E76361134F13443431
:10BC50003619314D3B442A400129924FFE51D23CC6
:10BC600070212838CCFC3E400C04506029064CDB87
:10BC700060F74E010C002554D8F36063F7F187AAF2
:10BC8000C1FF8DE3224BDC7136EE03C5084A8E28D6
:10BC90008C927410CD0420812BCEEF898304004058
:10BCA000B74FB0072010224988B04ED24F861258A5
:10BCB000EFA11D0F3BC0323C3F11CCF21C6F9740EF
:10BCC00072FB423DB51F02300004E3844B12F47650
:10BCD0000BA2788CB30948006262173B0202862DE2
:10BCE00052B8FF11E25E5D50B2C46D0A100C4030D4
:10BCF000408668312658594D241452330029410793
:10BD0000182407202900A48002C0C4808CFB0B9556
:10BD100022000B788E00AC928400A75423CFF80940
:10BD20002044F63043C0B5EE5E298FF0735A2323CA
:10BD3000CEB400118C3CCC0B480C4442BC90393E34
:10BD40009320082100203D46000004004000001020
:10BD5000000004040001000001400000410441B95A
:10BD600015376CFCD1170304C3CC500C0C3308609E
:10BD7000C4CCD0CC800411230A3FC6C80080FFBFCA
:10BD800078EE8A3F034C0322CC3401304C2100234F
:10BD900030108028C33062E2500005C01088C0FC1B
:10BDA000A30438C58424B34DCDE02B2F043C1230BE
:10BDB00028DE4038647D1374C6374208403EF603DF
:10BDC0000000C1402194C83E312220022085006B32
:10BDD00084CEC804599D5316097D7F71D8C532E1C0
:10BDE000463B8038133040C785224E5523DD0E0573
:10BDF0004F4490CC1CDDBFB88B44A074125022126B
:10BE00009130970300767FF74C17DF8445CE98F288
:10BE1000D9491402C42012513222C900048C4A3B71
:10BE20004BFC8003050B0051482B0E31EC502DF0DC
:10BE3000DF38C813ECCCD8513D300451FBC73EF37A
:10BE40007F0CD00C441348AD7056390C51844E58B9
:10BE50004488A18095BCF0B3D5888A3E23E6D7AB51
:10BE6000AA0A704DA47E7C81BC8D8CB0AA398873DF
:10BE700009504E5B0CDF98EA2DBE0AFC4DA459A474
:10BE8000AA0A5829A48A41A4CC57980647662F02CB
:10BE90002762130AAEFCCA7004B00A8AB0CA70E501
:10BEA000A47CE21FF6B362BF62ABF62BF61BF67FF3
:10BEB0000C5B980A468D8C59A498AA58081304B0B4
:10BEC0000A7C060F662F02EF62DBF5A8B0AA70E5C8
:10BED000A4EA98701CA18C98622362626E6258B0CA
:10BEE0006A77558246FC708A980A29A4BD8C6ADB61
:10BEF00020B070389C5898700E388E8E1CB63FB6A5
:10BF0000DCDCDB027B4AF01C6A101C02BBA66670FC
:10BF10000A4EF0987CAA698C70389C98F04670782C
:10BF2000A6682E660DBA6670EEF0EEC34670781CF9
:10BF300010701C0A38E039883E37FEFEFEB1839847
:10BF40000A7CAA698CFC4DA4AA58B00A4DA4AA0A7E
:10BF500070E5A47C22DDAFE078E64E30C0587083F7
:10BF600070383E931CEA277CEA2371841B5584C6F3
:10BF700006B0666FE07EEEA0FEDC58B098701CB094
:10BF8000FC6A6F7C705584DE7985AB000000000090
:10BF9000000000000000000000B0702E70380E3B62
:10BFA000558498702E58AEF0E07858EE8B1598EEC8
:10BFB000810A4CEF0C27D588671CB1182BCCC3A97C
:10BFC00018AEBC3076767627D588437AFA85140683
:10BFD000DA1A3006098366E64670787066BCFA386D
:10BFE000D884D8F0BA3A301C62027CA23C0E3A30B7
:10BFF0000A7E27EEEECBEE3C7066EEAEF0EEBC664F
:10C000003FEEAEDC901C3B3C2606467078A6681CD2
:10C0100002C4BD8C09B81D02B8463C584484B0E047
:10C020006259A66EE0C461A4CAD844D885A43C0A6B
:10C03000ED1ACCA0D5886A66A08CE746E000000027
:10C0400000000000386B3823380338E338C338A3C6
:10C0500038FCE00038E0389338733853383338937D
:10C06000387CE03CE07CE07CE03CE086EA667038CE
:10C07000CAE086E6667038C64B42EAEAEA22E2E6A1
:10C080001FC61BC6360A1B261B62620A707C302044
:10C09000FCE0AAC37CD80CE92F758879A085140C24
:10C0A000CD0719027CD80CD12F758841A4F80C83D8
:10C0B000E6DDA965504C1346261366E8DD8CFBE6E9
:10C0C0001F26E865144C1938655026E8E55C7506AE
:10C0D0007858EE87CC1F41A4A1A48584CDA8884EB2
:10C0E00066480B15981CEE1B0C7B810AAE668F848C
:10C0F0000C731B884E704C47CCC98F41A4F8CD847B
:10C10000E844B04470198C4C27B066CB95A47CAA47
:10C11000FC61A47C0A4CA9A76550E62398ADA01D3C
:10C120000245BC110C711C2DA84CAFE0390C086005
:10C13000BC580CA00498DDD83BA188B030C570CCA9
:10C140001F4C1B79A055C42DA87BAA0A584888F516
:10C15000A898AA58334E59A48D8C986ACFE0AA8A21
:10C16000700A7C3083FCE0AE1C8A700E7C3080B399
:10C170001DA44BCC3F4E70F84666E8467038AA0ABC
:10C18000CC57E21322E21322E2132228E04CC982A8
:10C1900059A49DA4AA0A29A4AA5839883E5F488CAC
:10C1A000337EFEFEFEE3B0E098EE4DA4E5A41C6AEB
:10C1B0004F06E64E7005BC95BCCE581C0A59A439F2
:10C1C00088FCEE987C1D88EE7CEE6A461746363673
:10C1D0000627767613266A698C980A84F5AA584A47
:10C1E000174A4A23666262E6E6E6E61322CA101C94
:10C1F0000A986D8C98E0B9844C1187AE41A444F83C
:10C20000E633E5A84C3748655026E8DD8E30DADAAB
:10C21000DAEEEEE0B02BB03A707A258CF3B02BB0AA
:10C220003A707A258CA3B02BB03A707A258C53B033
:10C230002BB03A707A258C3A3A3A7CEEEEE0B07048
:10C240003C467CE066BC1C3A3076F6E7E23FEAC347
:10C25000666AAF03222222227B9C229F224F3A3A17
:10C26000301C22274E4C7F488EA9186EBCCB3A302A
:10C2700066AF7A7A3C1CE044448641A4CC3FC6BCFD
:10C28000584C1B4DA4E5A47C82E2DFE237E2AFE22A
:10C2900023DDAC93F68384763CAEBC9C98161C667A
:10C2A000673C0E29A48C29A54E70AAE03C0EBB5910
:10C2B000A4A3E2E736C736C739883EA74C2FED184E
:10C2C00048234C3B41A44DA4DD8C4E70E0E5A4888E
:10C2D0004B7D9C98CCBF4CAF4C9BCB5C42EE2B0E65
:10C2E0004E701C4A33AA7C8E8ED33C58681598EE4B
:10C2F0009B0C1FC4934C7B8CA758B8E683B8589806
:10C30000BC30E64BE0C81C0A1DA4A37D9C84110030
:10C310007EFE4B8D08063064069B8D901C0AB8E6A5
:10C32000B38A636A8686A644D190EE60810A46701D
:10C33000CC2FB8584C83B80A38AAFC0EF8FCAAE8EF
:10C34000AE0930ABEA0130091E04CC7F4C6F069871
:10C350004C8D900C870ABD8CC102CC330A0238BCCC
:10C360003A30A6B63A30FCE64738AACA0C4B8A3BAC
:10C37000384AD308EE41A43DA43DA4AA0A559CEE38
:10C38000530C3BEA49A4E5A4D6E63342EAEAEA22A2
:10C39000E2E697C6EAAD3CD86A8C8346425366987B
:10C3A0005846704BC63673A2A2B3AA62620DA4832C
:10C3B00008AD3C84D8064891900AD8662702331B02
:10C3C000061B04AA464223666262E6E6E6E61322FC
:10C3D000CAE641A4EDA47CC63CFAFE8D8C59A4CEDD
:10C3E0007C8D8CE5A4D8840C1388D88D8C980A7524
:10C3F00096190856A08A16CCC3468B02A6588C3BC9
:10C40000849806384A4B0638AACA237D900A499672
:10C4100046BBEAEA868638E2AAE2270DA48B4622CA
:10C4200022421B6653A2A23B047D905841A47098FF
:10C43000662702331B061B08AA0DA45697E6567FF3
:10C44000E68AB0AA0C1322EAEAEAE63C8D8C98252B
:10C45000961C903C1E98EE6A21B0001CF61B101C26
:10C46000EEEA3CEA23BE2F7B3CEAF358845C4E7034
:10C4700050FADA9C30583A30E6575CDA22A3E5E20B
:10C4800000D0881C3A308C97E63A30C61FE663E647
:10C490000EBC427CA67CCA70BCA6F6F6F6A33A3A5D
:10C4A0000E303C1E78AE7E3A3A306A677E8E8EFE43
:10C4B0002F4A2F44E34A97BC631C06461F4EE030C8
:10C4C000DF0647C63C020ABC059AA6FCCA221C70BD
:10C4D000BC0E98AE7A30EA8304D88C1B8408D86AE4
:10C4E0003F8E8E0C4F4A777C8C173C019A4ACF487E
:10C4F000B09C108C9F0E3C7A7AFAFAFADAFAFA9C1F
:10C5000098FAFA9C901CAA08E0781C101C0A703853
:10C510003CE6359AD5883ED37C62588ACAFCCA0E5E
:10C520004DA459A498EE6E6E1CE5A46E1C6A578E3D
:10C530008E986258E24B4A871CCE7C0ABCA34ACF35
:10C540004670CE7C0444E0441CCC1F4C3BF80E38B3
:10C55000AA7CEAEBC8E247C4EAEAEAE66FC628AE7C
:10C560004A7CE8F84666E8890AC6369B4E7048D38E
:10C57000C44CA0F846E8CC5795A43C0AED184435C5
:10C58000BEA918DB36AF335836C7369903CC1F4CDB
:10C59000A349A43DA41DB43C3E6B980E4670110CFB
:10C5A0001B19088C60D91CB8492676C32106785817
:10C5B000EE319EB8AAA81598EEA19268B806FDBC07
:10C5C000EE3BB80E0801AC1B95BCB806EEEE787CCD
:10C5D000EE0CFF78AE3CEE1C4DA459A4C1A46E1C19
:10C5E0006AA06E1C58EE8D8C1C98EAA0AE46708531
:10C5F0005201AC0C604ECAFCAA3C7EEE1DA0EE3F80
:10C60000706E85500982705838EEF0982606C3E0A7
:10C610008E85506E0801AE41A4CC2F46CA4602B8A2
:10C62000AAA8E08C9F061CC3300B0604B898A8A6E5
:10C630003CB0FC1C1086BC5C221B29CA30E6D3E04F
:10C6400000000000382338F338C338933863383398
:10C65000387CCA3CB3FCCA7C933CCA7C737CCA3C21
:10C66000537CCAFC333CCA7C13CAF01CE03CEA7C15
:10C6700023D588223803389338633833380338D3C6
:10C6800038A37300385B3833381B38EB38BB388B32
:10C69000387CEA3CEB7CC2D63CF0AA0A6E701C1BCC
:10C6A000FCEA7C733CEA7C537CEA3C337CEAFC1376
:10C6B000EACA47F0983EAE4670E011A0EED3A5A4BA
:10C6C00061A47C1D88E6132E698C980A3C1C237695
:10C6D000DCDC76E34E70786E682E70E638E66670C5
:10C6E000E6F0E62666A7E6AEF04EAAAE38AEF098C3
:10C6F00070384AF098A9A6980A4329A44685A47ED2
:10C7000058FEC74C13C809824E1C70786E700638EC
:10C71000EE2F30C006A04EE0CC8795A43C0AB18C29
:10C7200041AA2DA8669FE68BE841A4CC2FA1A4D8EE
:10C730004A2709501B29A4EDA47CC4483BFCCAAE7F
:10C74000D851ACD88AAE06B7662F02976A833CC927
:10C75000AABC08307A76EF3C7E45AAA3583C0A4D25
:10C76000A4EDA49CD08D8C98E041A4AAD8A1803CD3
:10C770001BD588D8063F6660021F62607C8ACAFCAF
:10C78000D83E67D83CCA7CD8447EFEFE1348E617E4
:10C790000A4ED8E04E70381CCC17E20AE01CAEE618
:10C7A000BD9E5A268F263B301D7C44D1026666FC16
:10C7B000084DA8C50278101C0A703988E627095070
:10C7C0003BD5883E6F4DA4E5A47CE21FF6D3B06A4A
:10C7D000DB11A0EE09829C101C3020F0B070660ABC
:10C7E00038D88408D8F04E70786668C4B18C01805F
:10C7F000BD9CC102CC53AE0EBC30E04DA459A4AADE
:10C800000A707C3021FCE0C6C2A0BB1CCCB76262BF
:10C81000627186CC8F1C23A237A2A22FA2E0A2A213
:10C82000A2A2A2AEE06EE0469C5845A4AE58707C31
:10C830009C98E61C3084FCE0C98C8ECE5C581E9916
:10C84000A49EFE5B3E3EBBF5A891A4CDA883FE95B9
:10C85000AAFEF75C224BFC261CE2CF8D8C8B22A714
:10C86000042217088DA4300F0C2391A453F5A82699
:10C8700091A48DA4CDA841A459A49DA4698C7C69E0
:10C880008C0C63FC61A40A4DA4DD8CF846E8C5025B
:10C89000FEFE37CEDC95A4BB5C62439CE2B790FC05
:10C8A0005DAA62839CE26FD0BB8DA4FEFE33FC26A2
:10C8B0001CE20FD01DA45378EEA091A478CECE68D0
:10C8C000C330F0AE58782366CECEEEE798AEE0F8EF
:10C8D000261F66E0044E6EA05CE070CCA795A40C09
:10C8E000133C52D84A431BD5883E33E6DF09503308
:10C8F00059A4E5A47CC4488AD80EB0CA70AED851F9
:10C90000ACD832AE724B06AF662F028F627BAEE3BD
:10C91000A9184EAA58AA0C41A4B0AAD80E442BE5D7
:10C92000A84C3F7298121B0ABFAE707C066550A0DF
:10C930001C4C60A6E8B00ADD8CF8E0C41BC488CCAF
:10C9400027E5A403AABC3A30F6EB3A3076EF7A76C4
:10C95000E11B488CA91A7ABBA24BAA626266700AD4
:10C96000387CA27C82E2FB2222A0F62BF61BF64F3B
:10C97000EACA8DAC82E25322223BF6ABF69BF68BE1
:10C9800029A43CCAE0E2EBE2FF36EF36DF8C258FCC
:10C990008DAC8DAC2237484C6029A429A48C173962
:10C9A00088ED1AE28B8DACA253AA101C66700A386F
:10C9B000FCE0A27CE0E22FF66051AE7660EA8DAC3E
:10C9C000EA76DB0304781C10581CFCCAEE30BF2644
:10C9D000AED8666BD8AE7070383E437E1E1C6A239C
:10C9E0007C6AE74A7F1C8A8AA6B63CCA087C7E130A
:10C9F0007CF03B0C234A3CB33CD84670D8E0B08373
:10CA0000D813AEFCEE707C1C0A3988E6CBD5883E84
:10CA1000DBFCAA0E584DA4E5A48A1CDA7C0AFC6A49
:10CA2000B74A57461CDA707C0EB0EE730C33466E74
:10CA30008D8C3B9808231C980A7C8B3020061CF8B0
:10CA40006AF3B8E07F616263646500600604050113
:10CA50000C1D7E0D4EF05C90308C3C0EE5A41CEA63
:10CA60005730051C426AB7C1B06B3CC1B0E02B6EB9
:10CA700030051C426A9F9E301F0C23E8BE3726BE3D
:10CA80001FE8EBE020DE6DBA5E270C71B049241C74
:10CA9000E5A43C8ED91C7C5675B0AB3080A330C069
:10CAA0008B0616303A66AB302C66A3302E66F73014
:10CAB0004006B8D84C5F8C4FD8DC101EDE7E335356
:10CAC000D8E83020DE237EBE7E70E8E016302006F7
:10CAD0009730600673A6D844D806B03070A646A03A
:10CAE000061B4E5C90101C30663322E3303A5B3CF0
:10CAF00056363B0E41A4C1A41C426A60FC5C021D78
:10CB0000B48E9C5806164670307F66851DCE0E1C6E
:10CB10007C66DD8FFC0E1DB48E9C58467051B4733C
:10CB2000E0200C604C3FC8CC37486D00CC603080B2
:10CB3000E666FBE030107030FDF09C4ADC909C9083
:10CB40005C901C90282828E049246E1CCCE5A66E39
:10CB5000C9A6381C3CEA6D591C387C0EF87C0AAE1C
:10CB600028B87C0AAEE8787C0AAEA8AE9C9868E04B
:10CB7000E6251CE656069C58B87CD804D83CA8F696
:10CB8000F62F46878CE70C23300BE08C273077E0BC
:10CB90003087E0301C66273054E09D580CC922894C
:10CBA000BA84B898A82B88B898A80CA78CAB307F0B
:10CBB000069C98E68D2666AF652083B83CD808D8D9
:10CBC0007CA8D9207924BD2025241D0239B478FE03
:10CBD00037FED91CB81B09B8469875B031B8638CBC
:10CBE00041BB41A4198C4E70D92041A41E8EE5A4EE
:10CBF0001CEA2B6E8DA41E46700C1B29B8E05CA0AD
:10CC000078A0FE7B9E60FEDE7E5B8C4BFE301A3190
:10CC1000B8B37E60FEE0D4577822AF145762DC5080
:10CC200058D4A099A4130C778CC37EB77EA7C314E5
:10CC3000B794A70C931CA0301B31B878F65329B8D1
:10CC40003BA08DA4042BA08DA4088D141D02301CC4
:10CC50009C5899A6307F66937846977EFE2F410CAC
:10CC6000BD8AAE8D8C29A44670AE68633E236520D4
:10CC7000E3AE99A4BE008B1E41A459A4BE1EFC1CA9
:10CC8000D08D8C7E0723781E9ED91C5EA0BEB8E393
:10CC9000301FE83020DE7E6F1E3E5E23E8BEE34696
:10CCA000F07068E05ED3B8580C373CD888D87CA8C0
:10CCB000469C9806307F667F781CEA3FDC10FED9E0
:10CCC0001C1B09B861B6851CDC10FEC1B051B6C989
:10CCD0008C9C987041A41E30F19C5899A4B09C582B
:10CCE00099A4AE7E6815BA4E705C105CD0100EB878
:10CCF000B03C06FAFA7C4638BCA606583C28E0E66A
:10CD0000174E7009503344A180AA70040A4DA4ED57
:10CD1000A4D80C2704D8330804D88D8CB00E3988D9
:10CD2000E603D5883ED7AA0A704DA40CEB08EDA403
:10CD30007CA24BAA626266700A387CA27C82E2976F
:10CD4000E2EFE277E263DDAC4BB0E60F700C4B41F3
:10CD5000A44E70E828DD8CB8584CA0D5885FE27FDF
:10CD6000E217365F364F59A4E5A47C22D7E38DAC99
:10CD70000BEDA47C563C8D8CE5A41C4AEECE8D8C2C
:10CD8000CE7C63E5A41C4AEECE8D8CCE7C1BA6FC2B
:10CD9000586E1DB41C980120C3AEBCD91C0C733A4C
:10CDA0003A3006A63C2EEEB9BC04D5124D14091239
:10CDB000D91CB9BCCE3C061EA114B81CD0E8661E16
:10CDC000A11463A6EE1C1084101C421F02889C1B39
:10CDD000DCDCB6EBE6161FDCD64E94602213E2B61E
:10CDE000F30EF88C17B858B0E0EE2798022398AEEF
:10CDF0004EF0E0CE70989801207B0C3FB858B0AE52
:10CE0000BCE06E4D9CCE0592810A4404040C47455B
:10CE1000A4E5A459A42B6E2DB46E66E66ED91C4C05
:10CE2000D9B0D9120C23EE58EE04D80C230804080C
:10CE3000D8E0BD1C18120F0D20E00000000000001B
:10CE400000000CB962204038238038C4F800C403C5
:10CE50009D1033D410D0CC0C0011802C2E122151F7
:10CE6000C04411713333809043A21A1F00358020D3
:10CE700093C1477F20C4A3612032E2CCA3C83849C4
:10CE80001C524981304443C8C64304224B1204F16A
:10CE9000EB0030388431000000A00091869B8CE3C9
:10CEA000321070D02A8348F420B806B3F836E2C9AD
:10CEB0000F0A92803D86330033E3C94D03DC50C135
:10CEC00083230300440400300C00C07C373B280C53
:10CED0000A5359CC8A6892C4BDCC0431BD4C0C0EA7
:10CEE00004E2A07838E00326143003DA203E180468
:10CEF00070483C4B40E000002920CD9C84FC92EE21
:10CF00002E4F87C0804CE14430D00F461263E4833B
:10CF1000E0384E1086E1330334141258D131B23464
:10CF20008A104D4004C0A0A20894D3206A153E0583
:10CF30003D0BE1322138FCD7913944E61099436426
:10CF40008E7A5572B4EBE27EAA2FAEEF8804E9AB7D
:10CF5000701248C4C87675C4BED2C4D03CC8E4E8D8
:10CF6000E2E1121A3180CB4E02C258F8F06F8E08FF
:10CF700008A57D6D41C308EA1433A4015FE083F284
:10CF800060438200C02C50CE0743710E6E4C8FF769
:10CF9000C40C0D06211895C54C4851A37B8DCE8D30
:10CFA000D7D40C138A5A851332020C836C3854C8B8
:10CFB000030C2CDED1C404F37FC49C46D74D41330F
:10CFC0004CCC3C0F6195D01805C2D2A0C47A84C164
:10CFD000E3121ECD4EB838910C51A57DA23EBE8CF9
:10CFE0003DD2704F60813B152E2DF67C3C70BC0805
:10CFF000A4561794824F240AE00A40330108CF2335
:10D00000F240F808BA08D92008553CE038ECA8FAF4
:10D010000C5021C4722208C7805E0808CFE1608EE0
:10D02000388E16620B622F880833C20F01E7A00802
:10D03000032823226060FE084B0087B8C3913F2776
:10D0400059227B000400008C00444400C820CB0D12
:10D05000C4CC8C28C404008C0C4AFA00111100883E
:10D06000093E064088508FEFB82BA0880F026082DF
:10D070004D3180B908E01A12CF000522EE07413386
:10D080008C3C0041F0F3DFD43ACAD5C843078D4049
:10D09000F3F30049515BECD038508380486C28C9C9
:10D0A0001C1132808C2CCE8CC094688C8B3B003051
:10D0B00040FD0C49520D500D40145D55373324C3CB
:10D0C0004902C3184A4C50D8821B64491331843337
:10D0D00011038204D0C03C09CC4B0EE0394F8EBB0B
:10D0E000B33EBE0749EFF1E22100414403880F231C
:10D0F0000F051024F3F30F015540C544CD03013C47
:10D1000013FC0C48E4EEAE11E1816ADC861EE110EE
:10D1100086D2ED238788181116CF704444301ADC6C
:10D12000878313B84C01847421983DCDF02034C915
:10D13000E0868D01008580438D30C40C2081036022
:10D140004861F4FF000000004C71B204FCE01801DB
:10D1500043C461BC13D30422336110447C7C4CF47F
:10D16000217B0C1F42FCC4C470D7F14CCCE3313896
:10D1700021E3103081F11008040CC2DEF228DFF93F
:10D18000611C2030D50148E23A7B1D76D411D304CE
:10D1900034F7773500B1C4714C2C48F0C74F128D6D
:10D1A00033C2FD0D3131A0301310B1108010200BAF
:10D1B000030A302A0A3204AC608A38CC3C23C2CC41
:10D1C0004C800A32C1141333F18E22020C22223217
:10D1D0007131E4436ACCF771203937EBFCD4DF4C72
:10D1E000312DCE1032CE880C41CC30830236DF5B3D
:10D1F00091D1B8C1E4008D3C4D0F140E4A4C20076C
:10D20000AA71DB511DA342A0C3FB102632B21ACA79
:10D21000083200BC0C008F0002D0805EC83423337B
:10D2200010F30F73DB2E0DDFCFF152F7D84B123A0C
:10D2300030000FC53043CBC810240C3341B4E43F59
:10D24000000E00401A24005D0B6E08060F380B67B5
:10D250000B5F02D702E202EA02F306340407010080
:10D2600002C102C801790089016E0122011701354E
:10D270000B010423040F0B440CE5056009FB00EED1
:10D2800009410054006902D0007A00710061000079
:10D29000850D09142018032D83322020050D091453
:10D2A0002D94101713C5DA810D0C010C0341E68D86
:10D2B0000C010C031289E6930D0C01120C03C9CE6C
:10D2C00000000000000000000000970F0404A140CF
:10D2D000F944694863C1B0981E7E3570DDAC656461
:10D2E00098310258300370C158CE6152814084D5C4
:10D2F0004CF88C13B86ED330200C3330188C1326B6
:10D30000E6A18804B17022D91CB8C6E86564ED8A2C
:10D31000389C4AE03E3E3E8A1E4E62EFCECAD47E24
:10D32000C31E4EAAE05830107030FBF0E8E0850DC7
:10D330000914D9688E7C5E61446948BB6ED9708BD4
:10D3400085140104D968754C694843C1B008F54893
:10D35000656498EEB94A97130C0312514C04E544E6
:10D360009B86010C031295445B514CF8BC6944FE4A
:10D37000A0DC50E097130E1512514C68E08940A8CC
:10D3800038A0FE1B5C8A0E9E1EB1644E46D95C5CC2
:10D3900019688D70CE0E5C7CEACED95C5C4AFA1FAF
:10D3A0004E5BA00E665C1BFAA642EBAE0E60E099E7
:10D3B000040DB8BCD844D87CA8E0990D04B8BCD8FA
:10D3C00048AB0E8E8EA04E5C504E4E9C3E3ED05CC6
:10D3D0004140603CE00408E0DCA046F0980670386C
:10D3E000F61366663C7E60BCA6BCDC100EC1B0AE17
:10D3F0005C900E46F03C70380C435C04F2277CA233
:10D40000E370D91C8EB07C7075B06E8E5E4B5CA2E2
:10D41000A39CA2AF7AD30CE361009CD2BB9CD2A0A8
:10D42000C1B0DC10FE04041B300B3C0E1CF86A1F5C
:10D43000BEE3B849243E616A856869547008A968EA
:10D44000E60670381CFC6A6A1E6A337E7E98A6580F
:10D45000B08148ED4E6954BE3E0165DB000045DAFF
:10D460000000000000006954F693E0DCA01CEE9878
:10D470002670380EA0F2A65EEBA6728940387C3288
:10D48000320000321F12EF662792B2939260981D0D
:10D4900068A6049870CE1C42F0861E81487E98C60D
:10D4A000BE6066EBF613263C5E9E9870380C134EF9
:10D4B000709853267038A670A6F066A60626AFC6EA
:10D4C00070B0F0BE33E0300870A6DCD09C1E387C13
:10D4D0004A3CEE60A6BE60A6067038BB8940387C28
:10D4E0004666E6A6260E4B361CE2172AA649687049
:10D4F000383E607E1C128B1C42F0935C0A6029FE51
:10D50000AB05140104D9CE93190104048DCE980DF6
:10D510000C010C0311E6B2310B0C03DD48449828D2
:10D52000E0B4320B0C03DD4848AB940B0C03DD4830
:10D53000846B84140B0C03DD488823514CAD727549
:10D540004C46178E30020C6BE01CA01C50509C30D7
:10D5500005721766884884DD6C0C0BDDAC4E3020FC
:10D560000EB8B8B8662F7EB86623D888D8E84924A4
:10D5700038D91C9C4A9EF9447E3570492659CA8583
:10D58000683389404EA8E0454A93000099CA08C113
:10D59000B0494400B9620058894068F858A8B80EEC
:10D5A0004EA07A606E1F8CA0A84E2828A82828E8D4
:10D5B000E828E8A82828E8A8E04970136BDD48A00F
:10D5C0000E3CAA7CC6A670663004062B301246BA02
:10D5D0009A4EA6BC01700EB01A9A70DAA5709A7CA9
:10D5E0002B816CA00E0E4924389C0AAE284A7C0E72
:10D5F0004E5C50D010101090504E5CD0905090DC8B
:10D600004140AEBC0E389C4ABC70BAA57070BC0ECE
:10D610004E1CD010903A5C49404E5C100E2BCE7AD6
:10D620001A23AE7C06B0A6705A0170BC30120EB040
:10D63000BA5A7A6606237AA646FCDA3C5CAA7C0EC5
:10D64000DD48694694030512120F034843850D090E
:10D65000140513444E7D4070CD6C49503C2EFCBBEC
:10D66000851401041405134E7E708140EEB5A25856
:10D67000CD6C44844950704570380EB0284CD34965
:10D680002478AECE3010956078AE68CEF0AE5C4EA9
:10D69000138A0A301095607858B075604E3004587F
:10D6A0003A3024BC4960709544A0EE1FA01B2D6049
:10D6B000B02560EE3961216CC4F57C856813E061AA
:10D6C000481CCAF972E0AEBC0EA01C30120A334AE4
:10D6D0002356134A16E004E0DCA005688EB03E77BE
:10D6E0007E497013730950EA0A4BAE3C0E1C12D1EE
:10D6F000501B84ABD8EE271CD2D3D54CB540EE4D91
:10D70000704E1C50501C0A1BCD4290901C0AD36EC8
:10D71000816C4E0E8D70CE4EFD50A0980EE09ED9BD
:10D720005C4D701363D95C8A8A4B30030455701BBF
:10D73000616A8A8A8A1ED95CA04E9C909C0A931CBE
:10D740003C0A73A05C99704E5CA5700E0E60E00EF2
:10D75000695013EBD95CDE7098067C6627B00E2BFF
:10D760006670C158CED95CFE23A03E2B6E6D50234F
:10D770004C670BD95CDEA05CFE138A0EB0FE138AE8
:10D78000AECE5E6F9E2146307A66FB61020404983D
:10D790001D5C5AE1080698467CA6BC58E01C9870AF
:10D7A00038E09713783CE64EC67CC63CEE514CC43C
:10D7B000780ED1E2B1640E681CE260CE3C58B96CC0
:10D7C0006100CCED57080C7F44E544CCCFE05CB55C
:10D7D000708C171CD85346F0987CB95844CECC377F
:10D7E000FE2BA03E7E538C2B2D548B23497063045B
:10D7F00060B1702208D91C495C638ECC4FE01C21BB
:10D800004CCCF55CA0CCCF6089406C9BF89CE27B53
:10D810004970CC1D70CC4F89403031E8F9561CF866
:10D82000EA23A8380E98BC62EBCCAFA2023C580C9D
:10D83000AF0844AEF544CC47214CE05C115C3B6042
:10D8400046F0301371648713847434857535867699
:10D8500036371882C21283C37300230B363636362E
:10D860003636363636134B237BFBFB6B53306E66F6
:10D87000FBF1568B030F0C039170E5EE995ABB0533
:10D88000D40D5449248142115AB95A855A0DD49164
:10D8900070A56CA0F9CE73AB8C374C73195C061C69
:10D8A00062131C4262315D33D38940F81C0CFFEADD
:10D8B000BF4EA8289B4C8FB570A88C1B28136858A6
:10D8C0000C2555F38C178C1F883B842B4CD730329A
:10D8D000155CA08C2FA6FB415E66134660315C315F
:10D8E0005488E54CAB8C9F4C8F0C1F0813042D54AF
:10D8F00004434C378C370CCF08A55A044C1F4813EF
:10D9000044989C421C4258C3155C044C374666B68A
:10D9100048933676DF1C862233A24C47C62B629C86
:10D9200086A244315C4CCF3154BB4C778940A83837
:10D93000700C2555987CB958B004F544987C70AEAD
:10D94000F0C8CC7B08488C2D55C8CC3BE01CF55C5E
:10D9500046F0983CA02660F61348315C7C26BC5803
:10D960008CE54D6100987C26167616577038AE9877
:10D97000F038AEF0986E4971F9560CA04C43C8CC03
:10D9800060A06020E0CCED57E006983C0CA03CE0A5
:10D990003C0C173C58E0302E0C1B303DE830128C0C
:10D9A0001B3004E8195CD95C065E3E4C1B3E234CE0
:10D9B00017E630307CB6163C761B301FE8E67EABAF
:10D9C000E0A0C1B0600C495CD95C6EE00C2B5E4BF2
:10D9D000D43B5E131C4C135C2BE01CA05E0EC1B04C
:10D9E0003E04885C421B3EC3EAE0DCA07EBB8304AD
:10D9F00091704C4FD8C9705C422F3E33D8885E3E40
:10DA0000FED91C7868786860E0EAA09C9A5E339A38
:10DA1000509C0290DEDE1790D95C13D07EF3D0D0FC
:10DA2000D0D0D0D0D0E0DCD08C7F0A9417904C2797
:10DA30006210135050DC0210CA683828380AAE2829
:10DA4000A046F0E09401030D0C017D681B79666629
:10DA5000A65E3E58C4440D54E0C170843D6404CDBC
:10DA6000B47B758CE06564E04871682B6564416443
:10DA7000E04544EBB068CDB42BE5AC8813847870F6
:10DA80003D64E065443B8CE5AD3D6413208C758DB1
:10DA9000E0208433985E580D54214C492498FE2B85
:10DAA000CC6F15684330FFCC3766EB235162203CC6
:10DAB00056063018662D5A308766D3309366FBC8F9
:10DAC000CC6100FB4E9C90CCA7601B7A1F7ACBF5F3
:10DAD0005A894858C17085641385644B1C20E2B78D
:10DAE0008C73E54C300671643570C28512C3001327
:10DAF0003383533BDBBBD14413037966E168E09C7D
:10DB00008301644249621B985E3E4962E54C2B30BA
:10DB1000087164803534C2858712C300CB033B3B58
:10DB20006333538B73EB1568E365203BF168E05C6E
:10DB3000E170844162F168C1B008ED48B344716896
:10DB4000008B294E8568668698663315C84D68CB6C
:10DB5000C658E02030F1CC256366E3E0E0080172AE
:10DB600001EE8841DE9870C4F57CB058E0000000FA
:10DB7000A09C4ED090CEFBE0B87CD88C6089028D02
:10DB80000C011A1918300289407D4070514CE83858
:10DB900088084D507C46EE173A70842689400EEE78
:10DBA0006B8899502B301AF1424E360ECFAE7C4620
:10DBB00068600948B0300446068C1B66367066A65D
:10DBC00058851406980667882626061384856823D8
:10DBD0008C97A188C1B0BD1C0E0F20120F0F0D38FD
:10DBE000F8214286C626704E7EF0C6704EDC9090BC
:10DBF0001090F004A96858B0C6260E2568869806CD
:10DC0000B0556898A658A670660638D87066D8F0E1
:10DC100026ABC6702658B0F65BF04670780E98704A
:10DC20002658AEF0B09C629F0948EE173AD870268D
:10DC3000D8F0BE3FA6667006388BD152982B14815F
:10DC400040CD6C2E5899501BB5A2A0DE1B8E0E70D5
:10DC5000984E5E330ED164AE734E9C501090D050EF
:10DC600010D090AE0E874570380EB00E286B860629
:10DC7000B05568C67038FC1CAA0C2F0A3967134AC5
:10DC80007CF026A604A568A6A6E0A6496870381C04
:10DC90003E607E12B3E0067038F61366663C46FCC2
:10DCA0000606E0514C4EF0E0DCA030C0085C905C11
:10DCB0000E13664E7078067BA60670383EAF7E6205
:10DCC000A0FC5646EE770CA0A398496870383E6FCA
:10DCD00098A658E0894833D144E07EA060B03AE08D
:10DCE0006954F69B982670383C05688D70CE0EBC42
:10DCF000555CD91CB83B4C604EBB514C8940383305
:10DD0000987038463C0E0430059C5A109010DCDCAC
:10DD1000DCDCA0FA5A13229AF33A0C534C2BC8CCF1
:10DD2000A023CCED576627D4BA73945BFA5A5CD023
:10DD3000905CFA4626139423FA10C3FCAA0E60E006
:10DD40008601140513514CE838288140EE83497050
:10DD50001B4E5BDC50AEFC1E1B261FE6EBBC894055
:10DD60003CA8E8E04EDC5050501090E084E80444B9
:10DD7000D828E83029E8E0EE514CE8380E4E70AE75
:10DD800068A0E09713140513417013339E048D505F
:10DD90001BB5A24D4C98DE1BA08E28E0B432050DB9
:10DDA00009140184887B850D091401843B851401C5
:10DDB0000401888444417013CBB87C1C50600691E8
:10DDC000704C23D88813D8492430260213A222D8B5
:10DDD00088D88C7B8662271CEAEA0604E948E2B30D
:10DDE00008A3068C4FC9705C4267DC906B095060D9
:10DDF000AE3C0E13FA4C47DCD0A25D6C6E4BD91CC6
:10DE00009C10D0A27CE89CA2BB8C608C603020610E
:10DE10006C30414C1B3050616C304D6E5851B6B671
:10DE2000A31C8C7FA25390909C5D6C6E167693D051
:10DE300090BBA2CF302F0C4B664C73B8D848D81B80
:10DE40004C3BE84B0EEE0E0EEECEEE0EE0CE300466
:10DE50006944A0E081400E3001A0A65C4636616BAB
:10DE60007606138A66F3E0A0A01CE0DCA04EB2CEDA
:10DE7000EE4EEEE0F16804E09C23E09C08A0C1B007
:10DE8000AE707C5E0EAD5C0C60D91CF8F8B00EED87
:10DE90004A7E7C1AFA5AA57013150E0D0F0E141532
:10DEA00005170504140815061209130114B01A30D9
:10DEB000E83ABEE3E09806C44924B8BCF6F6F6A0FA
:10DEC00088E004C5703059D866F31BC570301E0C4D
:10DED0001BCC8766DB2308C570302DD80C1BCC1FEC
:10DEE00066D3C458A60658E030107030FBF0A8384E
:10DEF000238940F8D8E0AE8444BC0E30121C0A7767
:10DF00006A53A0CA0A374A881B563348234ADF0699
:10DF100060AE3C0EE00E4E7078EE894078A0AE8E7A
:10DF20000E68E09713100F1413514C28E060FCB0FA
:10DF30007CA0EE0E1CD09050A636369C133AA2F36D
:10DF40008E76E3AEBC0EDA3CDAB0BA5A707A9A4EEC
:10DF50005C109C4140AE3C0E3C5A4E1C50D01050C0
:10DF60009010AEDACEFC70B01AE05D1C0C13C884C1
:10DF700098A8150C711EE1688CD972E0C97020E078
:10DF8000894038A02E2E60E0000000000000000054
:10DF900000000000000000000000000000080B6C02
:10DFA000BB8CAB0E4E70B89CA2A8B5708C1B585B96
:10DFB0004C43C1B048042BA16C04448461760458DE
:10DFC0008940594C38580CC76C2F4C517EDBE8F80F
:10DFD000D84C4D76D80C1F4CC34670B83CD80C7347
:10DFE0008C674C57D80C7BC97491704898A828E866
:10DFF000381CEA578CA30568EA274E907BF83CFE54
:10E00000CFFEBF603D5BCC4B3B4E36682B8540441A
:10E01000E804D8A8288940BD6C8804440884448456
:10E02000608940F8D88C3BD83038E8FD7E0C27D882
:10E03000D57E58483031E8757A980670389C62CFA2
:10E04000F61366663C1EA6067038AE7E1B4E23266F
:10E050007038AEE0DCA05CEE5D7AF237B2EEEE7CBA
:10E06000D37C06305EA61C6A873C5CB27C0E4EB246
:10E07000EEEE521B3CD31CEE25510E917004E6C609
:10E080001CEA4BE008F174A8E8557E3C305E6A4714
:10E090008E8E8CBFCC87A3FE97C68C7F4C6FD844E6
:10E0A000CCD36554D0F0F9700D7EC6A16C49240C18
:10E0B00037B8D844D8A8AE6841683B8DE2F174A85F
:10E0C000E8CC99745D1C0C330498A809B8BC58843A
:10E0D000983CA87858EE091E44D5420C676554D088
:10E0E000F09888BC983C589974E020F97098BC5816
:10E0F0004C93C1B0BD1C14090D051220010C011276
:10E100000D205345441333C17098BC5846F06666E1
:10E11000FB610098DC1044E05830F1CCFF66EB2046
:10E1200030264C2B08FD7046CC9F66EB987E4B4CFE
:10E130001F482B488C979170A56C6B2020441C586D
:10E140003C1C0A49CA30C36A8B2E4C4544000D540E
:10E150006544004666CC3766EB0D54411C4C5F9C11
:10E160009856063072665F4CFBD57E8C6B480D7CF2
:10E17000CB4168BB98E3970F0E0D0C01514C88C43E
:10E1800008486085684B2315684389400EDB66317B
:10E19000687038E6463C0E8940F9740E630C474CB3
:10E1A0003F8C271CC217D5764C43F8D88C1B58E0FF
:10E1B00058AEA8E83038E84C60E00C132049244CF5
:10E1C000A7CC091F8C8B91704C37D88C53C502603B
:10E1D0003D5BC974F90C9170048498A82860A05D17
:10E1E0001C98CD9E58B8EE514C6C9B385888989C22
:10E1F000C2285D1C089842A84B4D4C38580484D95D
:10E200001C783C8940A8FE63084E2B00E080E02E7D
:10E210006889CE4CEBA56C33587D6813DBDC90F03D
:10E2200091708CA76148D6F970736576817ED96844
:10E23000C97071BAD57EE976008B93CBD3DB00032E
:10E24000320D14CE000000000000000000000000AD
:10E2500000000000000000000000000000000000BE
:10E260000400000000006C454C54434D6130763191
:10E270004C4C8C4CC1CC34CAAAF4BD031FC60F60F1
:10E280004811100066C4781400404503401794EB11
:10E2900000D4DF281B505047BB402060CD3D3930B3
:10E2A000B30FCCDC4B45DA6707C225523BE40D17B0
:10E2B00023307233300173171992E4E3C4793F7D40
:10E2C00060554024A348451455922000508E404A82
:10E2D000DEC7B1427CF45845324211EDE291008430
:10E2E00082183D621F2246E435C9C708060B94B860
:10E2F000FC3838000400020000C07503700D700E79
:10E30000C07999CD2144688C43D910FDD3B31F8EB9
:10E3100050544871300DD21847374FA8C3E0129BB4
:10E32000C4139A4843315140140AA790161A425810
:10E330001225050729C05104E961838D0150118818
:10E34000137A71560080008018642B00006242E44A
:10E35000C61559481122B05884214406012921804C
:10E360004253B16D4D79CC4C3C7220125843C531AB
:10E370004950061136063D6474670E11D01311F62C
:10E3800043423C3E5190798704E5501A90281C3E48
:10E39000E16288F454B848C554429F0C0388D434D1
:10E3A000242344F225D28109C71972A232044406FB
:10E3B0004DC1405D9C371CB6DD05353DD50E91261F
:10E3C0003405A61C040000000050AAAA5645851773
:10E3D00000069754CC998911501ED521961D5B33A8
:10E3E000B72DF3163E7719A53409564948885810B9
:10E3F000C210C004914520A1BF00E3536595375872
:10E400001944293E393D501CAA504A92A4344282F4
:10E410006DD5F2277F17CE091D12C7C44521481CB0
:10E420009311EF3352043033002134C623334E1698
:10E43000DB03830C8040CF1708042E1230801001BC
:10E440001F0004F0005050605B1294719219441A3E
:10E45000681820E48111732E51556463F4782414F4
:10E46000576CF98BC8843851445398464100C0809A
:10E47000724C06D154587410000004BC600A066443
:10E48000D978675C15CDD4F479B92790C444030AD0
:10E49000F5B70B008419356F23B2967C84E1336A9B
:10E4A000844D1249CD3A57333300601F288AA82083
:10E4B0001458515484469A8F868896862C26A6191D
:10E4C000685C80511DA01835109015047F850914D3
:10E4D000C2808618554C09EE9F488D763112ED1199
:10E4E0003E24EE43DE5422D1C4DD6625291E6D365E
:10E4F000DF5C07095684F52F6017F2F3C92F10056A
:10E500000EB0E400D4644280818877CE08D90777C2
:10E510003035213A0004744025CA00C000C00030E4
:10E5200010CE99C570D4E03F4F1F1610D823981015
:10E53000837030037F3CC745C405403EC11F34DEB5
:10E5400001F237FC65BD1FE556C86AC2BE84C0D55E
:10E5500026023220990FD365550000000000E4DB4D
:10E56000DF31D55FA54E458C539531BEF4617C1CDF
:10E570000F553C63134C7C428772483200D44B08E1
:10E5800052E8D43B858100E561462545102EA32F36
:10E590006192F487EA0000000000D44C786C3330BC
:10E5A00009D957579D83357303E17F541319DF2C25
:10E5B00072427048F5601CF11D6D0B1ECF01C13514
:10E5C00081952C5247828002B226FC5FF03B073FC8
:10E5D000BE93098712DA311F4E3030565B05853CF9
:10E5E0008F46104A02FCF4B3398AD6461379D530E7
:10E5F0000300008801D5AC4BA6C5F82D15E3B9780A
:10E6000066D406DCC4805107BE57C0500C94531B1F
:10E610000100D56281719009D8D108CB7EC0F38307
:10E62000013B473863304C4561FE89344D7D7F2482
:10E63000CE57FBE41D40B70D9315ABF6665D6654EF
:10E6400056FC0B880304050A08060BFF0209070D98
:10E65000010C00FF44697370206F66660D0A00426A
:10E660005400555352004700524144005348494614
:10E670005400300032003300340050474D00414C0C
:10E68000504841005FE6000062E6000066E60000D8
:10E6900068E600006CE6000072E600001B5F000008
:10E6A00074E6000076E6000078E600007AE60000F6
:10E6B0007EE60000000C1C2030484C50545860701E
:10E6C00005000000FFFFFFFF4D000000FFFFFFFF00
:08E6D0000F000000F40100003E
:00000001FF
